:020000040801F1
:10020000A8D1012071040108757A0108BD540108C4
:10021000A5790108C50D010859D3010800000000A7
:10022000000000000000000000000000DD8E01085A
:10023000FD1501080000000001050108A5A901083D
:100240008B0401088B0401088B0401088B0401084E
:100250008B0401088B0401088B0401088B0401083E
:100260008B0401088B0401088B0401088B0401082E
:10027000BD0F0108CD0F0108DD0F0108ED0F0108CA
:100280008B0401088B040108A90801088B040108EC
:100290008B0401088B0401088B0401088B040108FE
:1002A0008B04010885AE010875AE01088B040108B6
:1002B00095AE01088B0401088B0401088B0401082A
:1002C0008B0401088B0401088B0401088B040108CE
:1002D0008B0401088B0401088B0401088B040108BE
:1002E0008B0401088B0401088B0401088B040108AE
:1002F0008B0401088B0401088B0401088B0401089E
:100300008B0401088B0401088B0401088B0401088D
:100310008B0401088B040108A5AE0108B5AE0108E5
:100320000110010819100108551001086510010895
:100330008B0401088B0401088B0401088B0401085D
:100340008B0401088B0401088B0401088B0401084D
:100350008B0401087D1001089D1001088B04010821
:100360008B0401088B0401088B0401088B0401082D
:100370008B0401088B0401088B04010800000000B5
:100380008B0401088B04010800F002F800F060F80B
:100390000AA090E8000C82448344AAF10107DA45E0
:1003A00001D100F055F8AFF2090EBAE80F0013F0D2
:1003B000010F18BFFB1A43F001031847BCFF0000F0
:1003C000DCFF000010F8013B0A4413F0030408BFEF
:1003D00010F8014B1D1108BF10F8015B641E05D019
:1003E00010F8016B641E01F8016BF9D1002D15D0D6
:1003F00010F8014B03F00C030C2BA1EB04040ABF13
:1004000010F8013BA4EB8314A4EB032405F10103D2
:1004100014F8016B5B1E01F8016BF9D5914238BFEE
:1004200010F8013BD1D3704700230024002500269B
:10043000103A28BF78C1FBD8520728BF30C148BF47
:100440000B6070471FB50FF0C8FD1FBD10B510BD84
:1004500000F0E8F91146FFF7F5FF0EF0D7FE00F0C7
:1004600006FA03B4FFF7F2FF03BC00F009FA00003C
:100470000948804709480047FEE7FEE7FEE7FEE738
:10048000FEE7FEE7FEE7FEE7FEE7FEE70448054974
:10049000054A064B70470000BDAA01088903010800
:1004A000A8690120A8D10120A8710120A87101200C
:1004B000EFF3108072B6704780F310887047264CB7
:1004C0004FF6FF7525604FF0000484F30988234C34
:1004D0004FF001052570224C4FF08055256062B623
:1004E000FEE730B41E4C4FF08055256030BC70479D
:1004F00030B41B4C4FF08055256030BC704700BFB6
:1005000072B6EFF3098050B11EF0100F08BF20ED56
:10051000108A203880E8F00F12490968086000B599
:10052000114880475DF804EB104811490A780270C1
:100530000C4810490A680260106890E8F00F2030FB
:100540001EF0100F08BFB0EC108A80F309884EF03F
:10055000040E62B6704700BF22ED00E05206002094
:1005600004ED00E0580600206186010847060020DF
:10057000480600206006002053EA020C00F0698063
:100580002DE9F04B4FF00006002B1FBFB3FA83F5A7
:1005900003FA05F424FA05F65E4012BF1643B2FAD8
:1005A00082F502FA05F4C5F120051EBF22FA05FC0A
:1005B00044EA0C04203556EA044C4FEA144418BFB0
:1005C000641C4FF000084FF00009904271EB030CDF
:1005D00039D3002919BFB1FA81F701FA07F6B0FA49
:1005E00080F700FA07F6C7F120071EBF20FA07FCC4
:1005F00046EA0C062037B6FBF4FCA7EB0507103FD4
:1006000007F01F0BCBF120060CFA0BFB2CFA06F6B9
:1006100044BFB3460026202FA4BF5E464FF0000B18
:100620005BEA060C08BF4FF0010B19EB0B09ABFBA3
:10063000027C48EB0608C01B06FB02CC0BFB03CC7C
:1006400071EB0C01C1E70B46024641464846BDE846
:10065000F08B13B54FF000004FF00001AFF30080B6
:10066000BDE81C407047032A40F2308010F0030CB4
:1006700000F0158011F8013BBCF1020F624498BFF5
:1006800011F801CB00F8013B38BF11F8013BA2F192
:10069000040298BF00F801CB38BF00F8013B11F00D
:1006A000030300F08480083AC0F0088051F8043B4E
:1006B000083A51F804CBA0E80810F5E7121D5CBF1A
:1006C00051F8043B40F8043BAFF30080D20724BF4D
:1006D00011F8013B11F801CB48BF11F8012B24BFE1
:1006E00000F8013B00F801CB48BF00F8012B704730
:1006F00002F0FF0343EA032242EA024200F002B89A
:100700004FF000020429C0F0128010F0030C00F03A
:100710001B80CCF1040CBCF1020F18BF00F8012BB8
:10072000A8BF20F8022BA1EB0C0100F00DB85FEA86
:10073000C17C24BF00F8012B00F8012B48BF00F852
:10074000012B70474FF0000200B5134694469646C1
:10075000203922BFA0E80C50A0E80C50B1F12001D4
:10076000BFF4F7AF090728BFA0E80C5048BF0CC082
:100770005DF804EB890028BF40F8042B08BF7047E0
:1007800048BF20F8022B11F0804F18BF00F8012B52
:10079000704770477047704710B500F03BF800682D
:1007A00010BD10B5044600F035F8046010BD10B55A
:1007B000203AC0F00B80B1E81850203AA0E8185059
:1007C000B1E81850A0E81850BFF4F5AF5FEA027C1A
:1007D00024BFB1E81850A0E8185044BF18C918C089
:1007E000BDE810405FEA827C24BF51F8043B40F82A
:1007F000043B08BF7047D20728BF31F8023B48BF0F
:1008000011F8012B28BF20F8023B48BF00F8012B4C
:100810007047000000487047446901200048704755
:10082000446901207546FFF7F9FFAE4605006946A9
:10083000534620F00700854618B020B5FFF726FE86
:10084000BDE820404FF000064FF000074FF00008D1
:100850004FF0000B21F00701AC46ACE8C009ACE852
:10086000C009ACE8C009ACE8C0098D46704710B5B6
:100870000446AFF300802046BDE81040FFF7F1BD0D
:1008800001491820ABBEFEE72600020070470000B9
:1008900010B50820034908700821012000F0BAF8BB
:1008A00010BD00000600002010B5024801F063FFF3
:1008B00010BD00005461012054494A6822F44032BE
:1008C0004A604A6843681A434A600268526822F4E0
:1008D000807203685A6002685368026943EA022220
:1008E00003685A600268526822F0407203685A60D6
:1008F0000268526883681A4303685A600268926803
:1009000022F4006203689A6002689268C3681A431E
:1009100003689A603E4B826A9A4218D002689268D5
:1009200022F0706203689A6002689268836A1A43D0
:1009300003689A600268926822F0405203689A60E5
:1009400002689268C36A1A4303689A600BE00268FF
:10095000926822F0706203689A600268926822F0DE
:10096000405203689A600268926822F002020368AB
:100970009A6002689368826943EA420203689A6057
:10098000026AA2B10268526842F4006203685A60C7
:100990000268526822F4604203685A600268536831
:1009A000426A521E43EA423203685A6005E0026816
:1009B000526822F4006203685A600268D26A22F424
:1009C00070020368DA620268D36A828B521E43EABD
:1009D00002520368DA620268926822F400720368C5
:1009E0009A6002689368026B43EA422203689A6045
:1009F0000268926822F4806203689A6002689368D1
:100A0000426943EA822203689A60704700230140EA
:100A10000100000F70B504460D460948056001202D
:100A2000074948608860012C08D1064801F06EFD36
:100A300008B100F0EFFD034801F0F0FF70BD0000C9
:100A40009C6101205461012030B502460020002144
:100A500000BFDAE00020CCE032B1012A2ED0022A19
:100A600058D0032A7DD185E06D4B9B7A0B44C3EBB4
:100A700003136C4C04EB0313694CE47A044433F81D
:100A8000243001EB8104684D05EB441424F8203038
:100A9000634B9B7A0B44C3EB0313624C04EB0313CD
:100AA0005F4CE47A044403EB84039B7801EB8104FC
:100AB00005EB441404EB8004A37097E0584B9B7A39
:100AC0005B1E5B1AC3EB0313564C04EB0313544C2D
:100AD000E47A044433F8243001EB8104524D05EBF1
:100AE000441424F820304E4B9B7A5B1E5B1AC3EBF8
:100AF00003134C4C04EB0313494CE47A044403EB1A
:100B000084039B7801EB810405EB441404EB80041F
:100B1000A3706BE0424B9B7A5B1E5B1AC3EB031323
:100B2000404C04EB03143E4BDB7A5B1E1B1A34F87B
:100B3000233001EB81043C4D05EB441424F82030B4
:100B4000374B9B7A5B1E5B1AC3EB0313354C04EBEC
:100B50000314334BDB7A5B1E1B1A04EB83039B7875
:100B600000E033E001EB810405EB441404EB800466
:100B7000A3703BE02A4B9B7A0B44C3EB0313294C35
:100B800004EB0314264BDB7A5B1E1B1A34F823306C
:100B900001EB8104244D05EB441424F82030204B54
:100BA0009B7A0B44C3EB03131E4C04EB03141C4B46
:100BB000DB7A5B1E1B1A04EB83039B7801EB810439
:100BC00005EB441404EB8004A3700FE0002301EB59
:100BD0008104154D05EB441424F8203001EB810409
:100BE00005EB441404EB8004A37000BF00BF431C5A
:100BF00098B202EB82030D4C04EB4303DB795B1CE0
:100C000083423FF729AF4B1C99B202EB8203074C9A
:100C100004EB43035B795B1C8B423FF71BAF30BD9A
:100C2000ECE700205801012058E80020A8D9002056
:100C300030B5012806D002282FD003285AD0042826
:100C40007ED188E001EB81035B4C04EB431333F866
:100C500022305A4CA47A0C44C4EB0414584D05EBD2
:100C60000414564DED7A154424F8253001EB810328
:100C7000514C04EB431303EB82039B784F4CA47A53
:100C80000C44C4EB04144E4D05EB04144B4DED7AAB
:100C9000154404EB8504A3708BE001EB8103464C03
:100CA00004EB431333F82240444B9B7A5B1E5B1AE0
:100CB000C3EB0313424D05EB0313404DED7A15448E
:100CC00023F8254001EB81033B4C04EB431303EB7A
:100CD00082039C78394B9B7A5B1E5B1AC3EB031330
:100CE000374D05EB0313354DED7A154403EB8503C2
:100CF0009C705EE001EB81032F4C04EB431333F84F
:100D000022402E4B9B7A5B1E5B1AC3EB03132C4DC8
:100D100005EB0315294BDB7A5B1E9B1A25F8234054
:100D200001EB8103244C04EB431303EB82039C7817
:100D3000224B9B7A5B1E5B1AC3EB0313204D00E032
:100D400036E005EB03151D4BDB7A5B1E9B1A05EBAA
:100D500083039C702DE001EB8103174C04EB4313DC
:100D600033F82240154B9B7A0B44C3EB0313144D0D
:100D700005EB0315114BDB7A5B1E9B1A25F823400C
:100D800001EB81030C4C04EB431303EB82039C78CF
:100D90000A4B9B7A0B44C3EB0313094D05EB031578
:100DA000064BDB7A5B1E9B1A05EB83039C7000E00D
:100DB00000BF00BF30BD000058E80020ECE7002075
:100DC0005801012010B50448008840F0080002498D
:100DD000088000F0D3FF10BD8E06002030B58DB026
:100DE0000446182107A8FFF7ADFC182101A8FFF75A
:100DF000A9FC002503208DF81C0023208DF81D0080
:100E000001208DF81E00124800788DF81F0011484F
:100E10000068000E8DF820000E480068000C8DF868
:100E200021000C480088000A8DF82200094800784B
:100E30008DF82300022301AA082107A8009406F0D8
:100E400041FE0546294601A800F09AFD0DB030BDCF
:100E5000780600207C0600207047000030B58DB079
:100E60000446182107A8FFF76DFC182101A8FFF719
:100E700069FC002503208DF81C0021208DF81D0041
:100E800001208DF81E00124800788DF81F001148CF
:100E90000068000E8DF820000E480068000C8DF8E8
:100EA00021000C480088000A8DF8220009480078CB
:100EB0008DF82300022301AA082107A8009406F058
:100EC00001FE0546294601A800F05AFD0DB030BDCF
:100ED000780600207C06002002468A4206D9501A75
:100EE000FA2801D2002070470120FCE7881AFA286E
:100EF00001D20020F7E70120F5E7F0B505460E46E0
:100F0000002400219A4201DA0220F0BD002412E000
:100F1000002107E06018285C775CB84200D003E04D
:100F2000481CC1B29942F5DB00BF994201D10120B2
:100F3000EBE7601CC4B2D01AA042E9DA0220E4E771
:100F400090ED000AD1ED000A20EE200AD0ED010A52
:100F500091ED011A00EE810AD0ED020A91ED021A1C
:100F600000EE810A82ED000A90ED030AD1ED000A3D
:100F700020EE200AD0ED040A91ED011A00EE810A5C
:100F8000D0ED050A91ED021A00EE810A82ED010A08
:100F900090ED060AD1ED000A20EE200AD0ED070AF6
:100FA00091ED011A00EE810AD0ED080A91ED021AC6
:100FB00000EE810A82ED020A7047000010B5024877
:100FC00001F0FAFD10BD0000B867012010B502481D
:100FD00001F0F2FD10BD00007865012010B5024857
:100FE00001F0EAFD10BD00001868012010B50348AB
:100FF00001F0E2FD01480068406810BDD86501209D
:1010000010B5034801F0D8FD01200249087010BD59
:101010004C6201202502002010B50A4801F0CCFDE9
:10102000084800684068084908600846006840B9F8
:1010300001200649087004480068C0F146000449D0
:10104000088010BD7868012034050020300500209C
:101050003205002010B5024801F0AEFD10BD0000C1
:10106000F866012010B5034801F0A6FD01200249F1
:10107000087010BDAC6201202602002010B50548A2
:1010800001F09AFD03480068406810B90120024948
:10109000087010BDD86801203105002010B508483F
:1010A00001F08AFD06480068406838B9012005490A
:1010B00008700020044908800449088010BD000021
:1010C000586701203102002042020020580200200F
:1010D0000146087810381823B0FBF3F20848805C0A
:1010E000C865032A05D908686FF30900001D8865E3
:1010F00003E008686FF309008865886D7047000099
:10110000EE000208014600208A6A8B69CBB932B131
:10111000012A0DD0022A03D0032A10D10EE000BF0D
:10112000CB6A03F08073B3F1807F00D1012007E028
:10113000CB6AB3F1C07F00D1012001E000E000BF25
:1011400034E08B69B3F5005F1AD132B1012A07D0C0
:10115000022A03D0032A11D10AE000BF01200EE0C9
:10116000CB6A03F08073B3F1807F00D1012006E0E9
:10117000CB6AB3F1C07F00D1012000E000BF15E0D1
:1011800032B1012A05D0022A04D0032A0CD103E08F
:1011900000BF00BF012008E0CB6A03F08073B3F109
:1011A000807F00D1012000E000BF00BF704730B554
:1011B0000468246824F4802405682C600468636053
:1011C0008468402C04D10468A2600468E16003E0F4
:1011D0000468A1600468E26030BD000010B5002220
:1011E00040210D4802F08CF802200DF0C1FF0122D1
:1011F0004021094802F084F806200DF0B9FF402193
:10120000054802F071F808B1012400E000243C20F8
:101210000DF0AEFF204610BD0018024070B500264C
:10122000012508E0FFF7DAFF0446E00140EA660026
:10123000C6B2681CC5B2082DF4DD304670BD000092
:1012400010B50024002240211C4802F059F84FF448
:101250002F700DF08DFF01224021184802F050F848
:101260000F200DF085FF01224021144802F048F8BC
:1012700004E0601CC4B201200DF07AFF40210F4849
:1012800002F032F808B12D2CF3DB2D2C01DB01200C
:1012900010BD002404E0601CC4B201200DF068FF02
:1012A0004021064802F020F808B9F02CF3DBF02CBE
:1012B00001DB0120ECE70020EAE700000018024013
:1012C0002DE9F04186B000260025002700241421D6
:1012D00001A8FFF737FAA0460020A5490870FFF7DC
:1012E000AFFF0746002F7DD1CC2000F057F94420F6
:1012F00000F054F9642007F0B5F9FFF7A1FF0746A5
:10130000002F70D1CC2000F049F9BE2000F046F942
:10131000FFF784FF0646FFF781FF0546072D07DD2F
:10132000E843C5B2F043C6B200209249087002E01B
:101330000120904908702C46200204B2A01904B282
:1013400004EB8400C4108C480088204404B20020C0
:101350008A4908708748007820B9604200B28849FD
:10136000088001E08648048000208649087086488D
:10137000C078401C8449C8708448C07C02281CD1B5
:101380007F48B0F90000B0F5B97F12DA80480078E4
:10139000401C7F49087008460078052808DD0020B9
:1013A00008707A49C874002240217A4801F0A8FFE9
:1013B000DBE0002076490870D7E07448C07C012843
:1013C00021D16F48B0F9000010F1460F17DD7048C9
:1013D0000078401C6E490870084600780528E7DD53
:1013E000002001E09BE073E008706849C8740022A7
:1013F0004021684801F084FF07F00EFDB5E00020B1
:1014000063490870B1E05E48B0F9000010F1640F64
:1014100026DA5F480078401C5D490870084600786D
:101420000228C5DD0020087001224021594801F042
:1014300067FF07F0DBFC01205449C8748DF80400F5
:101440004F480088000A8DF805004D4800788DF857
:101450000600042201A94FF4A84009F003FD84E02E
:101460004748B0F90000B0F5C87F24DD484800784F
:10147000401C4749087008460078022875DD0020A6
:10148000087001224021434801F03AFF02203F4901
:10149000C8748DF804003A480088000A8DF80500E9
:1014A000374800788DF80600042201A94FF4A840BF
:1014B00009F0D8FC59E000224021364801F020FF15
:1014C00007F0AAFC0020324908703049C8744CE08B
:1014D00031480079401C304908712C48C07C0328F1
:1014E00043D028480078401C2649087008460078F8
:1014F00005283ADD0020087000224021254801F02F
:10150000FFFE07F089FC03202049C8748DF8040011
:10151000022201A94FF4A84009F0A4FC25E01E48CE
:101520000079401C1C4908711848C07C03281CD055
:1015300014480078401C13490870084600780528B4
:1015400013DD0020087000224021124801F0D8FE6F
:1015500007F062FC03200D49C8748DF804000222D4
:1015600001A94FF4A84009F07DFC06B0BDE8F08168
:10157000600500206C050020680500206105002042
:101580006A0500206D05002002090020EC080020FB
:1015900074050020000802400B09002070B50446C5
:1015A000012526E004F00106641086B100224021E6
:1015B000114801F0A5FE02200DF0DAFD01224021C4
:1015C0000D4801F09DFE3C200DF0D2FD0FE0002201
:1015D0004021094801F094FE3C200DF0C9FD012294
:1015E0004021054801F08CFE02200DF0C1FD681C71
:1015F000C5B2082DD6DD70BD0018024010B50448F4
:10160000008840F040000249088000F0B7FB10BDA0
:101610008E0600207047000030B500210022002314
:101620000478012C29D12C4D2C704378C47885780E
:1016300004EB0524A1B24FF6FF74A14208D19FED3F
:10164000270A274C84ED000A0224264D2C7014E052
:1016500000EE101AB8EE400ADFED230A80EE201AE1
:101660001F4C84ED001A2BB994ED000AB1EE400A2C
:1016700084ED000A01241B4D2C700479012C29D122
:101680001A4D2C704379C479857904EB0524A2B2F4
:101690004FF6FF74A24208D19FED100A144C84ED5E
:1016A000000A0224134D2C7014E000EE102AB8EE4C
:1016B000400ADFED0D0A80EE201A0D4C84ED001A71
:1016C0002BB994ED000AB1EE400A84ED000A012422
:1016D000084D2C7030BD00004402002000000000C6
:1016E00088050020900500200000C8424502002027
:1016F0008C0500209105002030B591B004462021D2
:1017000009A8FFF71FF8202101A8FFF71BF8002503
:101710008DF82440254800788DF8250003208DF8A9
:10172000260001208DF8270021480068000E8DF862
:1017300028001F480068000C8DF829001C4800880C
:10174000000A8DF82A001A4800788DF82B001948F5
:101750000068000E8DF82C0016480068000C8DF80B
:101760002D0014480088000A8DF82E0011480078DA
:101770008DF82F00104800788DF830000F48008851
:10178000000A8DF831000D4800788DF832000020F5
:101790008DF8330001AA102109A800F03BFD054691
:1017A000294601A800F0ECF811B030BD7806002001
:1017B000B0050020B4050020BB050020A4050020D2
:1017C00070B590B006461C2109A8FEF7BBFF1C218E
:1017D00002A8FEF7B7FF0025002404F0ABFA03F0DF
:1017E0006BFF1848007810B94FF6FF740BE01648ED
:1017F00090ED000ADFED150A20EE200ABCEEC00ACB
:1018000010EE100A84B203208DF824000E208DF80B
:10181000250005208DF82600200A8DF82700E0B26B
:101820008DF828000120022302AA0521009009A8B2
:1018300006F048F90546294602A800F0A1F810B0C4
:1018400070BD00005B0500205405002000007A44B4
:1018500070B505460C46164632462146284606F027
:1018600071F900B970BDE1B2284600F053F900B932
:10187000F8E700BFF6E7000010B58EB0182108A801
:10188000FEF760FF182102A8FEF75CFF002403208A
:101890008DF8200012208DF8210002208DF8220002
:1018A0008DF8230007480078032302AA0421009042
:1018B00008A806F007F90446214602A800F060F8DF
:1018C0000EB010BD7806002010B525480088B0F590
:1018D0007A7F04DA22480088401C21490880214888
:1018E000007800283BDD20480088401C1E49088005
:1018F00008460088042832DD002008801B48006864
:1019000040681B49096888420BD018480068406845
:101910001749086002201349087000201549088003
:101920001DE010480078022819D112480088401C98
:101930001049088008460088022810DD0020088031
:1019400001200D4908700A480068C0F1FA000B49EF
:101950000880064801F0EAF800200249087010BD2E
:10196000420200203C02002040020020F8660120D4
:10197000380200203E020020300200203402002005
:1019800070B504460D4600260CE0022006F06AFE03
:10199000701CC6B21E2E05DD19484078401C18493F
:1019A000487007E0174800780128EED116480088F3
:1019B0003228EADD00BF0020124908701348058074
:1019C000028821461248FEF74EFE12480068021DAA
:1019D0000E4803880E49104801F084FA30B10848D7
:1019E000C078401C0649C87000F088F800200B49F8
:1019F00008800B484078401C0949487070BD0000C1
:101A00000B09002031020020420200203202002097
:101A1000A0070020B8640120586701204A02002076
:101A20000209002010B500200C4908700C480288FB
:101A30000C490D4803F0FAFCFA200C49086001201B
:101A40000B49087000200B4908700B490880FA22E6
:101A50000A49054803F08EFC10BD00003102002049
:101A600032020020A0070020B864012038020020C4
:101A70003C0200203002002034020020A00600209A
:101A800010B515480078012825D101221348018896
:101A90001348FFF7DDFE114801881148FEF730FEBC
:101AA00000200D4908700F490870FA200E4908609F
:101AB00000200A4908800D480068011DFA23084AE1
:101AC0000B4801F00FFA012006490870002009496F
:101AD00008800949087010BD30020020340200203F
:101AE000A00600203C02002038020020B86401203B
:101AF000F8660120560200205D02002010B504485F
:101B000003F07FF805F03AF8FFF78CFF10BD0000F6
:101B1000B86401202DE9F05F054688460024A246FE
:101B2000A34646460027A14614E1285DA5287DD19D
:101B3000601C285C0128FAD1A01C285C052876D2FC
:101B4000DFE800F003417EB7DF000C2E3ADB04F142
:101B50000800285C010604F10900285C01EB004143
:101B600004F10A00285C01EB002104F10B00285C61
:101B70000F187B480068874224D1A01D285C0828E4
:101B800004D1281908210BF0F5FE19E0A01D285CEE
:101B9000092804D1281908210BF050FF10E0A01DDE
:101BA000285C0A2804D1281908210BF055FE07E00B
:101BB000A01D285C0B2803D1281908210BF092FEE8
:101BC0004FF00109BBE00C2E39DB04F10800285C62
:101BD000010604F10900285C01EB004104F10A0050
:101BE000285C01EB002104F10B00285C0F185C4815
:101BF0000068874223D15B480078F0B95A480078E2
:101C0000D8B9201D295CE01C285C01EB0020574955
:101C10000880A01D295C601D285C01EB0020544950
:101C2000088001204F490870002001E08EE085E027
:101C30005049087002204C4908704FF001097EE0BD
:101C40000C2E35DB04F10800285C010604F10900C4
:101C5000285C01EB004104F10A00285C01EB002143
:101C600004F10B00285C0F183D48006887421FD123
:101C70003C480078D0B93C480078B8B9201D295CB0
:101C8000E01C285C01EB002038490880A01D295C7D
:101C9000601D285C01EB0020354908800120314996
:101CA00008703449087002202F4908704FF001096C
:101CB00045E0092E24DBE01C285C0106201D285C81
:101CC00001EB0041601D285C01EB0021A01D285C98
:101CD0000F1823480068874212D12748008858B956
:101CE0002148007840B9A8EB0402D21F91B2E21D4E
:101CF000A8180BF0E9FC01E00BF04AFB4FF00109DA
:101D00001DE0082E19DBE01C285C0106201D285C64
:101D100001EB0041601D285C01EB0021A01D285C47
:101D20000F180F480068874207D1E01D285CAA28D9
:101D300001D10BF02DFB4FF0010900E000BF00BF07
:101D4000B9F1010F02D10020BDE8F09F601CC4B2C0
:101D5000701EC6B2082EBFF6E8AE0120F4E7000000
:101D60007C060020DB050020BB050020DE050020EE
:101D7000E0050020DC0500202806002000BFFEE76B
:101D800030B59DB000201A901B901C9000240025B7
:101D9000052200211AA800F087F89DF86800AA28FB
:101DA0000DD19DF86900DD2809D19DF86A00CC2885
:101DB00005D19DF86B00EE2801D11DB030BD36482D
:101DC0000088012802D1354801F0CEFA4FF4807125
:101DD000334801F091FA04220821324800F014F946
:101DE000C820ADF85800ADF85A004FF4AF60ADF818
:101DF00062004FF4FA70ADF85C006420ADF85E004C
:101E0000ADF8600002208DF8640000208DF86500B8
:101E10000E22102116A800F0F7F800208DF8180007
:101E20008DF81E000822402106A800F0EDF81A489F
:101E30000088012802D1194801F096FA4FF4807108
:101E4000174801F059FA4FF4FA70ADF80400002079
:101E5000ADF80600ADF80800ADF80A00ADF80C00CA
:101E6000CDF80E00CDF812001222202101A800F0BA
:101E7000CBF8AA208DF86800DD208DF86900CC2011
:101E80008DF86A00EE208DF86B00042200211AA85C
:101E900000F0BAF800BF90E78C06002038690120F6
:101EA000001402407C0600202DE9F04706460D464E
:101EB00014460027B846B9464FEA152805F0FF0931
:101EC000002280211E4801F01BFA03201D490870E2
:101ED000084680F8018080F802901B490C701B486E
:101EE000006800F10C01E31C194A1A4800F0FAFFDF
:101EF0001648006800F10C02E31C1249164800F075
:101F0000F1FF00BF154800780028FBD000201349DE
:101F100008701349087001228021094801F0F0F986
:101F2000094802780A49C91C3046FEF79CFB44F276
:101F3000A01700BF38467F1E0A28FBD8BDE8F087EF
:101F4000000402402500002027020020F461012047
:101F5000250100204C620120AC62012025020020F6
:101F60002602002010B5002401224021204801F063
:101F7000C7F90122D1031F4801F0C2F901228021D3
:101F80001B4801F0BDF944F2A01400BF2046641EB6
:101F90000A28FBD800228021154801F0B1F905205C
:101FA0001549087000204870887014490870144959
:101FB000087003221049134802F08AF800BF0F4846
:101FC00000780028FBD000200C4908700C490870EC
:101FD00001228021064801F093F944F2A01400BFC9
:101FE0002046641E0A28FBD800F09CF810BD0000B3
:101FF00000040240001802402501002025020020B4
:1020000026020020F46101202DE9F04706460C4627
:1020100015460027B846B9464FEA142804F0FF09D0
:1020200000228021374801F06BF9062036490870FC
:1020300000204870354908703549087035480068F7
:1020400000F10C010223344A344800F04BFF3148C0
:10205000006800F10C0202232B49314800F042FFD6
:1020600000BF2A4800780028FBD0002027490870CC
:102070002749087001228021224801F041F944F2E9
:10208000A01700BF38467F1E0A28FBD800228021F7
:102090001C4801F035F902201B490870084680F8F9
:1020A000018080F802902A463146C01CFEF7DBFA18
:1020B0001848006800F10C01EB1C174A174800F0A3
:1020C00011FF1448006800F10C02EB1C0E49144883
:1020D00000F008FF00BF0D4800780028FBD000206A
:1020E0000A4908700A49087001228021054801F058
:1020F00007F944F2A01700BF38467F1E0A28FBD814
:10210000BDE8F087000402402500002025020020E1
:1021100026020020F4610120250100204C620120EC
:10212000AC62012010B5002400228021314801F06A
:10213000E7F8062030490870002048702F480068F2
:1021400000F10C0102232E4A2E4800F0CBFE2B4852
:10215000006800F10C02022327492B4800F0C2FE60
:1021600000BF2A4800780028FBD0002027490870CB
:1021700027490870012280211E4801F0C1F844F26D
:10218000A01400BF2046641E0A28FBD8002280212C
:10219000184801F0B5F80120174908700020487070
:1021A0001648006800F10C010323154A154800F099
:1021B00099FE1248006800F10C0203230E491248F0
:1021C00000F090FE00BF114800780028FBD00020EE
:1021D0000E4908700E49087001228021054801F05F
:1021E0008FF844F2A01400BF2046641E0A28FBD8D2
:1021F00010BD00000004024025000020F461012011
:10220000250100204C620120AC6201202502002043
:102210002602002003460120704700002DE9FC4102
:1022200005460C4600260027B0468648807AA8421C
:102230007DDD8448C07AA0423CDD8248807A401B24
:10224000461E8048C07A001B471E7F49C88A00EBA3
:10225000D0714A107C49C98A06FB01210A22B1FBD0
:10226000F2F1784A9288511A89B2ADF80010764995
:10227000C88A00EBD0714A107349C98A07FB012153
:102280000A22B1FBF2F16F4AD288511A89B2ADF835
:102290000210C5EB05106D4901EB001030F8240069
:1022A00068490989081A80B2ADF8040001208DF848
:1022B0000600B6E06348807A401B461E6148C07A3B
:1022C000271A6149C88A00EBD0714A105E49C98A51
:1022D00006FB01210A22B1FBF2F15A4A9288511AF7
:1022E00089B2ADF800105849C88A00EBD0714A1085
:1022F0005549C98A07FB01210A22B1FBF2F1514A73
:10230000D288114489B2ADF80210C5EB05104F49CF
:1023100001EB001030F824004A490989081A80B2FC
:10232000ADF8040001208DF806007AE0FFE745488B
:10233000C07AA0423BDD4348807A2E1A4148C07AD9
:10234000001B471E4049C88A00EBD0714A103E4925
:10235000C98A06FB01210A22B1FBF2F1394A9288AF
:10236000114489B2ADF800103749C88A00EBD0712A
:102370004A103549C98A07FB01210A22B1FBF2F153
:10238000304AD288511A89B2ADF80210C5EB051057
:102390002E4901EB001030F824002A490989081A57
:1023A00080B2ADF8040001208DF8060039E0254820
:1023B000807A2E1A2348C07A271A2349C88A00EB4C
:1023C000D0714A102049C98A06FB01210A22B1FBBB
:1023D000F2F11C4A9288114489B2ADF800101A49F2
:1023E000C88A00EBD0714A101749C98A07FB01213E
:1023F0000A22B1FBF2F1134AD288114489B2ADF836
:102400000210C5EB0510114901EB001030F8240053
:102410000C490989081A80B2ADF8040001208DF832
:1024200006000848407B00FB0540802101EBC0000E
:102430001FFA80F8082241466846FFF7E5FDBDE82F
:10244000FC810000ECE70020A8D900205801012001
:1024500070B502460D46FF21FF23002409E012F863
:10246000010B80EA01040748005D80EA0301064889
:10247000035D281EA5F10106B5B2F0D143EA0120A3
:1024800070BD0000660200206603002010B5002029
:102490000021002200BF1A4B587D24E0184B997D83
:1024A00017E000EB8003174C04EB431303EB8103AD
:1024B0009B78012B09D100EB800304EB431333F825
:1024C00021300F4C2383012205E001B903E04B1EAC
:1024D000D9B20029E5DA00BF012A00D105E000B930
:1024E00003E0431ED8B20028D8DA00BF12B1044B73
:1024F0001B8B1BB9024B1B89014C238310BD0000B1
:10250000ECE7002058E800207047000038B502468C
:102510000020009000BF92F83C00012801D1022069
:1025200038BD012082F83C0000BF0868092816D990
:102530001068C0680C780A3C04EB44050724AC40E2
:10254000A0431468E0600C780A3C04EB44048868FB
:10255000A0401468E46820431468E06013E0106849
:1025600000690C7804EB44050724AC40A0431468D0
:1025700020610C7804EB44048868A0401468246946
:102580002043146820614868072817D21068406B00
:102590000C79641E04EB84051F24AC40A04314682E
:1025A0006063088880B20C79641E04EB8404A04048
:1025B0001468646B20431468606331E048680D2838
:1025C00017D21068006B0C79E41F04EB84051F24FC
:1025D000AC40A04314682063088880B20C79E41FE3
:1025E00004EB8404A0401468246B20431468206327
:1025F00016E01068C06A0C790D3C04EB84051F24BA
:10260000AC40A0431468E062088880B20C790D3CAD
:1026100004EB8404A0401468E46A20431468E06278
:10262000194B1A4C1068A04206D10868122803D131
:10263000586840F480005860144C1068A0421CD1C7
:102640000868102802D00868112816D1586840F48C
:1026500000005860086810280FD10D4800680D4C24
:10266000B0FBF4F000EB80004000009002E0009826
:10267000401E009000980028F9D100BF002082F889
:102680003C0000BF00BF4BE7002301400020014099
:102690009C06002040420F0010B5044629480078EF
:1026A000001F06284AD2DFE800F03040104903201E
:1026B000254800F05CF8254908600620214908708B
:1026C00006210120FEF7A6F939E01F4800F04FF877
:1026D0001F49086009201B4908701E48008818B966
:1026E00009210120FEF796F929E0174800F03FF88C
:1026F000194908600420134908701848008818B95F
:1027000004210120FEF786F919E00F4800F02FF8A8
:102710001349086005200B4908701248008818B951
:1027200005210120FEF776F909E0074800F01FF8BF
:102730000D49086008200349087000E000BF00BF91
:1027400010BD000006000020546101200800002098
:1027500014000020040000201800002000000020C9
:102760000C000020020000201000002070470146ED
:102770000868C06C704770B50446002500262068C4
:102780000068C0F3400520684068C0F3401695B368
:102790008EB3206C00F0100018B9206C40F400706B
:1027A00020642068806800F04050E8B9A069D8B97A
:1027B0002068C06A00F4700020B12068806800F4CE
:1027C000806088B92068406820F020002168486057
:1027D000206C20F480702064206C00F4805018B9C4
:1027E000206C40F0010020642046FFF755FF6FF099
:1027F00012002168086020680068C0F38005206826
:102800004068C0F3C016E5B3DEB3206C00F01000E2
:1028100018B9206C40F4005020642068806800F4EF
:10282000401038BB2068806B00F4401020B1206855
:10283000806800F48060E8B92068406800F4806037
:10284000C0B92068806800F0405098B9A06988B984
:102850002068406820F0800021684860206C20F4E7
:1028600080502064206C00F4807018B9206C40F017
:10287000010020642046FFF747FE6FF00C0021683E
:1028800008602068006800F0010520684068C0F317
:10289000801685B17EB12068006800F0010050B15B
:1028A000206C40F480302064204600F053F86FF034
:1028B00001002168086020680068C0F340152068A6
:1028C0004068C0F380667DB176B1606C40F0020074
:1028D00060646FF02000216808602046FFF746FF23
:1028E0006FF020002168086070BD000070B50446DC
:1028F00000250CB9012070BD1549A06A884200D09E
:1029000000BF206C30B90020606484F83C00204691
:1029100000F022F8206C00F0100088B9206C20F440
:10292000885040F0020020642046FDF7C5FF0020DB
:102930006064206C20F0020040F00100206400E0A0
:10294000012500BF002084F83C0000BF2846D2E7E4
:102950000100000F7047000010B586B00446142136
:1029600001A8FDF7EFFE2949206888424BD100BF3E
:10297000002000902648006840F4807024490860D8
:102980000846006800F48070009000BF00BF00BFE0
:10299000002000901E481438006840F001001C49D7
:1029A000143908600846006800F00100009000BF7C
:1029B00000BF00BF002000900846006840F0020001
:1029C00008600846006800F00200009000BF00BFE9
:1029D00070200190032002900020039001A90D486F
:1029E00000F082FB0320019002900020039001A9D7
:1029F000094800F079FB02221146122000F02BFD5D
:102A0000122000F01BFD06B010BD000000200140A8
:102A100044380240000002400004024008B501466C
:102A20000020009000BF91F83C00012801D1022055
:102A300008BD012081F83C0000BF0868806800F0F4
:102A40000100A0B90868806840F001000B68986038
:102A500031480068314BB0FBF3F000EB40000090D0
:102A600002E00098401E009000980028F9D1086804
:102A7000806800F0010000284BD0086C40F2016330
:102A8000984340F4807008640868406800F48060EF
:102A900028B1086C20F4005040F480500864086CA1
:102AA00000F4805020B1486C20F00600486401E03A
:102AB0000020486400BF002081F83C0000BF184A95
:102AC0006FF022000B68186008684068154B1843C7
:102AD0000B685860506800F01F0058B9086880689B
:102AE00000F04050A8B90868806840F080400B684A
:102AF00098600EE00C4B086898420AD1086880681C
:102B000000F0405028B90868806840F080400B68A9
:102B1000986000208CE700009C06002040420F00D7
:102B2000002301402000000400200140014691F8EC
:102B30003500022803D08020486501207047052019
:102B400081F835000868006820F001000A6810600C
:102B50000020F3E770B504460CB9012070BD94F86D
:102B60003500022800D1F9E72068006820F0010054
:102B70002168086000202168086021684860216899
:102B800088602168C8602168086121202168486147
:102B90002046FEF79DFA054694F85C103F208840D9
:102BA000A8600020606584F8350000BF84F8340018
:102BB00000BF00BFD2E70000F8B504460020009037
:102BC0008C4800684FF41651B0FBF1F7A56D2E68E4
:102BD00094F85C1008208840304098B12068006864
:102BE00000F0040070B12068006820F00400216843
:102BF000086094F85C1008208840A860606D40F080
:102C00000100606594F85C1001208840304068B194
:102C10002068406900F0800040B194F85C10012009
:102C20008840A860606D40F00200606594F85C1018
:102C300004208840304068B12068006800F002003D
:102C400040B194F85C1004208840A860606D40F0AA
:102C50000400606594F85C1010208840304078B320
:102C60002068006800F0080050B394F85C10102051
:102C70008840A8602068006800F4802080B1206847
:102C8000006800F4002028B9206CC8B12046216CEF
:102C9000884715E0A06C98B12046A16C88470FE0EA
:102CA0002068006800F4807028B92068006820F06F
:102CB000080021680860206C10B12046216C88470C
:102CC00094F85C10202088403040002865D02068AF
:102CD000006800F0100000285FD094F85C102020FD
:102CE0008840A86094F83500052828D1206800683D
:102CF00020F01600216808602068406920F08000FC
:102D000021684861206C08B9A06C28B1206800686F
:102D100020F008002168086094F85C103F2088408B
:102D2000A86000BF002084F8340000BF012084F8B0
:102D30003500206D10B12046216D8847F8BD206810
:102D4000006800F4802080B12068006800F4002052
:102D500028B9606C10B12046616C88471DE0E06BBB
:102D6000D8B12046E16B884717E02068006800F47E
:102D7000807068B92068006820F010002168086041
:102D800000BF002084F8340000BF012084F8350023
:102D9000E06B10B12046E16B8847606D38B3606D21
:102DA00000F00100F0B1052084F8350020680068CB
:102DB00020F001002168086000BF0098401C0090CE
:102DC000B84200D905E02068006800F00100002842
:102DD000F3D100BF00BF002084F8340000BF012001
:102DE00084F83500E06C10B12046E16C884700BFE4
:102DF000A4E700009C0600202DE9F04104460025D0
:102E000000F084FA074614B90120BDE8F081606A39
:102E100000B100BF00BF002084F8340000BF0220D2
:102E200084F835002068006820F0010021680860FF
:102E30000AE000F06BFAC01B052805D92020606568
:102E4000032084F83500E0E72068006800F0010006
:102E50000028EED12068056821480540D4E9010129
:102E60000843E16808432169084361690843A1698F
:102E70000843E1690843216A08430543606A04285E
:102E800003D1D4E90B01084305432068056020689D
:102E9000456925F00705606A0543606A04280DD17D
:102EA000A06A0543E06A48B12046FEF72BF928B135
:102EB00040206065012084F83500A6E72068456160
:102EC0002046FEF705F9064694F85C103F2088403E
:102ED000B06000206065012084F83500002094E790
:102EE0003F8010F02DE9F04704460D4616461F4678
:102EF0004FF00008D4F8589000BF94F8340001282F
:102F000002D10220BDE8F087012084F8340000BF20
:102F100094F8350001282BD1022084F835000020D8
:102F200060653B46324629462046FEF740F994F854
:102F30005C103F208840C9F808002068006840F015
:102F40001600216808602068406940F08000216810
:102F50004861206C28B12068006840F008002168B2
:102F600008602068006840F001002168086006E001
:102F700000BF002084F8340000BF4FF00208404634
:102F8000C0E70000F0B50C46002500220023002118
:102F900092E0012606FA01F504EA0502AA427DD173
:102FA00006684FEA410C032707FA0CF7BE43066098
:102FB000CF0800F1200656F827604F074FEAD76C7C
:102FC0000F2707FA0CF7BE434FEAD10C00F1200798
:102FD00047F82C6086684FEA410C032707FA0CF784
:102FE000BE438660466801278F40BE434660C66880
:102FF0004FEA410C032707FA0CF7BE43C660304E78
:103000008F0856F827308E07370F0F26BE40334003
:103010002C4EB04201D1002623E02B4EB04201D10C
:1030200001261EE0294EB04201D1022619E0284EA9
:10303000B04201D1032614E0264EB04201D104264D
:103040000FE0254EB04201D105260AE0234EB042E2
:1030500001D1062605E0224EB04201D1072600E04C
:1030600008268F073F0FBE409E4224D18E07370FA0
:103070000F2606FA07F3124E8F0856F827609E4374
:103080000F4F4FEA910C47F82C60164E3668964366
:10309000144F3E603E1D3668964300E00BE03F1D36
:1030A0003E603E1D366896433F1D3E603E1D3668BD
:1030B00096433F1D3E60491C1029FFF46AAFF0BDE6
:1030C00008380140000002400004024000080240AD
:1030D000000C0240001002400014024000180240A0
:1030E000001C0240003C0140F8B502460B4600259A
:1030F000002400200021DCE0012606FA01F51E680C
:1031000006EA0504AC4273D15E68022E02D05E6806
:10311000122E13D1CF0802F1200656F827004E07D1
:10312000F70E0F26BE40B0434F07FF0E1E69BE408C
:103130003043CF0802F1200646F8270010684F0000
:103140000326BE40B0431E7906F003064F00BE4082
:10315000304310605E68012E08D05E68022E05D0F4
:103160005E68112E02D05E68122E13D190684F0057
:103170000326BE40B0434F00DE68BE40304390603F
:10318000506801268E40B0431E79C6F300168E406B
:1031900030435060D0684F000326BE40B0434F001C
:1031A0009E68BE403043D0605E6806F08056B6F13F
:1031B000805F7DD100BF00260096404E366846F401
:1031C00080463E4F3E603E46366806F48046009696
:1031D00000BF00BF3A4E8F0856F827008E07370F02
:1031E0000F26BE40B043374EB24202D1002624E043
:1031F0005EE0354EB24201D101261EE0334EB242AE
:1032000001D1022619E0324EB24201D1032614E068
:10321000304EB24201D104260FE02F4EB24201D10E
:1032200005260AE02D4EB24201D1062605E02C4EBD
:10323000B24201D1072600E008268F073F0FBE40AB
:1032400030431F4E8F0846F82700264E3068A043B3
:103250005E6806F48036B6F5803F00D12043214EEB
:103260003060361D3068A0435E6806F40036B6F55F
:10327000003F00D120431B4E361D3060361D3068A4
:10328000A0435E6806F48016B6F5801F00D1204387
:10329000144E08363060361D3068A0435E6806F470
:1032A0000016B6F5001F00D120430E4E0C363060DC
:1032B000491C1029FFF420AFF8BD0000443802403B
:1032C00008380140000002400004024000080240AB
:1032D000000C02400010024000140240001802409E
:1032E000001C0240003C0140024613690B400BB138
:1032F000012000E00020704742694A404261704767
:103300000AB1816101E00B048361704701480068E4
:10331000704700009006002070B504460CB90120EB
:1033200070BD4CF6CC402168086045F255502168CC
:103330000860D4E9001048602168A0688860FFF741
:10334000E5FF054606E0FFF7E1FF401B302801D905
:103350000320E5E72068C0680028F4D14AF6AA20D7
:10336000216808600020DBE701464AF6AA200A68C7
:10337000106000207047000010B50A48006840F453
:103380000070084908600846006840F480600860E2
:103390000846006840F48070086000F02BF80020B8
:1033A00010BD0000003C024070B504460E48007895
:1033B0004FF47A71B1FBF0F00C490968B1FBF0F5FC
:1033C000284600F095FF08B1012070BD102C07D2EF
:1033D00003222146101F00F03EF80548046001E07A
:1033E0000120F2E70020F0E7980600209C0600206C
:1033F0009406002008B500BF002000900E48006829
:1034000040F480400C4908600846006800F48040A1
:10341000009000BF00BF00BF00200090081F0068A0
:1034200040F08050091F08600846006800F0805096
:10343000009000BF00BF08BD4438024000BF00F04C
:103440001F02012191404209920002F1E022C2F8DC
:10345000001100BF70472DE9F05F80460D4616460B
:10346000002704F013FB074639462A46334601F08D
:103470000700C0F1070ABAF1040F02D94FF0040A9D
:1034800001E0C0F1070AD14600F1040ABAF1070FC2
:1034900002D24FF0000A01E0A0F1030AD4464FF037
:1034A000010A0AFA09FAAAF1010A0AEA020A0AFA60
:1034B0000CFA4FF0010B0BFA0CFBABF1010B0BEA12
:1034C000030B4AEA0B042146404604F0E7FABDE844
:1034D000F09F000000BF00F00702064B19684FF68E
:1034E000FF031940044B0B4343EA0221014B1960CF
:1034F00000BF70470CED00E00000FA05F8B5044687
:1035000000250026207800F0010020B9207800F086
:10351000040004282FD100205B498866FFF7F6FEDF
:10352000054606E0FFF7F2FE401B022801D9032002
:10353000F8BD56480068C0F3C0600028F2D160684A
:103540008101207A41EA00705049843108600120ED
:103550004D498866FFF7DAFE054606E0FFF7D6FE1E
:10356000401B022801D90320E2E748480068C0F365
:10357000C0600028F2D0207800F0020002287DD13F
:1035800000BF0020009041484030006840F080506B
:103590003E49403108600846006800F080500090C5
:1035A00000BF00BF3A48006840F4807038490860A6
:1035B000FFF7ACFE054606E0FFF7A8FE401B022819
:1035C00001D90320B4E73248006800F48070002875
:1035D000F2D02E487030006800F440764EB3A089D7
:1035E00000F44070B04224D028487030006820F4C5
:1035F0004076012027490860002008602348703089
:103600000660006800F0010098B1FFF77FFE0546F4
:1036100008E0FFF77BFE401B41F28831884201D968
:10362000032085E7194870300068C0F34000002887
:10363000EFD000BFA08900F44070B0F5407F0CD1FE
:1036400012480830006820F4F810134AE16811406D
:1036500008430E490831086007E00C48083000684C
:1036600020F4F810094908310860084870300068F3
:10367000A189C1F30B010843044900E002E0703165
:10368000086000BF002053E70000474200380240B6
:1036900000700040400E4742FFFCFF0F70B504462B
:1036A0000D460CB9012070BD5848006800F00F00AD
:1036B000A84209D255490D700846006800F00F0075
:1036C000A84201D00120EEE7207800F00200022895
:1036D0001DD1207800F00400042805D14C48006872
:1036E00040F4E0504A490860207800F008000828BB
:1036F00005D14748006840F46040454908604448A7
:10370000006820F0F000A168084341490860207873
:1037100000F00100A8B36068012807D13C480838D0
:103720000068C0F34040B8B90120BCE760680228D7
:1037300002D06068032807D1354808380068C0F314
:10374000406048B90120AEE7314808380068C0F34E
:10375000400008B90120A6E72D48006820F00300CA
:10376000616808432A490860FFF7D0FD064609E072
:10377000FFF7CCFD801B41F28831884202D903203B
:1037800091E707E02248006800F00C006168B0EBA8
:10379000810FEDD11D48006800F00F00A84209D943
:1037A0001A490D700846006800F00F00A84201D0C9
:1037B000012078E7207800F00400042807D114489D
:1037C000006820F4E050E16808431149086020785F
:1037D00000F00800082808D10D48006820F4604077
:1037E000216940EAC1000A49086000F03DF8084933
:1037F0000968C1F30311074A515CC84006490860D3
:103800000220FFF7D1FD00204DE70000003C024000
:1038100008380240F60002089C06002001480068B3
:10382000704700009C06002000B5FFF7F7FF044931
:103830000968C1F38221034A515CC84000BD000001
:10384000083802400601020800B5FFF7E7FF044907
:103850000968C1F34231034A515CC84000BD000011
:1038600008380240060102082DE9F047002400252F
:103870000026A1462548006800F00C0020B104286D
:1038800005D008283AD105E0DFF8849039E0DFF868
:10389000849036E01D48001F006800F03F041B487C
:1038A000001F006800F4800078B11A481749091F0A
:1038B0000968C1F38811A0FB01700146224600236C
:1038C0003846FCF759FE05460EE011480F49091F1E
:1038D0000968C1F38811A0FB01700146224600234C
:1038E0003846FCF749FE05460848001F0068C0F34B
:1038F0000140401C4600B5FBF6F902E0DFF81090ED
:1039000000BF00BF4846BDE8F0870000083802400D
:103910000024F40000127A00F8B504460CB9012026
:10392000F8BD207800F00100002874D0F948006844
:1039300000F00C0004280DD0F648006800F00C00E0
:10394000082813D1F348001F006800F48000B0F588
:10395000800F0BD1EF4808380068C0F340400028C2
:1039600059D06068002856D10120D9E700BF6068AF
:10397000B0F5803F08D1E7480838006840F480304F
:10398000E449083908601EE06068B0F5A02F0DD149
:10399000E0480838006840F48020DE4908390860B3
:1039A0000846006840F4803008600CE0D9480838C8
:1039B000006820F48030D74908390860084600685C
:1039C00020F48020086000BF606890B1FFF79EFC83
:1039D000054606E0FFF79AFC401B642801D9032046
:1039E0009EE7CC4808380068C0F340400028F1D07A
:1039F00011E0FFF78BFC054606E0FFF787FC401B54
:103A0000642801D903208BE7C24808380068C0F356
:103A100040400028F1D1207800F0020002285FD158
:103A2000BC48006800F00C0058B1BA48006800F0CB
:103A30000C0008281CD1B748001F006800F4800063
:103A4000B0B9B44808380068C0F3400020B1E0685D
:103A5000012801D0012063E7AE480838006820F053
:103A6000F800216940EAC100AA490839086037E036
:103A7000E06800B30120A8490860FFF747FC05464D
:103A800006E0FFF743FC401B022801D9032047E76B
:103A9000A04808380068C0F340000028F1D09D48D5
:103AA0000838006820F0F800216940EAC10099490F
:103AB0000839086014E0002097490860FFF726FCE9
:103AC000054606E0FFF722FC401B022801D903202F
:103AD00026E7904808380068C0F340000028F1D17C
:103AE000207800F0080008282CD16069A8B10120D6
:103AF0008A490860FFF70AFC054606E0FFF706FC66
:103B0000401B022801D903200AE782486C30006874
:103B1000C0F340000028F1D014E000207F49086085
:103B2000FFF7F4FB054606E0FFF7F0FB401B022819
:103B300001D90320F4E677486C300068C0F34000F8
:103B40000028F1D1207800F00400042870D100266C
:103B500070483830006800F0805090B900BF0020F5
:103B600000906C483830006840F080506949383126
:103B700008600846006800F08050009000BF00BF59
:103B800001266748006800F48070B0B96448006896
:103B900040F4807062490860FFF7B8FB054606E014
:103BA000FFF7B4FB401B022801D90320B8E65C48AC
:103BB000006800F480700028F2D000BFA0680128DF
:103BC00008D154486830006840F00100514968311C
:103BD00008601DE0A06805280DD14E4868300068D7
:103BE00040F004004B49683108600846006840F026
:103BF000010008600CE047486830006820F00100D0
:103C00004449683108600846006820F004000860F4
:103C100000BFA068A8B1FFF779FB054609E0FFF7F0
:103C200075FB401B41F28831884202D9032077E6B8
:103C300026E0384868300068C0F340000028EED025
:103C400013E0FFF763FB054608E0FFF75FFB401B4F
:103C500041F28831884201D9032061E62D4868305D
:103C60000068C0F340000028EFD1012E07D1294899
:103C70003830006820F0805026493831086000BF95
:103C8000A069B8B32348006800F00C0008285ED093
:103C9000A069022846D100201F490866FFF736FBBD
:103CA000054606E0FFF732FB401B022801D903203E
:103CB00036E6184808380068C0F340600028F1D1A3
:103CC000D4E907010843616A40EA81110122A06A30
:103CD000C2EB500041EA00412C20005D41EA006047
:103CE0000C49091F086001200B490866FFF70EFB0D
:103CF000054607E02DE0FFF709FB401B022801D92C
:103D000003200DE6034808380068C0F3406000282F
:103D1000F1D01EE00838024000004742800E4742C2
:103D20000070004000200C490866FFF7EFFA0546D6
:103D300006E0FFF7EBFA401B022801D90320EFE56C
:103D400006480068C0F340600028F2D101E001207D
:103D5000E6E50020E4E500000000474200380240AC
:103D600070B505460B4616460024286840680E4983
:103D700000EA0104200CD870C4F30420587004F049
:103D80003F009870C4F3423018705EB9D87805F0DF
:103D900055F8D870587805F051F85870987805F0B3
:103DA0004DF89870002070BD3FFFFF0070B50446CD
:103DB0000B46164600252068806A58602068006916
:103DC000C0F30E009860206800680F4900EA010502
:103DD000C5F305401870C5F30620587005F07F0044
:103DE000987005F48000000CD8705EB9187805F062
:103DF00025F81870587805F021F85870987805F073
:103E00001DF89870002070BD7F7F7F0010B50446BC
:103E10000CB9012010BD607F20B90020207720461A
:103E200000F060F80220607700BFCA202168486275
:103E300053202168486200BF204605F00AF840B1CF
:103E400000BFFF202168486200BF04206077012086
:103E5000E0E720688068224908402168886021697D
:103E600060680843616908432168896808432168DC
:103E700088602168E068086120680169208941EA5A
:103E80000040216808612068C06820F08000216837
:103E9000C8602068806800F0200060B9204600F00B
:103EA0002DF840B100BFFF202168486200BF042008
:103EB00060770120AEE72068006C20F48020216844
:103EC00008642068006CA16908432168086400BF89
:103ED000FF202168486200BF01206077002099E739
:103EE000BFFF8FFF034A0168914202D10121024ABC
:103EF00011607047002800403C0E474270B50446F0
:103F000000252068C06820F0A0002168C860FFF785
:103F1000FDF9054607E0FFF7F9F9401BB0F57A7F98
:103F200001D9032070BD2068C06800F0200000287F
:103F3000F1D00020F6E7704710B504460CB9012017
:103F400010BD606A00B900BF0021A16294F8510061
:103F500028B9002084F85000204600F033F80220F1
:103F600084F851002068006820F040002168086053
:103F7000D4E901010843E168084321690843616904
:103F80000843218B01F400710843E1690843216A69
:103F90000843A16A0843216808600421A06901EA76
:103FA0001040616A0843216848602068C06920F4B5
:103FB00000602168C86100206065012084F851001C
:103FC0000020BDE710B586B00446142101A8FCF717
:103FD000B9FB3949206888426BD100BF00200090AE
:103FE0003648006840F4805034490860084600684C
:103FF00000F48050009000BF00BF00BF0020009080
:104000002E481438006840F002002C49143908602A
:104010000846006800F00200009000BF00BF382092
:1040200001900220029000200390032004900520BC
:10403000059001A92248FFF757F822482249086055
:104040004FF0C060486000211F488160C1604FF49C
:1040500080610161002141618161C1610162416250
:10406000FEF7CAFE08B1FDF7D5FA00BF1648E064B6
:10407000846300BF13484830144908604FF0C060A3
:1040800048604021114881600021C1604FF4806187
:104090000161002141618161C16101624162FEF7FC
:1040A000ABFE08B1FDF7B6FA00BF0848A064846310
:1040B00000BF06B010BD000000300140443802408F
:1040C00000040240106402404C620120AC620120F6
:1040D0002DE9F04104460E4615460027A06870B948
:1040E0006068B0F5827F0AD1042084F851002B4625
:1040F00032463146204600F063F8BDE8F08100BF4B
:1041000094F85000012801D10220F6E7012084F83C
:10411000500000BF94F85100012801D0022746E06A
:1041200006B10DB9012742E0042084F851000020B7
:104130006065A663A587E58720646064A086E08645
:10414000A068B0F5004F05D12068006820F48040D9
:10415000216808600020E16C0864E16CC8631748BE
:10416000E16CC8640020E16C0865E38FD4F800C0FE
:104170000CF10C01A26BE06CFEF7B4FE2068006845
:1041800000F04000402805D02068006840F0400062
:10419000216808602068406840F02000216848607D
:1041A0002068406840F001002168486000BF00BFFF
:1041B000002084F8500000BF38469EE7B58E010805
:1041C0002DE9F04704460E4617461D464FF00008FD
:1041D000C146C24600BF94F85000012802D1022017
:1041E000BDE8F087012084F8500000BF94F85180AA
:1041F000D4F80490B8F1010F0AD0B9F5827F04D148
:10420000A06810B9B8F1040F02D04FF0020A65E0BF
:104210000EB107B115B94FF0010A5FE094F85100F3
:10422000012802D1052084F8510000206065266332
:10423000A586E586A763A587E5872064606494F872
:104240005100042805D10020E16C0864E16CC863CA
:1042500004E00020E16C0864E16CC8632348E16C71
:10426000C8640020E16C0865E38FD4F800C00CF14D
:104270000C01A26BE06CFEF735FE2068406840F050
:104280000100216848600020A16C0864A16CC8632B
:10429000A16CC864A16C0865E38ED4F800C00CF171
:1042A0000C02216BA06CFEF71DFE2068006800F078
:1042B0004000402805D02068006840F04000216898
:1042C00008602068406840F020002168486020684D
:1042D000406840F002002168486000BF00BF002035
:1042E00084F8500000BF50467AE70000B58E010800
:1042F00070B504462546681EB0F1807F01D30120C9
:104300000FE0681E4FF0E02148610F214FF0FF30B1
:1043100003F0C4FB00204FF0E02188610720086112
:10432000002070BD70477047024600BF92F8380009
:10433000012801D102207047012082F8380000BF17
:10434000022082F839001068406820F0700013687D
:104350005860106840680B6818431368586010680C
:10436000806820F0800013689860106880684B684F
:10437000184313689860012082F8390000BF0020BC
:1043800082F8380000BF00BFD5E710B504460CB96D
:10439000012010BD94F8390028B9002084F83800B5
:1043A000204600F00DF8022084F83900211D206815
:1043B00006F088FD012084F839000020E9E70000BC
:1043C00038B5044648492068884218D100BF00200B
:1043D00000904648006840F01000444908600846D4
:1043E000006800F01000009000BF00BF0122022111
:1043F0003620FFF730F83620FFF720F873E03C490D
:104400002068884215D100BF00200090374800681E
:1044100040F02000354908600846006800F02000A0
:10442000009000BF00BF012202213720FFF713F8E0
:1044300059E03049206888421AD100BF002000901E
:104440002A48001D006840F001002849091D086045
:104450000846006800F00100009000BF00BF012284
:1044600002211920FEF7F7FF1920FEF7E7FF3AE0D7
:104470002068B0F1804F18D100BF002000901B4889
:10448000006840F00100194908600846006800F023
:104490000100009000BF00BF012202211C20FEF796
:1044A000DAFF1C20FEF7CAFF1DE01349206888428E
:1044B00019D100BF002000900C48001D006840F496
:1044C00080200A49091D08600846006800F4802021
:1044D000009000BF00BF012202211A20FEF7BBFF9F
:1044E0001A20FEF7ABFF38BD0010004040380240F4
:1044F00000140040000001400048014001460868E7
:10450000C06840F001000A68D0600868006840F0A8
:1045100001000A681060002070472DE9F041044650
:104520000D46002600BF94F83800012802D1022071
:10453000BDE8F081012084F8380000BF022084F833
:1045400039002068866826F0770626F47F462068C2
:104550008660286850283BD00CDC202860D004DC22
:10456000002853D0102865D155E030285DD0402870
:1045700060D141E0602835D070280DD0B0F5805F63
:1045800003D0B0F5005F55D115E02068806820F0B9
:104590000700216888604EE0D5E902136A68206848
:1045A00006F010FD2068866826F0770646F077064C
:1045B000206886603FE0D5E902136A68206806F04B
:1045C00001FD2068806840F480402168886032E006
:1045D000EA686968206806F0EBFD5021206806F063
:1045E000FDFC28E0EA686968206806F0F6FD6021B5
:1045F000206806F0F3FC1EE0EA686968206806F0AF
:10460000D7FD4021206806F0E9FC14E00021206875
:1046100006F0E4FC0FE01021206806F0DFFC0AE061
:104620002021206806F0DAFC05E03021206806F041
:10463000D5FC00E000BF00BF012084F8390000BFB6
:10464000002084F8380000BF00BF71E7704710B544
:10465000044620680069C0F34000D8B12068C068F3
:10466000C0F34000B0B16FF0020021680861012082
:1046700020762068806900F0030018B12046FFF71B
:10468000E5FF05E0204600F029F9204600F0C6F9D4
:104690000020207620680069C0F38000D8B120682F
:1046A000C068C0F38000B0B16FF0040021680861F9
:1046B000022020762068806900F4407018B12046FE
:1046C000FFF7C4FF05E0204600F008F9204600F09F
:1046D000A5F90020207620680069C0F3C000D8B199
:1046E0002068C068C0F3C000B0B16FF00800216856
:1046F0000861042020762068C06900F0030018B12A
:104700002046FFF7A3FF05E0204600F0E7F820462B
:1047100000F084F90020207620680069C0F30010C2
:10472000D8B12068C068C0F30010B0B16FF01000BD
:1047300021680861082020762068C06900F4407074
:1047400018B12046FFF782FF05E0204600F0C6F8CA
:10475000204600F063F9002020762068006900F010
:10476000010058B12068C06800F0010030B16FF05E
:10477000010021680861204600F0EAF9206800691C
:10478000C0F3C01058B12068C068C0F3C01030B189
:104790006FF08000216808612046FFF7C3FD2068A4
:1047A0000069C0F3801058B12068C068C0F3801061
:1047B00030B16FF0400021680861204600F020FA17
:1047C00020680069C0F3401058B12068C068C0F389
:1047D000401030B16FF02000216808612046FFF7DB
:1047E000A2FD10BD10B586B00446142101A8FBF748
:1047F000A9FF3549206888421DD100BF00200090E4
:104800003248006840F001003049086008460068FE
:1048100000F00100009000BF00BF88150190022049
:1048200002900020049003900120059001A92848DF
:10483000FEF75AFC45E02068B0F1804F1FD100BF61
:10484000002000902148006840F001001F490860E6
:104850000846006800F00100009000BF00BF4FF460
:10486000004001900220029001200490002003905B
:104870000120059001A91648FEF736FC21E01549F4
:10488000206888421DD100BF002000900F480068BA
:1048900040F020000D4908600846006800F0200044
:1048A000009000BF00BF80200190022002900120F4
:1048B0000490002003900320059001A90648FEF70C
:1048C00013FC06B010BD000000000140303802406B
:1048D000000002400048014000140240704770B5DB
:1048E00004460D46164600BF94F83800012801D151
:1048F000022070BD012084F8380000BF022084F837
:10490000390036B1042E1BD0082E31D00C2E5ED1CA
:1049100045E02946206806F06BFB2068806940F07E
:104920000800216888612068806920F004002168FF
:10493000886120688069296908432168886147E0A7
:104940002946206806F08CFB2068806940F40060EE
:10495000216888612068806920F48060216888610E
:1049600020688069296940EA0120216888612FE078
:104970002946206806F0B0FB2068C06940F00800B6
:104980002168C8612068C06920F004002168C861FE
:104990002068C069296908432168C86118E0294670
:1049A000206806F0D5FB2068C06940F400602168EB
:1049B000C8612068C06920F480602168C8612068EF
:1049C000C069296940EA01202168C86100E000BF90
:1049D00000BF012084F8390000BF002084F83800AF
:1049E00000BF00BF85E710B504460CB9012010BD1B
:1049F00094F8390028B9002084F83800204600F0E7
:104A00000CF8022084F83900211D206806F05AFABB
:104A1000012084F839000020E9E770477047000062
:104A200030B504460D462068C06840F0010021689A
:104A3000C86001222946206806F0B6FA0C492068B1
:104A4000884203D00B492068884201D1012000E050
:104A5000002028B12068406C40F400402168486480
:104A60002068006840F0010021680860002030BD27
:104A7000000001400004014030B504460D4635B148
:104A8000042D0BD0082D10D00C2D1CD114E0206863
:104A9000C06820F002002168C86015E02068C06886
:104AA00020F004002168C8600EE02068C06820F093
:104AB00008002168C86007E02068C06820F0100086
:104AC0002168C86000E000BF00BF2068C06820F017
:104AD00001002168C86000222946206806F064FAB7
:104AE00019492068884203D018492068884201D1BA
:104AF000012000E0002090B100BF2068006A41F270
:104B00001111084050B92068006A8910084028B97E
:104B10002068406C20F400402168486400BF00BF5A
:104B20002068006A41F21111084050B92068006AFB
:104B30008910084028B92068006820F00100216829
:104B4000086000BF002030BD0000014000040140AB
:104B500010B5044623492068884204D1FCF7B4FE0E
:104B600000F05AFD3CE020492068884238D01F49B7
:104B7000206888420ED181151D48FEF7B5FB01283B
:104B80002ED11C48007804282AD104210120FBF7EB
:104B900041FF25E02068B0F1804F0FD14FF4004174
:104BA0001348FEF7A1FB01281AD112480078052806
:104BB00016D105210120FBF72DFF11E00E492068D9
:104BC00088420DD180210D48FEF78EFB012807D1C8
:104BD00008480078092803D109210120FBF71AFFB2
:104BE00010BD000000100040001400400000014013
:104BF000000002400600002000480140001402406E
:104C0000704710B504460CB9012010BD242084F86B
:104C10003900204600F046F80020E06384F83900AF
:104C200084F83A0000BF84F8380000BF00BFECE70A
:104C3000704710B504460CB9012010BDA06900B141
:104C400000E000BF94F8390028B9002084F838004B
:104C5000204600F0BDF8242084F839002068C068A0
:104C600020F400502168C860204608F0C1F920688F
:104C7000006920F49040216808612068406920F0B4
:104C80002A00216848612068C06840F4005021680B
:104C9000C8600020E063202084F8390084F83A00DE
:104CA0000020CAE710B504463E492068884215D165
:104CB0003D48006820F400203B49086001213B4842
:104CC000FEF760F94FF400613948FEF75BF9606B5D
:104CD000FDF740FF206BFDF73DFF61E0354920689F
:104CE000884214D13048006820F480102E490860B2
:104CF00089142F48FEF746F904212F48FEF742F9A0
:104D0000606BFDF727FF206BFDF724FF48E02B4980
:104D10002068884213D12448001D006820F010004C
:104D20002149091D08604FF4C0612048FEF72AF9A7
:104D3000606BFDF70FFF206BFDF70CFF30E02049A3
:104D40002068884211D11848006820F48020164954
:104D500008604FF440611B48FEF714F9606BFDF7E3
:104D6000F9FE206BFDF7F6FE1AE01749206888422D
:104D700016D10D48001D006820F020000A49091DC9
:104D8000086080210A48FEF7FDF84FF480410F4883
:104D9000FEF7F8F8606BFDF7DDFE206BFDF7DAFE3D
:104DA00010BD0000004C00404038024000000240AE
:104DB0000008024000500040000C0240001001407A
:104DC0000048004000040240001401400018024066
:104DD00010B586B00446142101A8FBF7B3FCFD49C9
:104DE000206888427ED100BF00200090FA48006809
:104DF00040F40020F84908600846006800F40020EC
:104E0000009000BF00BF00BF00200090F2481038A3
:104E1000006840F00100F049103908600846006859
:104E200000F00100009000BF00BF00BF0020009014
:104E30000846006840F0040008600846006800F07A
:104E40000400009000BF00BF0120019002200290EA
:104E500001200390032004900820059001A9DF4859
:104E6000FEF742F94FF40060019002200290012009
:104E70000390032004900820059001A9D848FEF76C
:104E800033F9D848D8490860400548600021D64821
:104E90008160C1604FF480610161002141618161E5
:104EA000C16101624162FDF7A7FF08B1FCF7B2FBE7
:104EB00000BFCD486063846300BFCA483030CB492F
:104EC00008604FF0006048604021C84881600021C0
:104ED000C1604FF480610161002141618161C16164
:104EE000016200E00AE04162FDF786FF08B1FCF7CD
:104EF00091FB00BFBD482063846328E2BC49206861
:104F000088427DD100BF00200090B348006840F483
:104F10008010B14908600846006800F480100090D5
:104F200000BF00BF00BF00200090AB4810380068F1
:104F300040F00400A849103908600846006800F0F5
:104F40000400009000BF00BF00BF00200090084692
:104F5000006840F0080008600846006800F008009B
:104F6000009000BF00BF8814019002200290012031
:104F70000390032004900820059001A99848FEF7AB
:104F8000B3F8042001900220029001200390032036
:104F900004900820059001A99648FEF7A5F89148CD
:104FA000303895490860C00548600021924881600A
:104FB000C1604FF480610161002141618161C16183
:104FC00001624162FDF718FF08B1FCF723FB00BF47
:104FD00089486063846300BF8248783087490860ED
:104FE0004FF0006048604021844881600021C1602A
:104FF0004FF480610161002141618161C16100E084
:105000000BE001624162FDF7F7FE08B1FCF702FB1D
:1050100000BF7A482063846399E179492068884217
:105020006ED100BF002000906B48001D006840F06A
:1050300010006949091D08600846006800F010006A
:10504000009000BF00BF00BF0020009062481038F1
:10505000006840F0010060491039086008460068A7
:1050600000F00100009000BF00BF4FF4C06001904D
:105070000220029001200390032004900720059055
:1050800001A95648FEF730F85E485F4908604FF0C6
:105090000060486000215C488160C1604FF480611D
:1050A0000161002141618161C16101624162FDF7DD
:1050B000A3FE08B1FCF7AEFA00BF534860638463F7
:1050C00000BF50487830514908604FF00060486098
:1050D00040214E4881600021C1604FF48061016130
:1050E000002141618161C16101624162FDF784FE7D
:1050F00008B1FCF78FFA00BF44482063846326E1BF
:1051000043492068884264D100BF002000903248A3
:10511000006840F48020304908600846006800F4C8
:105120008020009000BF00BF00BF002000902A48F0
:105130001038006840F0020027491039086008461E
:10514000006800F00200009000BF00BF4FF4406014
:105150000190022002900120039003200490072078
:10516000059001A92B48FDF7BFFF1E4818382A49B2
:1051700008604FF000604860002127488160C160EE
:105180004FF480610161002141618161C16101626F
:105190004162FDF731FE08B1FCF73CFA00BF1E4842
:1051A0006063846300BF0F4818301C4908604FF0EB
:1051B000006048604021194881600021C1604FF4BF
:1051C00080610161002141618161C16101624162CF
:1051D00026E02FE0004C0040403802400000024032
:1051E000000802404060024078650120D865012037
:1051F00000500040000C02403866012098660120F3
:105200000010014040640240F86601205867012008
:105210000048004000040240B867012018680120DF
:10522000FDF7EAFD08B1FCF7F5F900BF4948206336
:1052300084638CE0484920688842FAD100BF00208E
:1052400000904648006840F0200044490860084645
:10525000006800F02000009000BF00BF00BF0020E9
:1052600000903E481438006840F004003B4914396F
:1052700008600846006800F00400009000BF00BF0E
:1052800000BF002000900846006840F04000086021
:105290000846006800F04000009000BF00BF80207A
:1052A0000190022002900120039003200490082026
:1052B000059001A92A48FDF717FF4FF4804001909F
:1052C0000220029001200390032004900820059002
:1052D00001A92448FDF708FF2348244908608005F8
:1052E0004860002121488160C1604FF48061016104
:1052F000002141618161C16101624162FDF77CFD74
:1053000008B1FCF787F900BF18486063846300BFE9
:1053100015487830164908604FF0206048604021F9
:10532000134881600021C1604FF480610161002158
:1053300041618161C16101624162FDF75DFD08B1BA
:10534000FCF768F900BF0A482063846300BF06B019
:1053500010BD0000186801200014014044380240CC
:1053600000080240001802402864024078680120CA
:10537000D868012077B581B00446154694F83A0004
:1053800020284FD1029800B115B9012004B070BD9A
:1053900000BF94F83800012801D10220F6E701206F
:1053A00084F8380000BF0298A062A5850020E06361
:1053B000222084F83A000020616BC863616B0864A6
:1053C0001948616BC8640020616B086502AE3268E1
:1053D0002368191D2B46606BFDF784FD00BF00207C
:1053E000009020680068009020684068009000BF2E
:1053F00000BF00BF002084F8380000BF2068C068EC
:1054000040F480702168C8602068406940F0010065
:10541000216848612068406940F040002168486187
:105420000020B3E70220B1E76BCF0108F7B50446CF
:10543000154694F8390020283CD1019800B10DB9E7
:105440000120FEBD00BF94F83800012801D10220E0
:10545000F7E7012084F8380000BF01982062A58496
:10546000E5840020E063212084F839000020216BCE
:10547000C863216B08641048216BC8640020216B4D
:10548000086501AE23681A1D31682B46206BFDF7B5
:1054900029FD6FF040002168086000BF002084F8FB
:1054A000380000BF2068406940F0800021684861F2
:1054B0000020C6E70220C4E76BCF010810B50448FE
:1054C000008840F0020002490880FCF757FC10BD3C
:1054D0008E06002010B50120094908804FF4FA40DB
:1054E00008490860084809490860042048600548E0
:1054F0000068410905488160FDF70EFF10BD0000FE
:105500008C06002088060020003000403869012009
:105510000020002100BF12E000210CE09FED220AD4
:1055200000EB4002214B03EB820202EB810282ED91
:10553000000A4A1CD1B20329F0DB421CD0B2032876
:10554000EADBB7EE000A194A82ED000AB7EE000A5C
:1055500082ED040AB7EE000A82ED080A002012E08C
:1055600000210CE09FED100A00EB4002104B03EB12
:10557000820202EB810282ED000A4A1CD1B20329A9
:10558000F0DB421CD0B20328EADBB7EE000A084A7F
:1055900082ED000AB7EE000A82ED040AB7EE000AB7
:1055A00082ED080A704700000000000060D900206A
:1055B00084D9002010B501200F49087000200F4940
:1055C00008700F49088064200E4908600E48007872
:1055D000012808D10D480068011D64230C4A0D48BC
:1055E000FDF780FC07E0642209490848FFF7C2FE86
:1055F00001200549087010BD4C0500204005002021
:10560000440500204805002058050020F8640120CA
:10561000C4080020B867012010B520480078002891
:105620003BDD1F480088401C1D4908800846008853
:10563000042832DD002008801A48006840681A49B2
:10564000096888420BD0174800684068164908600E
:105650000220124908700020144908801DE00F48FC
:105660000078022819D111480088401C0F49088091
:1056700008460088022810DD01200D4908700A48FC
:105680000068C0F164000B4908800648FDF74EFA37
:105690000020064908800149087010BD4C05002013
:1056A00050050020B8670120480500204E05002065
:1056B000400500204405002070B500240025FFF7B8
:1056C00079FF1FE01048007898B9052002F0CAFF62
:1056D000601CC4B21E2C15DD0C48002101608180C5
:1056E00002200B49088000F055F8022002F0BAFFB2
:1056F00070BD00F05BF80748007810B9FFF75AFF5B
:1057000000E0F5E7DEE7000040050020D8080020B3
:10571000420500205B05002070B505460C460C488C
:105720000480224629460B48FAF79DFF0A48006884
:10573000021D234607490948FDF7D4FB30B108484C
:10574000C079401C0649C87100F024F870BD000003
:1057500042050020D8080020F864012018680120C4
:105760000B09002010B50020054908700549087094
:105770000548028805490648FFF758FE10BD00009D
:10578000580500204C05002042050020D8080020C4
:10579000F864012010B50448FFF733FA01F00AFA63
:1057A000FFF7E0FF10BD0000F86401202DE9F04193
:1057B0002DED028B8AB0142105A8FAF7C3FF14213E
:1057C0006846FAF7BFFF0025002400260027A04600
:1057D000002008EE100A6B4800880C2873DD694829
:1057E0000088142802DD1420664908806548028874
:1057F00065496846FAF737FF6248057863480078DC
:10580000113805287ED2DFE800F00319305F470029
:10581000FA208DF8140004208DF8150081208DF8F1
:1058200016008DF8170004232A4605A96846FBF7E1
:1058300064FB012801D15649087098E0FA208DF8E0
:10584000140004208DF8150089208DF816007920A9
:105850008DF8170004232A4605A96846FBF74DFB7F
:10586000012801D14B49087081E0FA208DF814001D
:1058700004208DF815008C208DF8160076208DF808
:10588000170004232A4605A96846FBF736FB0128C2
:1058900001D1414908706AE0FA208DF81400042013
:1058A0008DF8150088208DF816007A208DF81700E5
:1058B00004232A4605A96846FBF71FFB012801D1EE
:1058C0003649087053E053E0002441E01DF804001D
:1058D000AA283BD1601C1DF80000B0BBA01C1DF81D
:1058E000000090BBE01C1DF8000022282ED1201DD6
:1058F0001DF8000048BB601D1DF80000032825D1DD
:10590000012000E032E026490870A01D1DF80000CB
:105910000106E01D1DF8000001EB004104F1080044
:105920001DF8000001EB002104F109001DF8000042
:10593000084408EE100AB8EE480ADFED1A0A80EEB5
:10594000201A194880ED001A06E0FFE7601CC4B277
:10595000A5F10D00A042B9DA00BF1148007820B9C6
:1059600012488079401C1149887100E000BF04E0B2
:105970000E488079401C0D4988710AB0BDEC028B3D
:10598000BDE8F08144050020C4080020590500202E
:105990005A0500205C0500205D0500205E05002002
:1059A0005B05002000007A44540500200B0900200C
:1059B0001FB500F085FE00F0FFFD00F0CBFD4FF4B9
:1059C00080713248FDF798FC00F062FF01F090F81A
:1059D00001F0B2F800F0E8FF01F038F800F094FFB1
:1059E0002B480088012802D12A48FDF7BDFC00F0B1
:1059F00069FF01F0DFF84FF4E13001F0F7F801F052
:105A0000BDF8FCF7AFFA00F065FBFFF7ABFEFCF763
:105A100009F809F07FFCFFF77BFD1D48008801288D
:105A200002D11C48FDF7A0FC4FF480711748FDF728
:105A300063FCFCF7A5F901F0C3FA05F0FDF924E0D9
:105A400001F06EFD322002F00DFE13480079401C7B
:105A50001149087111480078B8B911480088B0F5AB
:105A6000167F12DD0F480088401C0E490880012077
:105A700000900190029042F22833024601460390C2
:105A800005F02AFF012005490870D9E700140240FB
:105A90008C0600203869012002090020BC05002086
:105AA000780500209205002015E00B4800880128A9
:105AB00002D10A48FDF758FC4FF480710848FDF701
:105AC0001BFCFBF7DDFF022002F0CCFD054840790E
:105AD000401C04494871E8E78C0600203869012021
:105AE000001402400209002015E04FF480710A48BA
:105AF000FDF702FC09480088012802D10848FDF79B
:105B000033FCFBF7DDFB642002F0ACFD0548807937
:105B1000401C04498871E8E7001402408C0600200C
:105B200038690120020900200024002579E03D4861
:105B30000088012802D13C48FDF716FC4FF4807123
:105B40003A48FDF7D9FB601CC4B2092C11DD0024D2
:105B5000681CC5B2042D03DD0025002034490870FF
:105B600034480088401C3349088020213248FDF722
:105B7000C3FB012C01D0062C01D103F089F9022CC2
:105B800001D103F029F92D480088C82806DD00203E
:105B90002A49088003212A48FBF7F2FE2948008899
:105BA000B0F5FA7F12DD2848C078401C2649C8703D
:105BB0000020244908800320244908800122084647
:105BC00001882348FAF794FDFBF798FF21480088E5
:105BD000B0F5FA7F1DDD1C488078401C1A4988709A
:105BE00000201C490880032018490880012208462B
:105BF00001881748FAF77CFDFBF780FF164800780C
:105C0000401C1549087008460078022801DD002074
:105C100008700A2002F026FD1048C079401C0F4988
:105C2000C87184E78C060020386901200014024006
:105C30005C02002078050020001002404A0200208B
:105C40004C020020580200200B09002032020020E4
:105C5000A0070020560200205D020020020900205B
:105C6000002443E04FF480712148FDF745FB2148B3
:105C70000088012802D12048FDF776FB04F050FF90
:105C8000032002F0EFFC1D48007A401C1B490872FB
:105C90001B480088012825D11A480078401C194962
:105CA000087008460078322820DD00200870164869
:105CB000007868B9032C02DD00F0CAF90FE040F269
:105CC000E24012490968486301200F49087006E064
:105CD000FA200E490968486300200B490870601CCF
:105CE000C4B203E00024002006490870BAE70000AF
:105CF000001402408C0600203869012002090020AF
:105D00000000002075050020760500208463012036
:105D100010B506480088012806D100210448FEF786
:105D2000ABFE00200149088010BD000004000020E7
:105D3000FC63012000B585B014216846FAF702FD26
:105D4000AA208DF8000000208DF801008DF80200D7
:105D500020208DF8030000208DF8040001208DF82C
:105D6000050000208DF8060002208DF80700232092
:105D70008DF80800142005490870002004490870B7
:105D800009216846FFF7C8FC05B000BD5905002091
:105D90005B05002030B595B020210DA8FAF7D2FCA4
:105DA000202105A8FAF7CEFC002400250120864911
:105DB00008708649087086480088401C844908801D
:105DC000002084490880844908708448B0F8440061
:105DD000824991F84110824A1278824B1B78CDE9B2
:105DE0000032CDE902107D48B0F8423090F84020F2
:105DF0007D4801787D48007805F06EFD012806D1C8
:105E000001217B48007801F0D9FD15B030BD6E4806
:105E10000078012806D1774890ED000A6F4880EDA0
:105E2000120A05E001217248007801F0C7FDECE795
:105E300066480078012806D16F4890ED000A67484F
:105E400080ED130A05E001216948007801F0B6FDF4
:105E5000DBE7624890ED120ADFED680AB4EEE00A73
:105E6000F1EE10FA53D290ED130AB5EEC00AF1EE3E
:105E700010FA23DD0120594981F8340081F85000DF
:105E8000084690ED120ADFED5E0A20EE200ABCEE15
:105E9000C00A10EE100AA1F85200012081F851004A
:105EA000084690ED130ADFED560A20EE200ABCEEFC
:105EB000C00A10EE100AA1F854007DE00420474902
:105EC00081F83400012081F85000084690ED120A54
:105ED000DFED4B0A20EE200ABCEEC00A10EE100ADD
:105EE000A1F85200022081F85100084690ED130AF3
:105EF000DFED440A30EEC00ADFED410A20EE200A51
:105F0000BCEEC00A10EE100AA1F8540054E0334869
:105F100090ED130AB5EEC00AF1EE10FA24DD03206D
:105F20002E4981F83400012081F85000084690ED98
:105F3000120ADFED330A20EE200ABCEEC00A10EE92
:105F4000100AA1F85200012081F85100084690ED96
:105F5000130ADFED2B0A20EE200ABCEEC00A10EE79
:105F6000100AA1F8540027E002201C4981F83400EF
:105F7000012081F85000084690ED120ADFED200A5A
:105F800020EE200ABCEEC00A10EE100AA1F8520062
:105F9000022081F85100084690ED130ADFED190A3E
:105FA00030EEC00ADFED160A20EE200ABCEEC00A71
:105FB00010EE100AA1F8540000210D48007801F0FD
:105FC000FDFC00BF21E700009005002091050020A6
:105FD0009205002078050020BC050020ECE7002099
:105FE00063020020610200206202002060020020A3
:105FF0005F020020880500208C0500200000B442CC
:106000000000C8420000000010B50C480088A0B98C
:106010000B48007C88B901200849088040F2E24022
:1060200008490968486301200749087000200749AA
:10603000087000210348FEF7F3FC10BD00000020AB
:10604000EC080020846301207605002075050020FF
:1060500010B506480088012806D100210448FEF743
:106060000BFD00200149088010BD00000000002049
:106070008463012010B500240CE0032002F0F2FA42
:10608000601CC4B2322C05DD0648407A401C05492C
:10609000487210BD044800780028EED000F042F8A5
:1060A00000BFF6E70B0900203005002010B50020E6
:1060B0000549087005490870054908804FF4E1302A
:1060C00000F022F810BD00003C0500203005002043
:1060D0003205002010B54620064908600020064918
:1060E000087006490880462205490648FFF742F92C
:1060F00010BD0000340500203005002032050020CE
:10610000680400203865012010B504460448FEF7F5
:1061100078FD204600F06AFDFFF7DCFF10BD0000AF
:106120003865012070B52DED068B82B00024002566
:10613000002600200190DEE1F348005D552802D0E2
:10614000601C84B2D7E1601C84B2EF48005D512826
:1061500004D0522803D053287ED101E000BF00BFF5
:106160000026601E85B205E0E748405D3044C6B2B7
:10617000681C85B204F109008542F5DBE248405D08
:10618000B0426AD1E048005D512867D1DE4A611C07
:10619000525CDD4BA11C595C02EB012009F04FFB66
:1061A00041EC1A0B9FEDD90B53EC102B09F0C0F901
:1061B00041EC190B9FEDD70B53EC102B09F0A6FB0C
:1061C00041EC180B09F0CEF8D4490860CE4AE11C26
:1061D000525CCD4B211D595C02EB012009F02FFBD5
:1061E00041EC1A0B9FEDC90B53EC102B09F0A0F9F1
:1061F00041EC190B9FEDC70B53EC102B09F086FBFC
:1062000041EC180B09F0AEF8C4494860BE4A611D64
:10621000525CBD4BA11D595C02EB012009F00FFB44
:1062200041EC1A0B9FEDB90B53EC102B09F080F9E0
:1062300041EC190B9FEDB70B53EC102B09F066FBEB
:1062400041EC180B09F08EF8B4498860AE4AE11DA4
:10625000525CAD4B491C02E036E132E11EE0595C74
:1062600002EB012009F0EBFA41EC1A0B9FEDAC0BAD
:1062700053EC102B09F05CF941EC190B9FEDAA0BC4
:1062800053EC102B09F0A0F841EC180B09F06AF858
:10629000A749086001208DF804000EE19A48005DCE
:1062A00052287CD1984A611C525C974BA11C595CC6
:1062B00002EB012009F0C3FA41EC1A0B9FED930B9E
:1062C00053EC102B09F034F941EC190B9FED990BAD
:1062D00053EC102B09F01AFB41EC180B09F042F8B3
:1062E00096490860884AE11C525C874B211D595C25
:1062F00002EB012009F0A3FA41EC1A0B9FED830B8E
:1063000053EC102B09F014F941EC190B9FED890B9C
:1063100053EC102B09F0FAFA41EC180B09F022F8B3
:1063200086494860784A611D525C774BA11D595CD3
:1063300002EB012009F083FA41EC1A0B9FED730B7D
:1063400053EC102B09F0F4F841EC190B9FED790B8D
:1063500053EC102B09F0DAFA41EC180B09F002F8B3
:1063600076498860684AE11D525C674B491C595C5C
:1063700002EB012009F063FA41EC1A0B9FED680B68
:1063800053EC102B09F0D4F841EC190B9FED660B80
:1063900053EC102B09F018F841EC180B00E007E063
:1063A00008F0E0FF6249086001208DF8050084E0F4
:1063B000554A611C525C544BA11C595C02EB0120F4
:1063C00009F03DFA41EC1A0B9FED500B53EC102BEA
:1063D00009F0AEF841EC190B9FED590B53EC102B63
:1063E00009F094FA41EC180B08F0BCFF564908601C
:1063F000454AE11C525C444B211D595C02EB0120D3
:1064000009F01DFA41EC1A0B9FED400B53EC102BD9
:1064100009F08EF841EC190B9FED490B53EC102B52
:1064200009F074FA41EC180B08F09CFF46494860EB
:10643000354A611D525C344BA11D595C02EB0120B1
:1064400009F0FDF941EC1A0B9FED300B53EC102BCA
:1064500009F06EF841EC190B9FED390B53EC102B42
:1064600009F054FA41EC180B08F07CFF36498860BB
:10647000254AE11D525C244B491C595C02EB01206A
:1064800009F0DDF941EC1A0B9FED250B53EC102BB5
:1064900009F04EF841EC190B9FED230B53EC102B38
:1064A00008F092FF41EC180B08F05CFF20490860EF
:1064B00001208DF806002549087004F10A0084B215
:1064C00001E0601C84B200E000BF00BF1F480078FC
:1064D000012803D102B0BDEC068B70BD9DF804000D
:1064E0009DF8051008449DF806100844032801D1C2
:1064F0000120EFE700BF164800880C38A0423FF7A4
:106500001BAE0020E6E70000680400200000000049
:106510000000E0400000000000003040A008002023
:10652000000000000090AA400000000000000D40A4
:10653000380500200000000000409F40AC0800200B
:106540000000000000806640B80800203C050020E4
:106550003205002010B51448144908604FF480300B
:106560004860002111488160016181610162C1625E
:106570000F4981620021C1600121C16100210163D5
:1065800001214161FCF7B2F908B1FBF743F808209B
:10659000084908600120486088600448FBF7B6FF9E
:1065A00008B1FBF737F810BD00200140546101200D
:1065B0000100000F9C61012008B500BF0020009081
:1065C0003E48006840F480003C4908600846006886
:1065D00000F48000009000BF00BF00BF00200090CA
:1065E0000846006840F4001008600846006800F49F
:1065F0000010009000BF00BF022211460B20FCF7E4
:106600002AFF0B20FCF71AFF022211460C20FCF790
:1066100022FF0C20FCF712FF022211460D20FCF78E
:106620001AFF0D20FCF70AFF022211460E20FCF78C
:1066300012FF0E20FCF702FF022211460F20FCF78A
:106640000AFF0F20FCF7FAFE022211462F20FCF76A
:1066500002FF2F20FCF7F2FE022211463820FCF741
:10666000FAFE3820FCF7EAFE022211463920FCF738
:10667000F2FE3920FCF7E2FE022211463A20FCF736
:10668000EAFE3A20FCF7DAFE022211463B20FCF734
:10669000E2FE3B20FCF7D2FE022211464520FCF729
:1066A000DAFE4520FCF7CAFE022211464620FCF71E
:1066B000D2FE4620FCF7C2FE08BD00003038024082
:1066C00000B587B0142102A8FAF73CF800BF0020FB
:1066D00001906948006840F010006749086008466A
:1066E000006800F01000019000BF00BF00BF002054
:1066F00001900846006840F02000086008460068E5
:1067000000F02000019000BF00BF00BF00200190FA
:106710000846006840F0010008600846006800F084
:106720000100019000BF00BF00BF0020019008469B
:10673000006840F0020008600846006800F00200AF
:10674000019000BF00BF00BF002001900846006814
:1067500040F0400008600846006800F040000190EA
:1067600000BF00BF00BF002001900846006840F055
:10677000040008600846006800F00400019000BFB3
:1067800000BF00BF002001900846006840F00800EC
:1067900008600846006800F00800019000BF00BFD4
:1067A000002220213548FCF7ABFD00224FF4807118
:1067B0003348FCF7A5FD00224AF240013148FCF7BE
:1067C0009FFD002240213048FCF79AFD0022C021A5
:1067D0002E48FCF795FD2020029001200390002018
:1067E0000490059002A92548FCF77EFC4FF48070C8
:1067F00002900120039000200490059002A92048F7
:10680000FCF772FC4FF4204002900120039000201E
:106810000490059002A91B48FCF766FC40200290FA
:1068200011200390002004900220059002A9154831
:10683000FCF75AFC402002900120039000200490B5
:10684000059002A91048FCF74FFC4FF480500290CD
:1068500000200390049002A90A48FCF745FCC020E0
:1068600002900120039000200490059002A907489F
:10687000FCF73AFC07B000BD30380240001002407F
:1068800000140240001802400008024000040240C8
:1068900010B50A480A490860002048607F2108486E
:1068A0008160FF21C1600021016141618161FDF7CB
:1068B000ADFA08B1FAF7AEFE10BD000000280040A6
:1068C000AC61012010B50E480E4908604FF482708B
:1068D000486000210B488160C160016141614FF453
:1068E000007181611821C1610021016241628162F0
:1068F0000A21C162FDF720FB08B1FAF78BFE10BD3B
:1069000000300140F461012000B58DB000200990F5
:106910000A900B900C90079008901C216846F9F79C
:1069200011FF1F481F490860A720486020211D480B
:1069300081603221C16000210161FDF726FD08B1AF
:10694000FAF768FE4FF48050099009A91548FDF741
:10695000E4FD08B1FAF75EFE1248FEF744F808B10C
:10696000FAF758FE00200790089007A90D48FDF798
:10697000DBFC08B1FAF74EFE602000907D2001900C
:10698000002002900490002269460648FDF7A7FF08
:1069900008B1FAF73FFE0348FDF724FF0DB000BD34
:1069A00000480140FC63012000B58DB00020099033
:1069B0000A900B900C90079008901C216846F9F7FC
:1069C000C1FE204820490860A720486020211E48B9
:1069D000816042F21071C160002101614161FDF7E7
:1069E000D4FC08B1FAF716FE4FF48050099009A9BB
:1069F0001548FDF792FD08B1FAF70CFE1248FDF7B5
:106A0000F2FF08B1FAF706FE00200790089007A9E8
:106A10000D48FDF789FC08B1FAF7FCFD60200090F5
:106A2000FA20019000200290049000226946064856
:106A3000FDF755FF08B1FAF7EDFD0348FDF7D2FE6B
:106A40000DB000BD000001408463012000B58DB091
:106A5000002009900A900B900C90079008901C2140
:106A60006846F9F76FFE4FF08040204908605320D8
:106A7000486020211D4881604FF47A71C160002177
:106A80000161FDF782FC08B1FAF7C4FD4FF48050B4
:106A9000099009A91548FDF740FD08B1FAF7BAFDBC
:106AA0001248FDF7A0FF08B1FAF7B4FD00200790E7
:106AB000089007A90D48FDF737FC08B1FAF7AAFDC1
:106AC0006020009040F2DC50019000200290049081
:106AD000002269460548FDF702FF08B1FAF79AFD62
:106AE0000248FDF77FFE0DB000BD0000C06301202D
:106AF0001CB50020009001900D480E49086014203C
:106B0000486000210B4881604FF47A61C160FDF755
:106B10003CFC08B1FAF77EFD002000900190694628
:106B20000448FDF701FC08B1FAF774FD1CBD000034
:106B3000001000400C6301201CB500200090019063
:106B40000C480D4908601420486000210A48816003
:106B50006421C160FDF719FC08B1FAF75BFD002064
:106B60000090019069460448FDF7DEFB08B1FAF792
:106B700051FD1CBD001400404863012010B50B48B6
:106B80000B4908604FF416504860002108488160A6
:106B9000C16001610C21416100218161C161FEF789
:106BA00048F808B1FAF736FD10BD000000100140AA
:106BB000B864012010B50B480B4908604FF49640AB
:106BC0004860002108488160C16001610C21416179
:106BD00000218161C161FEF72CF808B1FAF71AFDB6
:106BE00010BD000000480040F864012010B50446C4
:106BF00009480A4908600846446000218160C16074
:106C000001610C21416100218161C161FEF711F830
:106C100008B1FAF7FFFC10BD0014014038650120EF
:106C20002DED068BD0ED009AB0EE695AD0ED019AA9
:106C3000F0EE695AD0ED029AB0EE696AD0ED039A8F
:106C4000F0EE696AD0ED049AB0EE697AD0ED059A5B
:106C5000F0EE697AD0ED069AB0EE698AD0ED079A27
:106C6000F0EE698AD0ED089AB0EE699A65EE079A5F
:106C700069EE899AB0EE690A25EEA7AAF0EE409A6D
:106C80004AEE089AB0EE690A26EE26AAF0EE409A7D
:106C90004AEE289AB0EE690A26EE07AAF0EE409A6C
:106CA0004AEE489AB0EE690A25EEA6AAF0EE409A9E
:106CB0004AEE499AB0EE690A25EE27AAF0EE409A0C
:106CC0004AEE689AB0EE690AD0ED009AF0EE690AD1
:106CD000D0ED019AB0EE691AD0ED029AF0EE691A81
:106CE000D0ED039AB0EE692AD0ED049AF0EE692A4D
:106CF000D0ED059AB0EE693AD0ED069AF0EE693A19
:106D0000D0ED079AB0EE694AD0ED089AF0EE694AE4
:106D100062EEA49A44EE439A89EE80AA81ED00AA1D
:106D200064EE219A41EE649A89EE80AA81ED01AA6F
:106D300061EE039A41EEE29A89EE80AA81ED02AA01
:106D400063EE239A44EEC29A89EE80AA81ED03AAEB
:106D500064EEA09A41EEE39A89EE80AA81ED04AA3E
:106D600061EE829A40EEC39A89EE80AA81ED05AA6F
:106D700062EE049A43EEE29A89EE80AA81ED06AAB9
:106D800063EE819A40EEC49A89EE80AA81ED07AA4B
:106D900060EEA29A41EE429A89EE80AA81ED08AA9D
:106DA000BDEC068B704700002DE9F04104460D460E
:106DB00000260027002C14DD601EC0EB00103E49A9
:106DC00001EB001000EB85008078012809D1601EDE
:106DD000C0EB001001EB001030F825000744701CD8
:106DE00086B236484179C07B0844401CA04214DD7D
:106DF000601CC0EB0010304901EB001000EB850077
:106E00008078012809D1601CC0EB001001EB001054
:106E100030F825000744701C86B2002D15DDC4EB48
:106E20000410254901EB0011681E01EB80008078F9
:106E300001280AD1C4EB04101F4901EB0011681EA0
:106E400031F820000744701C86B21C48C17990F8C4
:106E500025000844401CA84215DDC4EB0410164967
:106E600001EB0011681C01EB8000807801280AD139
:106E7000C4EB0410104901EB0011681C31F820002C
:106E80000744701C86B2002E14DDB7FBF6F0C4EB8D
:106E90000411094A02EB011121F825000120C4EB7D
:106EA000041102EB011101EB85018870E9B2E0B237
:106EB000FBF7B4F9BDE8F08158010120A8D9002002
:106EC00070B58AB0142105A8F9F73CFC1421684676
:106ED000F9F738FC00260024002505208DF8140061
:106EE0001C4800788DF8150003208DF816001B2033
:106EF0008DF8170000208DF818006A46052105A8B6
:106F0000FBF788F9064631466846FAF739FD002056
:106F1000114908701149087012E00A2001F0A2FB23
:106F2000601CC4B20E2C0BDD0024681CC5B2032DFE
:106F300002DD01200AB070BD31466846FAF720FD37
:106F4000054800780028E8D0044800780028E4D0FC
:106F50000020EFE7780600204402002045020020D0
:106F600010B590B0202108A8F9F7ECFB2021684665
:106F7000F9F7E8FB0024104800788DF820000F484E
:106F800000788DF8210003208DF8220006208DF86E
:106F9000230002208DF8240000208DF825006A4689
:106FA000062108A8FBF736F9044621466846FAF799
:106FB000E7FC10B010BD00005B0200207806002046
:106FC00000B599B0042208213048FAF76DFF0E226F
:106FD000102115A8FAF768FFBDF854002C49088065
:106FE000BDF856002B490880BDF858002A49088092
:106FF000BDF85A0029490880BDF85C00284908807E
:10700000BDF85E00274908809DF860002649087099
:107010009DF861002549087023480078012803D0B5
:1070200021480078FF2802D102201F49087002225F
:10703000402105A8FAF738FF9DF81400012801D176
:107040001B490870122220216846FAF72DFFBDF86F
:10705000000018490880BDF8020017490880BDF8F3
:10706000040016490880BDF8060015490880BDF8DF
:10707000080014490880DDF80A0013490860DDF8AB
:107080000E001249086019B000BD00007C06002007
:107090009405002096050020980500209A05002000
:1070A0009C0500209E05002078060020A6050020F3
:1070B000C0050020A8050020AA050020AC0500207E
:1070C000AE050020A4050020B0050020B405002076
:1070D00010B590B0202108A8F9F734FB20216846AC
:1070E000F9F730FB0024104800788DF820000F4895
:1070F00000788DF8210003208DF8220007208DF8FC
:10710000230002208DF8240000208DF825006A4617
:10711000062108A8FBF77EF8044621466846FAF7E0
:107120002FFC10B010BD00005B020020780600208C
:1071300030B52DED0A8B83B000240025002000908F
:107140000190029004F062FB01280ED1D849087525
:107150008DF80000022269464FF4AA4003F082FE37
:10716000012003B0BDEC0A8B30BD04F017FA0128F2
:107170000DD1CF4988748DF80000022269464FF482
:10718000A64003F06FFE0020CA49087002E001200B
:10719000C8490870C848006808F0AEFE41EC1B0BF7
:1071A0009FEDC60B53EC102B08F0B0FB41EC1A0B13
:1071B0009FEDC40B53EC102B08F0BAF941EC190BFE
:1071C000B0EE490AF0EE690A07F0CEF8B0EE408A58
:1071D000F0EE608A51EC180B08F0C4F8BB49086067
:1071E0009FEDBB0A084680ED010AB348006808F02D
:1071F00083FE41EC1B0B9FEDB10B53EC102B08F001
:1072000085FB41EC1A0B9FEDAF0B53EC102B08F0F4
:107210008FF941EC190BB0EE490AF0EE690A07F05C
:1072200007F9B0EE408AF0EE608A51EC180B08F0D6
:1072300099F8A64988609FEDA60A084680ED030AE2
:10724000B7EE000A80ED040A9FEDA10A80ED050A61
:107250009948006808F050FE41EC1C0B9FED970B1D
:1072600053EC102B08F052FB41EC1B0B9FED950BE0
:1072700053EC102B08F05CF941EC1A0BB0EE4A0A03
:10728000F0EE6A0A07F0D4F8B0EE409AF0EE609A99
:1072900051EC190B08F05AF841EC180B08F062F8A1
:1072A0008A4988619FED8A0A084680ED070A82486C
:1072B000006808F021FE41EC1B0B9FED800B53ECA6
:1072C000102B08F023FB41EC1A0B9FED7E0B53ECC7
:1072D000102B08F02DF941EC190BB0EE490AF0EE35
:1072E000690A07F041F8B0EE408AF0EE608A51EC8E
:1072F000180B08F037F875490862B7EE000A7548B0
:1073000080ED000A9FED720A80ED010A9FED700A80
:1073100080ED020A9FED6E0A80ED030A6E48006858
:1073200008F0EAFD41EC1B0B9FED640B53EC102BB6
:1073300008F0ECFA41EC1A0B9FED620B53EC102BAA
:1073400008F0F6F841EC190BB0EE490AF0EE690AC4
:1073500007F00AF8B0EE408AF0EE608A51EC180BA4
:1073600008F000F85B4908615B48006808F0C4FD5C
:1073700041EC1C0B9FED510B53EC102B08F0C6FA9F
:1073800041EC1B0B9FED4F0B53EC102B08F0D0F88A
:1073900041EC1A0BB0EE4A0AF0EE6A0A07F048F820
:1073A000B0EE409AF0EE609A51EC190B07F0CEFF68
:1073B00041EC180B07F0D6FF464948619FED440A9F
:1073C000084680ED060A4448006808F095FD41EC47
:1073D0001B0B9FED3A0B53EC102B08F097FA41EC86
:1073E0001A0B9FED380B53EC102B08F0A1F841EC71
:1073F000190BB0EE490AF0EE690A07F019F8B0EE81
:10740000408AF0EE608A51EC180B07F0ABFF31496F
:10741000C8613148006808F06FFD41EC1B0B9FED1F
:10742000270B53EC102B08F071FA41EC1A0B9FED6F
:10743000250B53EC102B08F07BF841EC190BB0EE48
:10744000490AF0EE690A06F08FFFB0EE408AF0EECE
:10745000608A51EC180B07F085FF1E490862002472
:1074600012E000250CE09FED1A0A04EB44001B49D2
:1074700001EB800000EB850080ED000A681CC5B2BE
:10748000032DF0DB601CC4B2032CEADBB7EE000A6C
:10749000124880ED000AB7EE000A80ED040AB7EE4C
:1074A000000A80ED080A0E49FFF7BAFB002058E6F3
:1074B000EC080020BA05002080050020F1D4C85354
:1074C000FB210940000000000080664018D9002020
:1074D000000000003CD900207C05002060D900207D
:1074E00084D9002000B591B00020094908700949ED
:1074F000087009490870094908708DF804008DF872
:107500000A000822402101A8FAF77EFD11B000BD53
:10751000BE050020BF050020C1050020BB050020DE
:1075200000B593B00020019002905F4800780128D8
:1075300055D15E48C07B012803D05C48C07B02283F
:1075400008D100F051F958480078012808D100F01E
:10755000CBF805E05548C07B032801D100F0C4F802
:107560005148007801283AD104F012FE50480078C2
:10757000012803D14F480078FAF7BEF800204E49A1
:1075800008704E490870484908708DF80C000120B9
:107590008DF812004A4800894A4908804848408AC4
:1075A00009880844474908804548808B0988084471
:1075B000444908804248C08C0988084441490880F1
:1075C00001208DF8130008460088ADF814000A2247
:1075D000402103A8FAF718FD00203B4908703B48FA
:1075E0000078012811D13848007870B90020374957
:1075F000087002203449087003F030FE012801D1E0
:10760000FFF7AEFC002030490870314800780128AF
:1076100011D12D48007870B900202D490870022042
:107620002949087003F084FE012801D1FFF750FDBD
:1076300000202549087027480078012813D102202E
:107640002149087005F0EEFA012805D10022012138
:107650002148007806F056FA00201B4908701D49A1
:1076600008701D4908701D480078012809D10220C2
:1076700015490870FEF78EFB002013490870174962
:1076800008701748008801280CD102200E490870A4
:1076900005F040F800200C490870114908800120CD
:1076A0001049088013B000BDC1050020ECE70020A0
:1076B000C30500205B020020BE050020BF0500209E
:1076C000A8D90020B8050020BB050020190600201D
:1076D0001A060020DB050020DC0500205E020020E9
:1076E000280600202A0600202DE9F0410026002768
:1076F0000024002539484179C07B0844801CC6B26B
:107700003648C17990F825000844801CC7B200BFF4
:1077100015E000250FE0C4EB0410314901EB001027
:1077200000EB85008078012803D12946204605F02A
:1077300019FC681C85B2BD42EDDB601C84B2B4420A
:10774000E7DB00241CE0002516E0C4EB041024490C
:1077500001EB001000EB8500807858B929462046DF
:10776000FFF722FB1F480078012803D1E9B2E0B2FD
:1077700004F0C0FA681C85B2BD42E6DB601C84B22E
:10778000B442E0DB701E84B222E0781E85B218E0BD
:10779000C4EB0410124901EB001000EB8500807867
:1077A00058B929462046FFF7FFFA0E48007801280D
:1077B00003D1E9B2E0B204F09DFA05B903E0681E16
:1077C00085B2002DE4DA00BF04B903E0601E84B284
:1077D000002CDADA00BFBDE8F0810000A8D9002053
:1077E00058010120C305002030B591B0202109A81F
:1077F000F8F7A8FF202101A8F8F7A4FF002400252E
:10780000C0E06448C07B8DF824000122422109A811
:10781000FAF7FAFBAAE05F48007C00EB80005E49C3
:1078200001EB4000407800B99BE05A48007C8DF89D
:1078300024000122432109A8FAF7E6FB5549087CF8
:10784000F9F702F90020534908830846007C00EB51
:107850008000514901EB400040884E49488208466B
:10786000007C00EB80004C4911F810004949087574
:10787000002081F86A000846007C00EB8000464941
:1078800001EB40000079434948755DE04148007CC8
:1078900000EB8000404901EB400080793D4988754C
:1078A00041E004F009FA012801D111B030BD394896
:1078B000407D00EB8000394901EB40103549897D5E
:1078C00000EB8100807840BB3248008B08B9FAF7A2
:1078D000DDFD01F051FB2F4A2832A2F10C013048A6
:1078E000F9F72EFB01F0C0FB02F0B4F8012800D13B
:1078F00019E002F0D1FA012800D114E002F092FC64
:10790000012805D12348807D401C224988750AE062
:107910002049087C02F012FE04E01E48807D401CD5
:107920001C49887500BF1B48807D1A49097C01EB02
:107930008101194A02EB4101C9798842B1DD15483C
:10794000407D401C134948751248407D1149097C0F
:1079500001EB8101104A02EB41014979884295DD32
:1079600000BF0C48007C401C0A4908740948007C90
:107970000428FFF650AF0020064908740846C07B73
:10798000401CC8730348C07B0328FFF63AAF00BF12
:107990008BE70000ECE70020A8D9002058E8002081
:1079A00084D9002010B50448008840F00400024942
:1079B0000880FAF7E3F910BD8E06002070B592B08A
:1079C00004460D4620210AA8F8F7BCFE202102A893
:1079D000F8F7B8FE002603208DF8280004208DF863
:1079E000290035BB01208DF82A00214890F850006D
:1079F0008DF82B001E48B0F85200000A8DF82C00BC
:107A00001B4890F852008DF82D0001208DF82E00B3
:107A1000174890F851008DF82F001548B0F8540021
:107A2000000A8DF83000124890F854008DF83100AB
:107A300010E0FF208DF82A008DF82B008DF82C0027
:107A40008DF82D008DF82E008DF82F008DF8300068
:107A50008DF83100022302AA0A210AA8009400F03E
:107A600031F80646314602A8F9F78AFF12B070BD18
:107A7000ECE7002010B50448008840F001000249FE
:107A80000880FAF77BF910BD8E06002002480068D6
:107A9000C0F30220704700000CED00E010B5002894
:107AA00007DA0A07140E054A00F00F031B1FD4540F
:107AB00003E00A07130E024A135410BD18ED00E04C
:107AC00000E400E02DE9F04707460D4614469846CD
:107AD000DDF8209000266820207005F10900607014
:107AE00016480078A07084F8038084F80490144845
:107AF0000078607112480078A07107212046FAF7DB
:107B0000A7FC0646300AE07126722A46394604F17F
:107B10000900F8F7A8FD29463846FAF799FC064609
:107B2000310A05F109002154401C26541621401C3D
:107B30002154401CC0B2BDE8F0870000650200205F
:107B4000780600202DE9F047044689469246C8464B
:107B5000002500260027BEE1605D682879D1681CF9
:107B6000265C0D2E75DBA8F10300B042FADBA819E4
:107B7000801C205C1628F1D160190721FAF768FCF7
:107B80000746E81D205CB0EB172FE7D1F9B205F1ED
:107B90000800205C8142E1D1A6F1090291B205F111
:107BA0000902A018FAF754FC0746A819205CB0EBAC
:107BB000172FD3D1F9B2A819401C205C8142CDD136
:107BC000E81C205C01287BD1281D205CFF2822D1E5
:107BD00005F10900205C03280ED105F10A00205CA4
:107BE0000A2809D105F10B00205C012804D1691D88
:107BF000605C01F07FF965E105F10900205C032874
:107C0000F9D105F10A00205C2128F4D1691D605CDE
:107C1000F9F724F956E1281D205CB2490978884219
:107C2000E9D1A81C205CB049087005F10900205C6E
:107C30000328E0D105F10A00205C122863D009DC9A
:107C400004287BD00A280CD00D287CD00E2877D1B0
:107C500016E03AE1132834D0212872D02328F6D137
:107C6000D3E005F10B00205C032808D105F10C00DE
:107C7000205C9C490870691D605C01F03BF9F5E0EF
:107C800005F10B00205C052803D10120F9F798FDD0
:107C900015E005F10B00205C022810D105F10C0065
:107CA000205C01280BD105F10D00205C012806D1D4
:107CB00005F10E00205C012801D1FEF7A5F9D5E001
:107CC000D5E005F10C00205C88490978884219D17B
:107CD00005F10F00205CEE2814D105F10D00205CA9
:107CE00077280FD105F10E00205C88280AD1804842
:107CF0000078401C7E49087008460078012801DDA4
:107D000000BFFEE7B2E005F10B00205C012804D1C2
:107D100000207849088000BFFEE705F10B00205CD9
:107D200002280FD105F10C00205C704909788842C7
:107D300008D100206F49088000BFFEE714E002E090
:107D400093E05DE092E005F10B00205C01280AD190
:107D500005F10C00205C65490978884203D1691D52
:107D6000605CF9F779F881E063480078F0BB63481C
:107D70000078D8BB681D205C6149087005F10B00D4
:107D8000205C6049087005F10C00205C5E490870B9
:107D900005F10D00205C5D4981F8400005F10F0000
:107DA000215C401E205C01EB00205849A1F84200F4
:107DB00005F11000205C5649087005F11100205CA7
:107DC0005449087005F11200205C504981F84100C7
:107DD00005F11400215C401E205C01EB00204B49A2
:107DE000A1F8440005F11500205C00E007E04A49D5
:107DF000087001204049087002204049087035E0B1
:107E0000691D605CF9F72AF830E005F10B00205C91
:107E1000012804D1691D605CF8F7E0FF24E005F15A
:107E20000B00205C02281FD105F10C00205C2D49BD
:107E30000978884218D105F10D00205C010605F192
:107E40000E00205C01EB006105F10F00205C01EBEE
:107E5000006105F11000205C0844304908600422EC
:107E600008212E48FAF7D0F800E000BF2AE0E81C0D
:107E7000205C032826D105F10900205C032821D1CC
:107E800005F10A00205C042814D00A2818D105F155
:107E90000B00205C01280CD105F10C00205C11497D
:107EA0000978884203D101201D49087001E003F0E0
:107EB000ABF906E005F10B016018F9F7ADFB00E046
:107EC00000BF00BF0020BDE8F087A8F101001FFA45
:107ED00080F8681C85B2B8F1100FBFF63DAE0120E6
:107EE000F1E70000780600206502002075060020FA
:107EF0005C0200208C0600205E020020BB050020F2
:107F00005F0200206002002062020020ECE70020F7
:107F10006102002063020020DA0500207C060020B8
:107F20004602002010B500F013F800F0CDFC00F080
:107F3000F5FC00F015FD00F09DFC00F05DFC00F08C
:107F4000A9FD00F04DFD00F073FD00F002F810BD3A
:107F50007047704706480078012808D10548007826
:107F6000FF2804D203480078401C0249087070477B
:107F7000520600204506002010B500241A4800785B
:107F8000012830D1F8F794FA04461848007820B157
:107F900016480078401E1549087014480078F8B952
:107FA00013480078E0B900F0D7FD1248124909786B
:107FB00050F82100114908600F48007810490978ED
:107FC00088420DD00D480068806B401C0B49096841
:107FD00088630C480068401C0A490860F8F788FA72
:107FE0002046F8F769FA10BD520600204506002029
:107FF00046060020EC5B01204806002060060020B9
:10800000470600202C06002010B50B48007890B9D8
:1080100000F0A2FD0948007809490870094807499D
:10802000097850F8210008490860084600680749A7
:108030000860F8F744FA10BD5206002048060020F8
:1080400047060020EC5B0120600600205806002057
:10805000704700002DE9FE4F06460F4690461C462D
:108060004FF00009F8F724FA81461F48007828B13C
:108070004846F8F721FA3C20BDE8FE8F1B4850F82F
:10808000240060BB0120194941F824004846F8F754
:1080900013FA002342463946304600F0B5F98246CD
:1080A000002000900190034602465146029020466F
:1080B00000F068FD054635B90D48007801280CD15F
:1080C00000F010FD09E0F8F7F3F9814600200749B8
:1080D00041F824004846F8F7EFF92846CCE748462F
:1080E000F8F7EAF92820C7E745060020EC5B0120F5
:1080F000520600202DE9F04F85B081468A4693460E
:108100001C46DDE90F78129D00200390F8F7D0F9A6
:1081100003902348007830B10398F8F7CDF93C205C
:1081200005B0BDE8F08F1F4850F8240088BB01203F
:108130001C4941F824000398F8F7BEF92A46414645
:10814000384600F03BFE2B465A465146484600F062
:108150005BF904901198CDE9008002953A462046DB
:108160000E9B049900F00EFD064636B90E480078C5
:1081700001280CD100F0B6FC09E0F8F799F903905A
:108180000020084941F824000398F8F795F9304693
:10819000C6E7FFE70398F8F78FF92820C0E700004B
:1081A00045060020EC5B01205206002070470000CD
:1081B0002DE9F041054600274748007810B14020DE
:1081C000BDE8F0813F2D01D13E20F9E7F8F770F9C5
:1081D0000746FF2D03D14148006890F832504048CF
:1081E00050F8254024B93846F8F766F94320E7E708
:1081F000012C04D13846F8F75FF93D20E0E714F888
:10820000340F3849085C617888432178354A5054E6
:1082100014F834091146085C30B994F83610324825
:108220000078884330490870E06918B12046E16958
:1082300000F0CCFA666A16B1304600F009FB002067
:10824000E06284F8300084F8310028480078FF2884
:1082500004D226480078401C244908703846F8F7B4
:108260002BF900F0B2FAF8F723F907461F48007817
:1082700020B11E480078401E1C490870204600F0BE
:1082800041F81B480078401E194908700020144925
:1082900041F82500A06930B900206169886115495D
:1082A0006069086005E0D4E905014861D4E905107A
:1082B00088611148006860610F4804600FA0E064A5
:1082C0003846F8F7F9F80E480078012801D100F097
:1082D00009FC002074E70000450600205806002035
:1082E000EC5B01204A0600204906002046060020DB
:1082F00053060020640600205C0600203F000000BA
:1083000052060020704770472DE9F04106460F469F
:1083100014464FF000081548007818B1122020705C
:10832000BDE8F081F8F7C4F88046FF2E03D110486D
:10833000006890F832600F4850F826502DB940463A
:10834000F8F7BAF843202070EAE7012D05D140463E
:10835000F8F7B2F843202070E2E7EF644046F8F700
:10836000ABF80020207000BFDAE7000045060020CF
:1083700058060020EC5B0120704770472DE9F0475C
:1083800007460D464FF0000A002028606860F8F7A5
:108390008FF88246FF2F03D11948006890F8327099
:1083A000184850F827402CB95046F8F785F8432074
:1083B000BDE8F087012C04D15046F8F77DF8432042
:1083C000F6E7207C00F0010020B95046F8F774F879
:1083D0004520EDE70026D4F80C90D4F808805046EC
:1083E000F8F76AF800E0761C58F8041B0029FAD068
:1083F000B0002860A9EB0600800068600020D7E785
:1084000058060020EC5B012070B50446104600269B
:10841000051F28462E604FF48056051F28462E6003
:108420001526051F28462E601426051F28462E6097
:108430001326051F28462E601226051F28462E608B
:108440001126051F28462E601026051F28462E607F
:108450000926051F28462E600826051F28462E607F
:108460000726051F28462E600626051F28462E6073
:108470000526051F28462E600426051F28462E6067
:108480000326051F28462E600226051F28462E605B
:108490000126051F28462E600026051F28462E604F
:1084A0004FF080750560051F28462C60414E051F62
:1084B00028462E604FF01236051F28462E604FF0DA
:1084C0000336051F28462E604FF00236051F28464A
:1084D0002E607610051F28462E60051F284629604D
:1084E0003126051F28462E603026051F28462E609F
:1084F0002926051F28462E602826051F28462E609F
:108500002726051F28462E602626051F28462E6092
:108510002526051F28462E602426051F28462E6086
:108520002326051F28462E602226051F28462E607A
:108530002126051F28462E602026051F28462E606E
:108540001926051F28462E601826051F28462E606E
:108550001726051F28462E601626051F28462E6062
:108560004FF01136051F28462E604FF01036051FBC
:1085700028462E604FF00936051F28462E604FF022
:108580000836051F28462E604FF00736051F28467F
:108590002E604FF00636051F28462E604FF0053638
:1085A000051F28462E604FF00436051F28462E6012
:1085B00070BD0000E18C01082DE9F04105464FF047
:1085C0000008F7F775FF8046FF2D05D120480068A9
:1085D00090F83250012608E01D48006890F83200FB
:1085E000A84201D1012600E000261A4850F8254093
:1085F0002CB94046F7F760FF4820BDE8F081012C18
:1086000004D14046F7F758FF4320F6E794F834705A
:108610001148C05D94F8351088430F49C855084685
:10862000C05D30B994F836100C48007888430B4987
:10863000087094F8300040F0080084F8300040469C
:10864000F7F73AFF012E01D100F04CFA0020D4E7F1
:1086500058060020EC5B01204A0600204906002055
:108660007047000070B5054600261748007800B135
:1086700070BD1648007800B1FAE71DB3F7F718FF90
:1086800006461348006890F834401248005D1049CF
:10869000096891F8351088430E4908550846005D71
:1086A00040B90B48006890F836100B4800788843B2
:1086B0000949087006480068C5623046F7F7FCFEB5
:1086C00000F010FA00BFD3E7450600204606002060
:1086D000580600204A0600204906002070B50026F2
:1086E00000F072F8F7F7E4FE064631480068401CD7
:1086F0002F4908603046F7F7DFFE2E480078012842
:1087000053D12D48007820B1012804D0022809D186
:1087100003E001250BE0002509E0012501202649A1
:10872000087004E0012500202349087000BF00BF45
:1087300005B970BD2148046833E0F7F7B9FE064675
:10874000E06A50B3E06A401EE062E06A28BB94F839
:10875000300000F0370040B114F8300F00F0C800CE
:10876000207001206070303C02E0002084F831006D
:1087700094F8300000F0080078B93434A07810493B
:10878000097808430E49087020780E49085C617822
:10879000084314F834190B4A505464693046F7F70B
:1087A0008BFE94F832003F28C7D100BFC1E700001C
:1087B0007006002052060020680600206406002093
:1087C000490600204A0600207047704710B590F80F
:1087D000342001F10B039B5C90F83540A34301F179
:1087E0000B04A35423469B5C23B98B7A90F8364044
:1087F000A3438B7210BD00002DE9F04150211148B8
:1088000000F03EF900250DE0681C86B20D4800EB33
:10881000051400EB06170020207067600AA0E060D6
:10882000681C85B2042DEFD3064800EB0514002028
:108830002070606004A0E060024804490860BDE860
:10884000F08100009C5701203F000000340600200A
:1088500030B501464A6808682AB9CC68606028B11A
:108860000025456002E0106000B142608B68002581
:108870005D6230BD70B5C821114800F001F90023D8
:108880000FE0581C85B203EB83000D4901EB800417
:1088900005EB850001EB8006002020706660581C07
:1088A00083B2092BEDD303EB8300054901EB800470
:1088B00000202070606008460249086070BD00001A
:1088C000D45601203006002000200A4908600A49D9
:1088D00008700A4908700A4908700A4908700A496C
:1088E00008600A4908600A4908600A4908600A499C
:1088F00008707047700600204506002046060020DC
:1089000053060020520600202C06002054060020AA
:10891000400600203C0600204406002000210A4AB0
:108920001170002004E00021084A1154411CC8B213
:108930000828F8D30021064A1170064A1170064A29
:108940001160064A11607047490600204A0600205F
:108950004706002048060020600600205806002038
:1089600070B54FF47C71194800F08AF84FF48071AB
:10897000174800F085F8002413E0601CC5B2C4EB72
:10898000C40000EB4000114901EB8003C5EBC500BA
:1089900000EB400001EB80065E610EA0D864601C15
:1089A000C4B20B2CE9D3C4EBC40000EB4000074970
:1089B00001EB80030020586106A0D864002006491E
:1089C000086002480549086070BD0000EC5C0120A9
:1089D000EC5B01203F000000640600205C060020E4
:1089E00000B587B00320002180220A4BCDE9013277
:1089F000CDE903104FF6FF703F23074A0090074868
:108A0000FFF778FB06AA06A13F20FFF77DFC07B021
:108A100000BD0000EC590120E85B0120B98C010881
:108A200075432F4F532D49492049646C6500000060
:108A300000B587B00320002180220A4BCDE9013226
:108A4000CDE903104FF6FE703E23074A0090074819
:108A5000FFF750FB06AA06A13E20FFF755FC07B022
:108A600000BD0000EC570120E8590120F98C0108F5
:108A700075432F4F532D49492053746174000000F2
:108A800004E0002200F8012B4A1E91B20029F8D11F
:108A9000704700002DE9F04178211048FFF7F0FF02
:108AA00000240DE0601C86B204EB44000B4901EB8E
:108AB000C00506EB460001EBC0072F60601C84B2C6
:108AC000042CEFD304EB4400044901EBC005002063
:108AD0002860084602490860BDE8F081DC6001209A
:108AE0006C06002010B50024F7F7E2FC044613489A
:108AF0000078F8B912480078E0B900F02DF8114874
:108B00001149097850F82100104908600E48007892
:108B10000F49097888420DD00C480068806B401CD2
:108B20000A49096888630B480068401C09490860C5
:108B3000F7F7D7FC2046F7F7BFFC10BD450600202D
:108B400046060020EC5B012048060020600600205D
:108B5000470600202C0600200649074A1278885C48
:108B60000649095C034A515C01EBC001044A1170DB
:108B700070470000EEFF0108490600204A06002069
:108B8000480600202DE9F84F05460F4690469946C5
:108B9000DDE90AAB00200090F7F78AFC00903F481F
:108BA0000468002C74D0183454F8040C3B49086055
:108BB0000098F7F781FC44F8187CA5760020207611
:108BC0006076606144F814BC44F80CAC44F8108C36
:108BD0000C9824F8080C24F8069C0020E077E81094
:108BE000207705F00700E076217F01208840A077FC
:108BF000E17E01208840607700206060E060A06036
:108C00002062A0626062E062206325A06063183C7D
:108C1000002606E0002104F1500040F82610701CE8
:108C2000C6B2002EF6D02046FFF712FA2046FFF714
:108C3000BDFAF7F73DFC00901A4840F825401A4865
:108C4000006860610020A0611748006810B11648F4
:108C500000688461144804603434A07813490978AA
:108C600008431249087020781149085C617808436C
:108C700014F834190E4A50540E480078401C0D491F
:108C800008700098F7F718FC0020BDE8F88FFFE7A0
:108C90000098F7F711FC4220F7E700005C0600207F
:108CA0003F000000EC5B0120640600204906002024
:108CB0004A06002053060020002400BF00BFF7F73B
:108CC000F7FB044605480068401C0449086020463C
:108CD000F7F7F2FBFFF717FBF1E70000540600205F
:108CE00010B504480068FFF747FBFF20FFF760FA64
:108CF00010BD000058060020002400BF02E0142030
:108D0000FFF7B0FC194800780028F8D01848006830
:108D10006421B0FBF1F0164908600846006828B9E4
:108D2000002014490870FF20FFF746FC00BFF7F74A
:108D3000BFFB0446104800681049086000200E4937
:108D400008602046F7F7B8FB0C4800680849096836
:108D5000B0FBF1F0C0F1640006490870FFF70DFBAD
:108D600000F00EF80A20FFF77DFCE0E74406002043
:108D70003C06002038060020540600204006002053
:108D80007CB5002514E069462846FFF7F7FA064649
:108D900066B9094850F8254044B1012C06D0D4E901
:108DA000020100EB810060640198A064681CC5B2F8
:108DB0003F2DE8D97CBD0000EC5B012002F00103EF
:108DC00043B102F002032BB102E0491E002308C0A8
:108DD0000029FAD17047000010B50348007808B99F
:108DE00002F012FA10BD00004602002010B507483C
:108DF000008848B90648407B30B901200349088003
:108E000000210448FBF70CFE10BD0000020000200A
:108E1000EC080020C063012010B506480088012836
:108E200006D100210448FBF727FE002001490880F5
:108E300010BD000002000020C0630120014600BFF9
:108E4000080900EB8000420001F00F001044C0B29E
:108E5000704770B5044600252068C06800F04000E7
:108E6000A0B9681E2168C860FAF750FA054607E005
:108E7000FAF74CFA401BB0F57A7F01D9032070BD98
:108E80002068C06800F040000028F1D00020F6E71C
:108E900010B5002204490548FAF788FF002204496A
:108EA0000248FAF75DFF10BDCC610120AC610120E2
:108EB0008006002070B50546AC6B2068406820F045
:108EC000030021684860606D40F01000606501207B
:108ED00084F851002046FBF72EF870BD10B5044809
:108EE000008840F0200002490880F8F747FF10BDD5
:108EF0008E06002030B58DB00446182107A8F7F77C
:108F000021FC182101A8F7F71DFC002503208DF88E
:108F10001C000A208DF81D0001208DF81E0011484C
:108F200000788DF81F00104800788DF820000F4859
:108F300000788DF821000E4800788DF822000D4849
:108F400000788DF82300022301AA082107A80094C5
:108F5000FEF7B8FD0546294601A8F8F711FD0DB04A
:108F600030BD000078060020750600207406002041
:108F700077060020760600203949488A00EBD07138
:108F8000491000EE101AB8EEC00A3549497D00EECE
:108F9000901AB8EE601A3249498A00EE901AF8EE3B
:108FA000600A01EE200ADFED2F0A80EE201A2C491C
:108FB00081ED071A488A00EBD071491000EE101AB3
:108FC000B8EEC00A2649897D00EE901AB8EE601A04
:108FD0002349498A00EE901AF8EE600A01EE200A51
:108FE000DFED200A80EE201A1D4981ED081A08469F
:108FF000008B00EE100AB8EE400ADFED1A0A80EE90
:10900000201A084680ED091A007D012806D00228A2
:1090100005D003280BD004281FD116E01EE010480D
:1090200090ED070AB1EE400A80ED070A16E00C4801
:1090300090ED070AB1EE400A80ED070A90ED080AAC
:10904000B1EE400A80ED080A08E0054890ED080AF4
:10905000B1EE400A80ED080A00E000BF00BF704793
:10906000ECE7002000007A4400B593B0FE4890ED94
:109070000A0AB5EEC00AF1EE10FA54DD806A0F90CC
:1090800006F03AFF9FEDF90B53EC102BCDE91001E0
:109090009DED100B51EC100B06F0FCFB04D29FED84
:1090A000F50AF14880ED0A0AEF4890ED0B0AB5EE9B
:1090B000C00AF1EE10FA1ADDC06A0F9006F01CFF2C
:1090C0009FEDEA0B53EC102BCDE910019DED100B39
:1090D00051EC100B06F0DEFB04D29FEDE60AE248ED
:1090E00080ED0B0A0120E04981F8340070E0DE4891
:1090F000C06A0F9006F000FF9FEDDF0B53EC102BC2
:10910000CDE910019DED100B51EC100B06F0FCFCAD
:1091100004D29FEDDB0AD44880ED0B0A0420D2492B
:1091200081F8340054E0D048806A0F9006F0E4FEE5
:109130009FEDD10B53EC102BCDE910019DED100BE1
:1091400051EC100B06F0E0FC04D29FEDCD0AC648AE
:1091500080ED0A0AC44890ED0B0AB5EEC00AF1EEA4
:1091600010FA1ADDC06A0F9006F0C6FE9FEDBF0B25
:1091700053EC102BCDE910019DED100B51EC100BB1
:1091800006F088FB04D29FEDBB0AB74880ED0B0ABE
:109190000220B54981F834001AE0B348C06A0F9044
:1091A00006F0AAFE9FEDB40B53EC102BCDE9100195
:1091B0009DED100B51EC100B06F0A6FC04D29FEDB8
:1091C000B00AA94880ED0B0A0320A74981F83400B2
:1091D000A54890F83400012806D002287ED0032844
:1091E0007DD004287CD10DE39F4890ED0A0A20EE43
:1091F000000AD0ED0B0A90ED0B1A00EE810AA1488F
:10920000D0ED000A90ED001A00EEC10A8DED070ABC
:10921000079806F071FECDE908019DED080B05F0F9
:109220006BF98DED0C0B904890ED0C0A9648D0ED43
:10923000000A30EE600A8DED090A099806F05CFE1E
:10924000CDE90A019DED0C0B53EC102B9DED0A0BA3
:1092500051EC100B06F06CF9CDE90E019DED0E0BF3
:1092600004F016FF8DED100B9DED100B51EC100B63
:1092700006F078F87C498863084690ED0A0A20EEEB
:10928000000AD0ED0B0A90ED0B1A00EE810A8DED6D
:10929000030A039806F030FECDE904019DED040BAE
:1092A00005F02AF98DED080B7648006806F024FEDB
:1092B000CDE906019DED080B53EC102B9DED060B3F
:1092C00051EC100B06F034F9CDE90A019DED0A0BC3
:1092D00004F032FD8DED0E0B634802E079E0A0E171
:1092E0008AE3D0ED0B0A90ED0A1A80EE810A8DED2B
:1092F000070A079806F000FECDE908019DED080B6E
:1093000004F0C6FE8DED0A0B9FED600B53EC102BA5
:109310009DED0A0B51EC100B06F056F8CDE90C014F
:109320009DED0E0B53EC102B9DED0C0B51EC100B27
:1093300006F0F8FCCDE910019DED100B51EC100B7F
:1093400006F010F84849C863084690ED0E0ADFEDB4
:10935000510A20EE200A8DED0D0A0D9806F0CCFD85
:109360009FED4D0B53EC102BCDE90E019DED0E0B37
:1093700051EC100B06F0DCF8CDE910019DED100B5F
:1093800051EC100B05F0EEFF37498863084690ED6D
:109390000F0ADFED400A20EE200A8DED0D0A0D9830
:1093A00006F0AAFD9FED3C0B53EC102BCDE90E010E
:1093B0009DED0E0B51EC100B06F0BAF8CDE9100143
:1093C0009DED100B51EC100B05F0CCFF2649C86346
:1093D0001CE3254890ED0A0A20EE000AD0ED0B0AA6
:1093E00090ED0B1A00EE810A2648D0ED000A90EDB0
:1093F000001A00EEC10A8DED050A059806F07CFD05
:10940000CDE906019DED060B05F076F88DED0A0B12
:10941000154890ED0C0A1C48D0ED000A30EE600AA9
:109420008DED070A079806F067FDCDE908019DED6F
:109430000A0B53EC102B9DED080B51EC100B06F0B2
:1094400077F8CDE90C019DED0C0B04F021FE8DEDBC
:109450000E0B9FED110B53EC102B9DED0E0B51ECF1
:10946000100B06F087FB1BE0ECE700207B14AE47F7
:10947000E17A843F0AD7233C7B14AE47E17A84BF6C
:109480000AD723BCCC050020D0050020F1D4C85356
:10949000FB21F93F00003443F1D4C853FB210940BC
:1094A000CDE910019DED100B51EC100B05F05AFFAA
:1094B000FE498863084690ED0A0A20EE000AD0EDC6
:1094C0000B0A90ED0B1A00EE810A8DED010A01984E
:1094D00006F012FDCDE902019DED020B05F00CF83E
:1094E0008DED060BF248006806F006FDCDE904019B
:1094F0009DED060B53EC102B9DED040B51EC100B66
:1095000006F016F8CDE908019DED080B04F014FCF7
:109510008DED0C0BE54890ED0B0AF1EE400A90ED55
:109520000A1A80EE810A8DED050A059806F0E4FC22
:10953000CDE906019DED060B04F0AAFD8DED080BAB
:109540001FED2E0B53EC102B9DED080B51EC100B67
:1095500005F03AFFCDE90A019DED0C0B53EC102B01
:109560009DED0A0B51EC100B06F0DCFB9FEDD10BCF
:1095700053EC102BCDE90E019DED0E0B51EC100BB1
:1095800006F0F8FACDE910019DED100B51EC100B2F
:1095900005F0E8FEC549C863084690ED0E0A5FED88
:1095A000430A20EE200A8DED0D0A0D9806F0A4FC6A
:1095B0001FED470B53EC102BCDE90E019DED0E0B6B
:1095C00051EC100B05F0B4FFCDE910019DED100B2F
:1095D00051EC100B05F0C6FEB4498863084690EDC7
:1095E0000F0A5FED540A20EE200A8DED0D0A0D984A
:1095F00006F082FC1FED580B53EC102BCDE90E0149
:109600009DED0E0B51EC100B05F092FFCDE9100112
:109610009DED100B51EC100B05F0A4FEA349C8639F
:10962000F4E1A24890ED0A0A20EE000AD0ED0B0A00
:1096300090ED0B1A00EE810A9D48D0ED000A90EDE6
:10964000001A00EEC10A8DED050A059806F054FCDB
:10965000CDE906019DED060B04F04EFF8DED0A0BE2
:10966000924890ED0C0A9548D0ED000A30EE600A61
:109670008DED070A079806F03FFCCDE908019DED46
:109680000A0B53EC102B9DED080B51EC100B05F061
:109690004FFFCDE90C019DED0C0B04F0F9FC8DEDB5
:1096A0000E0B1FED830B53EC102B9DED0E0B51ECAD
:1096B000100B06F05FFACDE910019DED100B51EC97
:1096C000100B05F04FFE794988630846D0ED0A0A71
:1096D00090ED0B1A80EE810A8DED090A099806F0CB
:1096E0000BFCCDE90A019DED0A0B04F0D1FC8DEDD8
:1096F0000E0B6E4890ED0A0A20EE000AD0ED0B0A20
:1097000090ED0B1A00EE810A8DED030A039806F026
:10971000F3FBCDE904019DED040B04F0EDFE8DEDAE
:10972000080B6348006806F0E7FBCDE906019DEDF4
:10973000080B53EC102B9DED060B51EC100B05F0B4
:10974000F7FECDE90A019DED0A0B04F0F5FA8DED67
:109750000C0B9DED0E0B53EC102B9DED0C0B51ECF7
:10976000100B06F0DFFACDE910019DED100B51EC66
:10977000100B05F0F7FD4D49C863084690ED0E0A41
:109780005FEDBC0A20EE200A8DED0D0A0D9806F063
:10979000B3FB1FEDBF0B53EC102BCDE90E019DED7C
:1097A0000E0B51EC100B05F0C3FECDE910019DED41
:1097B000100B51EC100B05F0D5FD3C4988630846B1
:1097C00090ED0F0A5FEDCD0A20EE200A8DED0D0A17
:1097D0000D9806F091FB1FEDD00B53EC102BCDE94B
:1097E0000E019DED0E0B51EC100B05F0A1FECDE925
:1097F00010019DED100B51EC100B05F0B3FD2B4942
:10980000C86303E1294890ED0A0A20EE000AD0ED72
:109810000B0A90ED0B1A00EE810A2548D0ED000AE4
:1098200090ED001A00EEC10A8DED070A079806F0C8
:1098300063FBCDE908019DED080B04F05DFE8DEDA5
:109840000C0B1A4890ED0C0A1C48D0ED000A30EEC3
:10985000600A8DED090A099806F04EFBCDE90A0170
:109860009DED0C0B53EC102B9DED0A0B51EC100BE6
:1098700005F05EFECDE90E019DED0E0B04F008FC37
:109880008DED100B9DED100B51EC100B05F06AFDEA
:1098900006498863084690ED0A0AF1EE400A90ED09
:1098A0000B1A80EE810A8DED070A09E0ECE7002033
:1098B000CC0500200000000000000000D0050020C2
:1098C000079806F019FBCDE908019DED080B04F09F
:1098D000DFFB8DED0C0B574890ED0A0A20EE000AD5
:1098E000D0ED0B0A90ED0B1A00EE810A8DED010A06
:1098F000019806F001FBCDE902019DED020B04F099
:10990000FBFD8DED060B4C48006806F0F5FACDE93D
:1099100004019DED060B53EC102B9DED040B51EC57
:10992000100B05F005FECDE908019DED080B04F0D4
:1099300003FA8DED0A0B9DED0C0B53EC102B9DEDF6
:109940000A0B51EC100B06F0EDF9CDE90E019DED7F
:109950000E0B51EC100B05F0F9FCCDE910019DED5B
:10996000100B51EC100B05F0FDFC3249C8630846A2
:1099700090ED0E0ADFED310A20EE200A8DED0D0A82
:109980000D9806F0B9FA9FED2E0B53EC102BCDE994
:109990000E019DED0E0B51EC100B05F0C9FDCDE94C
:1099A00010019DED100B51EC100B05F0DBFC214973
:1099B0008863084690ED0F0ADFED200A20EE200AAA
:1099C0008DED0D0A0D9806F097FA9FED1D0B53ECE7
:1099D000102BCDE90E019DED0E0B51EC100B05F097
:1099E000A7FDCDE910019DED100B51EC100B05F01A
:1099F000B9FC1049C86309E09FED130A0D4880EDDA
:109A00000E0A9FED110A80ED0F0A00BF00BF0F483C
:109A1000008800EE100AB8EE400ADFED0D0A80EE75
:109A2000201A044890ED0E0A31EE000A80ED0E0A6D
:109A300013B000BDECE70020CC050020000034434B
:109A4000F1D4C853FB21094000000000D4050020D8
:109A50000000C84200B52DED028B85B000200490B7
:109A6000FD4890ED0E0AB5EEC00AF1EE10FA10DDD9
:109A700090ED0E0ADFEDF90A20EE200ABCEEC00AD6
:109A800010EE100AF449A1F84200012081F84000CC
:109A900014E0F14890ED0E0ADFEDF10A30EEC00A55
:109AA000DFEDEE0A20EE200ABCEEC00A10EE100A2E
:109AB000E949A1F84200022081F84000E64890ED13
:109AC0000F0AB5EEC00AF1EE10FA10DD90ED0F0AA4
:109AD000DFEDE20A20EE200ABCEEC00A10EE100A0A
:109AE000DD49A1F84400012081F8410014E0DA4882
:109AF00090ED0F0ADFEDDA0A30EEC00ADFEDD70A8B
:109B000020EE200ABCEEC00A10EE100AD249A1F8DD
:109B10004400022081F841000120D2490870D24956
:109B20000870D2480088401CD0490880CA48C07BD1
:109B3000012803D10020CE49087002E00120CC4961
:109B40000870C548B0F84400C34991F84110C64AAE
:109B500012780123CDE90032CDE90210BE48B0F8F9
:109B6000423090F84020BF480178012001F0B4FE57
:109B700001281CD1BF480078401CBE490870084627
:109B800000780A280EDD002008700220BA4908700B
:109B9000BA4908758DF81000022204A94FF4AA40B2
:109BA00001F060F9012005B0BDEC028B00BD002082
:109BB000B0490870AB480078012808D1B04890ED52
:109BC000000AA54880ED120A002088720DE0A9481D
:109BD000807A401CA74988720846807A052802DDF1
:109BE0000220A54908700120DDE79F480078012880
:109BF00009D1A44890ED000A974880ED130A00208F
:109C00009C49C8720DE09B48C07A401C9949C872B3
:109C10000846C07A052802DD022097490870012015
:109C2000C1E78D4890ED0E0AD0ED120A30EE600AC1
:109C300080ED160A90ED160AB5EEC00AF1EE10FAA4
:109C400007D290ED160ADFED860A30EEC00A80EDED
:109C5000160A814890ED0F0AD0ED130A30EE600A23
:109C600080ED170A90ED170AB5EEC00AF1EE10FA72
:109C700007D290ED170ADFED7A0A30EEC00A80EDC8
:109C8000170A754890ED160A10EE101A084606F0ED
:109C900033F941EC180B9FED7C0B53EC102B05F0C6
:109CA000F9FD0FD26C4890ED170A10EE101A084615
:109CB00006F022F941EC180B9FED730B53EC102BBF
:109CC00005F0E8FD7248008800EE100AB8EE400A80
:109CD000DFED620A80EE201A5F4890ED120A30EE46
:109CE000410A80ED120A90ED120ADFED6A0AB4EE25
:109CF000E00AF1EE10FA55D290ED130AB5EEC00A63
:109D0000F1EE10FA24DD0120534981F8340081F886
:109D10005000084690ED120ADFED500A20EE200AAE
:109D2000BCEEC00A10EE100AA1F85200012081F822
:109D30005100084690ED130ADFED480A20EE200A94
:109D4000BCEEC00A10EE100A80B2A1F8540080E008
:109D50000420414981F83400012081F85000084670
:109D600090ED120ADFED3D0A20EE200ABCEEC00A9B
:109D700010EE100AA1F85200022081F851000846A6
:109D800090ED130ADFED360A30EEC00ADFED330A3C
:109D900020EE200ABCEEC00A10EE100A80B2A1F834
:109DA000540056E02C4890ED130AB5EEC00AF1EECF
:109DB00010FA25DD0320284981F83400012081F8BC
:109DC0005000084690ED120ADFED240A20EE200A2A
:109DD000BCEEC00A10EE100AA1F85200012081F872
:109DE0005100084690ED130ADFED1C0A20EE200A10
:109DF000BCEEC00A10EE100A80B2A1F8540028E0B0
:109E00000220154981F83400012081F850000846ED
:109E100090ED120ADFED110A20EE200ABCEEC00A16
:109E200010EE100AA1F85200022081F851000846F5
:109E300090ED130ADFED0A0A30EEC00ADFED070AE3
:109E400020EE200ABCEEC00A10EE100A80B2A1F883
:109E5000540000BFA7E60000ECE700200000C84265
:109E600000000000900500209105002092050020D0
:109E7000DA0500200B090020BD050020EC080020B9
:109E8000880500208C050020000000000000E03F55
:109E9000D40500200000B44200B52DED108B87B032
:109EA00000200490059001F017FC012809D1D34847
:109EB000007A401CD1490872012007B0BDEC108B1C
:109EC00000BD0020CD490872CD4890ED130A10EE78
:109ED000101A084606F010F841EC1F0B9FEDC90B55
:109EE00053EC102B05F012FD41EC1E0B9FEDC70B40
:109EF00053EC102B05F01CFB41EC1D0BB0EE4D0A92
:109F0000F0EE6D0A04F030FAB0EE40BAF0EE60BA4E
:109F1000BB4890ED120A10EE101A084605F0ECFF4F
:109F20009FEDB80B53EC102BCDE900019DED000B1C
:109F300051EC100B05F0EAFC9FEDB40B53EC102B29
:109F4000CDE902019DED020B51EC100B05F0F0FA8A
:109F500041EC1F0BB0EE4F0AF0EE6F0A04F004FA6A
:109F6000B0EE40DAF0EE60DAAA4890ED000AAA48B6
:109F7000D0ED000A30EE200A10EE101A084605F067
:109F8000BBFF41EC1E0B53EC1D2B05F0BFFC41EC5D
:109F90001C0B53EC1B2B05F0B9FC41EC190B98483A
:109FA00090ED130A10EE101A084605F0A5FF41ECDB
:109FB0001F0B9FED940B53EC102B05F0A7FC41EC0D
:109FC0001E0B9FED920B53EC102B05F0B1FA41ECF8
:109FD0001D0BB0EE4D0AF0EE6D0A04F029FAB0EE5A
:109FE00040BAF0EE60BA8D48006805F085FF41EC9C
:109FF0001C0B53EC1B2B05F089FC41EC1A0B53ECAA
:10A00000192B05F0E1F941EC180B05F0ABF97C498F
:10A010008862084690ED130A10EE101A084605F003
:10A020006BFF41EC1D0B9FED770B53EC102B05F0F4
:10A030006DFC41EC1C0B9FED750B53EC102B05F0E8
:10A0400077FA41EC1B0BB0EE4B0AF0EE6B0A04F012
:10A05000EFF9B0EE409AF0EE609A694890ED120A7E
:10A0600010EE101A084605F047FF41EC1F0B9FED5C
:10A07000650B53EC102B05F049FC41EC1E0B9FEDDA
:10A08000630B53EC102B05F053FA41EC1D0BB0EEB3
:10A090004D0AF0EE6D0A04F067F9B0EE40BAF0EE4A
:10A0A00060BA5C4890ED000A5B48D0ED000A30EEE3
:10A0B000200A10EE101A084605F01EFF41EC1C0B9A
:10A0C00053EC1B2B05F022FC41EC1A0B53EC192B23
:10A0D00005F01CFC41EC180B494890ED130A10EEFA
:10A0E000101A084605F008FF41EC1D0B9FED450BCB
:10A0F00053EC102B05F00AFC41EC1C0B9FED430BBD
:10A1000053EC102B05F014FA41EC1B0BB0EE4B0A8C
:10A11000F0EE6B0A04F028F9B0EE409AF0EE609A87
:10A120003E4890ED000AB1EE400A10EE100A05F02C
:10A13000E3FE41EC1A0B53EC192B05F0E7FB53EC53
:10A14000182BCDE900019DED000B51EC100B05F033
:10A150003BF9CDE902019DED020B51EC100B05F02E
:10A1600001F92749C862084690ED120A10EE101A4C
:10A17000084605F0C1FE41EC1F0B9FED220B53EC8E
:10A18000102B05F0C3FB41EC1E0B9FED200B53EC95
:10A19000102B05F0CDF941EC1D0BB0EE4D0AF0EEA1
:10A1A0006D0A04F045F9B0EE40BAF0EE60BA194815
:10A1B00090ED000A1848D0ED000A30EE200A10EEAB
:10A1C000101A084605F098FE41EC1C0B53EC1B2BB3
:10A1D00005F09CFB41EC190B1148006805F08CFE62
:10A1E00041EC1A0B53EC192B05F0EEF841EC180B6F
:10A1F00005F0B8F80249086300BF5EE60B090020CD
:10A20000ECE70020F1D4C853FB2109400000000016
:10A210000080664054050020C8050020CC050020C1
:10A22000D005002000B52DED108B81B09FEDB60A52
:10A230008DED000AB54A02F10C01B548F6F780FE33
:10A24000B448008800EE100AB8EE400A10EE100A7A
:10A2500005F052FE41EC1F0B9FEDAF0B53EC102BA2
:10A2600005F054FB41EC1E0B9FEDAD0B53EC102B96
:10A2700005F05EF941EC1D0BB0EE4D0AF0EE6D0AF3
:10A2800004F07AF9B0EE40BAF0EE60BA9F481C389C
:10A2900090ED080A10EE101A084605F02DFE41EC6C
:10A2A0001C0B53EC1B2B05F031FB41EC190B9E48AA
:10A2B000008800EE100AB8EE400A10EE100A05F011
:10A2C0001BFE41EC1F0B9FED940B53EC102B05F084
:10A2D0001DFB41EC1E0B9FED920B53EC102B05F078
:10A2E00027F941EC1D0BB0EE4D0AF0EE6D0A04F0BB
:10A2F00043F9B0EE40BAF0EE60BA84481C3890EDF5
:10A30000070A10EE101A084605F0F6FD41EC1C0B8A
:10A3100053EC1B2B05F0FAFA41EC1A0B53EC192BFA
:10A3200005F052F841EC180B05F01CF80090774846
:10A330001C38D0ED090A9DED000A30EE800A80ED50
:10A34000090A90ED070AB5EEC00AF1EE10FA48DDF1
:10A3500090ED080AB5EEC00AF1EE10FA1FDD0120FB
:10A360006A491C3981F86000084690ED070ADFED64
:10A370006F0A20EE200ABCEEC00A10EE100AA1F807
:10A380006200084690ED080ADFED680A20EE200A18
:10A39000BCEEC00A10EE100AA1F864006FE00420C1
:10A3A0005A491C3981F86000084690ED070ADFED34
:10A3B0005F0A20EE200ABCEEC00A10EE100AA1F8D7
:10A3C0006200084690ED080AB1EE400ADFED570A38
:10A3D00020EE200ABCEEC00A10EE100AA1F86400BC
:10A3E0004DE04A481C3890ED080AB5EEC00AF1EE7F
:10A3F00010FA21DD022045491C3981F86000084629
:10A4000090ED070AB1EE400ADFED480A20EE200A7F
:10A41000BCEEC00A10EE100AA1F86200084690EDEA
:10A42000080ADFED420A20EE200ABCEEC00A10EE58
:10A43000100AA1F8640022E0032034491C3981F895
:10A440006000084690ED070AB1EE400ADFED370ADA
:10A4500020EE200ABCEEC00A10EE100AA1F862003D
:10A46000084690ED080AF1EE400A9FED300A20EE12
:10A47000800ABCEEC00A10EE100AA1F8640023485E
:10A480001C3890ED090A10EE101A084605F034FD4C
:10A4900041EC180B9FED260B53EC102B05F034FB11
:10A4A00026D21A481C38D0ED090A008900EE100A9D
:10A4B000B8EE400AF4EEC00AF1EE10FA07DD1348D8
:10A4C0001C38008911491C39A1F866001AE00F48B0
:10A4D0001C3890ED090ADFED180A20EE200ABCEEC8
:10A4E000C00A10EE100A09491C39A1F8660009E0FB
:10A4F000002006491C39A1F86600012001B0BDEC1E
:10A50000108B00BD0020F9E70000000008E80020E3
:10A5100060D90020D8050020F1D4C853FB210940A0
:10A52000000000000094D140D60500200000C84281
:10A530009A9999999999B93F00007A4470B504465F
:10A5400000250026F74890ED070AB5EEC00AF1EEA7
:10A5500010FA62DD90ED080AB5EEC00AF1EE10FACD
:10A560002CDD0120EF4981F86000084690ED070AD4
:10A57000DFEDED0A60EE200A408A00EE100AB8EE28
:10A58000400A80EE801ABCEEC10A10EE100A81F873
:10A590006800084690ED080ADFEDE30A60EE200A45
:10A5A000408A00EE100AB8EE400A80EE801ABCEE37
:10A5B000C10A10EE100A81F8690094E0D94890EDC4
:10A5C000070ADFEDD90A60EE200A408A00EE100A81
:10A5D000B8EE400A80EE801ABCEEC10A10EE100AF6
:10A5E000D04981F86800084690ED080AB1EE400AAB
:10A5F000DFEDCD0A60EE200A408A00EE100AB8EEC8
:10A60000400A80EE801ABCEEC10A10EE100A81F8F2
:10A610006900042081F8600065E0C24890ED080AF6
:10A62000B5EEC00AF1EE10FA2DDD90ED070AB1EE9D
:10A63000400ADFEDBD0A60EE200A408A00EE100AF3
:10A64000B8EE400A80EE801ABCEEC10A10EE100A85
:10A65000B44981F86800084690ED080ADFEDB20AB7
:10A6600060EE200A408A00EE100AB8EE400A80EE42
:10A67000801ABCEEC10A10EE100A81F869000220AF
:10A6800081F860002FE0A74890ED070AB1EE400A7C
:10A69000DFEDA50A60EE200A408A00EE100AB8EE4F
:10A6A000400A80EE801ABCEEC10A10EE100A9D49E5
:10A6B00081F86800084690ED080AB1EE400ADFED27
:10A6C0009A0A60EE200A408A00EE100AB8EE400AAC
:10A6D00080EE801ABCEEC10A10EE100A81F8690003
:10A6E000032081F860008F4890F8680004EB840133
:10A6F0008E4A02EB41014979884209DC894890F889
:10A70000690004EB840102EB4101C97988420ADD4A
:10A7100000208449088381F86A000846807D401C37
:10A720008875012070BD7F4890F860007D49097DE3
:10A73000884273D17B4890F8680000EB80007C4928
:10A7400001EB4010774991F8691000EB81008078A7
:10A75000002874D17348B0F86600724991F8681007
:10A7600001EB8101724A02EB41116E4A92F86920B5
:10A7700021F8220001206B4991F8681001EB81015A
:10A780006B4A02EB4111674A92F8692001EB8201A2
:10A790008870644B93F8692093F8681093F8600010
:10A7A000F6F746FA5F4890F86000012806D00228C4
:10A7B00013D0032821D0042842D130E0594890F822
:10A7C00068005849897A0844C5B2564890F869002B
:10A7D0005449C97A0844C6B233E05248807A514994
:10A7E00091F86810401A401EC5B24E4890F86900B2
:10A7F0004C49C97A0844C6B223E04A48807A49499C
:10A8000091F86810401A401EC5B24648C07A4549C2
:10A8100091F86910401A401EC6B212E0B2E04148F9
:10A8200090F868003F49897A0844C5B23D48C07A2B
:10A830003C4991F86910401A401EC6B201E058E048
:10A8400000BF00BF31462846F7F7E8FC354890F8CE
:10A8500068003449497D884217D1324890F8690030
:10A860003049897D884210D100202E49088381F823
:10A870006A0030480078012801D101F05DF92948CB
:10A88000807D401C2749887587E02648C07B0128C9
:10A8900010D100202349088381F86A0025480078F8
:10A8A000012801D101F048F91E48807D401C1D4956
:10A8B000887572E01B48B0F866001A49088308469C
:10A8C00090F86A00401C81F86A001A480078012854
:10A8D00001D101F031F9134890F86A0003285CDDDA
:10A8E0000020104981F86A000846807D401C887568
:10A8F00053E00C4890F868000A49497D88421BD112
:10A90000084890F869000749897D884214D10020E1
:10A910000449088381F86A000846807D401C8875D8
:10A920003BE00000ECE7002000007A44A8D90020BA
:10A9300058E80020C30500201948C07B012809D130
:10A9400000201749088381F86A000846807D401C72
:10A95000887522E01248B0F866001149088308465D
:10A9600090F86A00401C81F86A00084690F86A0076
:10A97000032812DD002081F86A000846807D401C13
:10A9800088750AE000200649088381F86A000846B5
:10A99000807D401C88750120C4E60020C2E60000CE
:10A9A000ECE7002010B50C480088401C0A490880DC
:10A9B0000A480088401C0949088009480088401C52
:10A9C00007490880F5F764FFFDF7C4FAFDF786FE36
:10A9D000FDF7D2FA10BD00004A0200205602002006
:10A9E0005802002000B597B030210BA8F5F7AAFE59
:10A9F000142106A8F5F7A6FE00200290039004900B
:10AA0000059000BF01902B48006840F08050294914
:10AA100008600846006800F08050019000BF00BF49
:10AA200000BF002001902448006840F48040224983
:10AA300008600846006800F48040019000BF00BF35
:10AA400009200B904FF480300C90012010900220D0
:10AA5000119041051291082113914FF4A87114919E
:10AA600002211591042116910BA8F8F755FF08B1A2
:10AA7000F6F7D0FD0F2006900220079000200890E6
:10AA80004FF4A05009904FF480500A90052106A879
:10AA9000F8F704FE08B1F6F7BDFD022002900002AF
:10AAA000059002A8F8F72AFD08B1F6F7B3FD17B034
:10AAB00000BD0000403802400070004013480068AC
:10AAC00040F47000114908601148006840F001002E
:10AAD0000F49086000200E49083108600C480068E2
:10AAE0000C4908400A4908600B48091D0860081F06
:10AAF000006820F48020091F0860002004490C3100
:10AB000008600648014980390860704788ED00E018
:10AB100000380240FFFFF6FE10300024000201085A
:10AB200000B585B014216846F5F70CFEB548007BEA
:10AB3000002846D1B448006840F6753188421AD9D9
:10AB4000B2480088401CB14908800020B049088004
:10AB5000AE4800880A280DDD0020AC49088001209D
:10AB6000A84908738DF800000B2269464FF49A40FB
:10AB700000F078F990E0A4480068B0F5A96F1AD801
:10AB8000A3480088401CA249088000209F490880F3
:10AB90009F4800880A287FDD00209D490880022008
:10ABA000984908738DF800000B2269464FF49A40CB
:10ABB00000F058F970E0002094490880944908801A
:10ABC0006AE09048007B012803D08E48007B032870
:10ABD0002DD18D48006840F60431884212D28C484D
:10ABE0000088401C8A4908800020884908808848DD
:10ABF0000088B0F5FA7F4FDD002085490880814943
:10AC0000087349E081480088401C80490880002082
:10AC10007F4908807D480088C8283DDD00207B49A9
:10AC2000088003207749087302F0A2FB34E07548DE
:10AC3000007B022803D07348007B04282CD1724883
:10AC4000006840F29C61884212D970480088401C1C
:10AC50006E49088000206E4908806C480088B0F575
:10AC6000FA7F19DD0020694908806649087313E0FE
:10AC700067480088401C66490880002063490880B6
:10AC800063480088C82807DD002061490880042047
:10AC90005C49087302F06CFB5A48807B38BB5D4806
:10ACA00000689B2824D95C480078401C5A490870E9
:10ACB0000846007832281EDD002008700120514926
:10ACC00088738DF8000053480088000A8DF8010051
:10ACD000504800788DF80200032269464FF49E40E8
:10ACE00000F0C0F8002240214C48F8F709FB02E0D0
:10ACF0000020494908704348407B20BB4848006811
:10AD00009B2821D947480078401C464908700846CE
:10AD1000007832281BDD0020087001203949487373
:10AD20008DF800003E480088000A8DF801003C487C
:10AD300000788DF80200032269464FF49C4000F031
:10AD400091F8FEF769F802E00020364908702D48B6
:10AD5000C07B20BB344800689B2821D93348007849
:10AD6000401C324908700846007832281BDD00205C
:10AD7000087001202349C8738DF800002A48008814
:10AD8000000A8DF80100284800788DF8020003229F
:10AD900069464FF4A04000F065F8FAF7B9FF02E009
:10ADA0000020224908701748007C20BB204800681A
:10ADB0009B2821D91F480078401C1E49087008466E
:10ADC000007832281BDD0020087001200D4908742E
:10ADD0008DF8000016480088000A8DF8010014481C
:10ADE00000788DF80200032269464FF4A24000F07B
:10ADF00039F8FBF72DF902E000200E49087005B084
:10AE000000BD0000EC080020080000201C0000200D
:10AE10001E00002014000020220000200008024034
:10AE20001000002021000020180000202300002036
:10AE30000C0000202000002010B515210648F5F771
:10AE40005FFC064800210160416001720448016016
:10AE50004160816010BD0000EC0800200209002064
:10AE60000B09002010B50323014C237010BD000016
:10AE70002400002010B50248F9F7E9FB10BD0000DE
:10AE8000FC63012010B50248F9F7E1FB10BD00009A
:10AE90008463012010B50248F9F7D9FB10BD00000A
:10AEA000C063012010B50248F9F7D1FB10BD0000C6
:10AEB0000C63012010B50248F9F7C9FB10BD000072
:10AEC00048630120002202682C4B98420ED0B0F15A
:10AED000804F0BD02A4B984208D02A4B984205D07D
:10AEE000294B984202D0294B984201D1012300E01E
:10AEF00000231BB122F070024B681A431F4B98428B
:10AF000020D0B0F1804F1DD01D4B98421AD01D4B60
:10AF1000984217D01C4B984214D01C4B984211D029
:10AF20001B4B98420ED01B4B98420BD01A4B9842A9
:10AF300008D01A4B984205D0194B984202D0194BB1
:10AF4000984201D1012300E000231BB122F440729A
:10AF5000CB681A4302608B68C3620B688362074B3D
:10AF6000984202D0094B984201D1012300E000230E
:10AF70000BB10B690363012343617047000001407B
:10AF80000004004000080040000C004000040140A4
:10AF900000400140004401400048014000180040CA
:10AFA000001C00400020004030B50023012404FABA
:10AFB00001F3046A9C430462046A02FA01F52C431B
:10AFC000046230BD30B50C460021816821F47F4118
:10AFD00042EA032525432943816030BD0A4600210A
:10AFE000816821F0700142F00703194381607047C6
:10AFF00030B5002400220023056A25F00105056212
:10B00000026A4368846924F0700424F003040D6824
:10B010002C4322F002028D682A430F4DA84202D031
:10B020000E4DA84201D1012500E000256DB122F0AE
:10B030000802CD682A4322F0040223F4807323F42B
:10B0400000734D692B438D692B43436084614D68C8
:10B050004563026230BD0000000001400004014071
:10B0600030B5002400220023056A25F01005056292
:10B07000026A4368846924F4E04424F440740D684F
:10B0800044EA052422F020028D6842EA0512104DA0
:10B09000A84202D00F4DA84201D1012500E00025B1
:10B0A00085B122F08002CD6842EA051222F040020A
:10B0B00023F4806323F400634D6943EA85038D69BB
:10B0C00043EA8503436084614D688563026230BD55
:10B0D000000001400004014030B50024002200239C
:10B0E000056A25F480750562026A4368C46924F024
:10B0F000700424F003040D682C4322F400728D6860
:10B1000042EA0522104DA84202D0104DA84201D1BA
:10B11000012500E0002585B122F40062CD6842EAF5
:10B12000052222F4806223F4805323F400534D69F6
:10B1300043EA05138D6943EA05134360C4614D6812
:10B14000C563026230BD0000000001400004014000
:10B1500030B5002200230024056A25F480550562DD
:10B16000036A4468C26922F4E04222F440720D6826
:10B1700042EA052223F400538D6843EA05330A4D61
:10B18000A84202D0094DA84201D1012500E00025C6
:10B1900025B124F480444D6944EA85144460C261B9
:10B1A0004D680564036230BD0000014000040140A9
:10B1B00030B50B46144600210022026A056A25F0CC
:10B1C00001050562816921F0F00141EA041122F0D4
:10B1D0000A021A438161026230BD30B50B46144643
:10B1E00000210022056A25F0100505628169026AC6
:10B1F00021F4704141EA043122F0A00242EA031234
:10B200008161026230BD000010B58EB0182108A81F
:10B21000F5F798FA182102A8F5F794FA002403200C
:10B220008DF820000A208DF8210001208DF82200E1
:10B23000094800788DF8230007480078032302AA04
:10B240000421009008A8FCF73DFC0446214602A812
:10B25000F6F796FB0EB010BD7806002070B50025FD
:10B26000002400BF4BE0FBF72BFE012800D144E097
:10B2700027480078012809D1264890ED000A264881
:10B2800080ED120A00202549887205E02348807A63
:10B29000401C2249887230E021480078012809D1F9
:10B2A000204890ED000A1C4880ED130A00201B493D
:10B2B000C87205E01948C07A401C1849C8721CE0E1
:10B2C0001948008800EE100AF8EE400A9FED171AA0
:10B2D00080EE810A1048D0ED120A30EEC00A80EDEF
:10B2E000120AFEF7D9FD012800D106E0FEF79AFF09
:10B2F000012800D101E0012400BF681CC5B2032D64
:10B30000B1DB012C01D100F0F9F9204670BD00003D
:10B310009005002088050020ECE700200B090020A4
:10B32000910500208C050020D40500200000C842B3
:10B330002DE9F0412DED048B82B0002000900190AA
:10B34000002500260027804609EE100A09EE900A23
:10B350009FED870AB0EE408A9FED850AF0EE408AA5
:10B360000024844840788349097800EB012080B2AA
:10B3700009EE100A7F48C0787E49897800EB0120E9
:10B3800080B209EE900A7B4840797A49097900EB4E
:10B39000012084B2F8EE490A7748008800EE100ACE
:10B3A000B8EE400A30EEC00ADFED740A80EE201AD3
:10B3B000B0EE418AF8EE690A7148008800EE100A82
:10B3C000B8EE400A30EEC00ADFED6C0A80EE201ABB
:10B3D000F0EE418A6B48007860B9FBF7A9FE0128BE
:10B3E00008D1002068490870012002B0BDEC048B30
:10B3F000BDE8F08165480088654908830025ABE019
:10B40000634880ED078AC0ED088A008B00EE100AC1
:10B41000B8EE400ADFED5F0A80EE201A5C4880ED4E
:10B42000091A00F1280200F11C015B48F5F788FDBC
:10B43000FDF71AFEFEF70EFB012800D18AE0FEF7A9
:10B440002BFD012800D185E0FEF7ECFE012804D198
:10B450004E4800884E4908837CE000274C4890ED18
:10B46000070AB4EEC80AF1EE10FA14DD014691EDB8
:10B47000070A30EE480ADFED470A20EE200ABCEE4C
:10B48000C00A10EE101A89B204EBD472B1EB620F4D
:10B4900015DA012713E03E4991ED070A38EE400A1C
:10B4A000DFED3C0A20EE200ABCEEC00A10EE101AB6
:10B4B00089B204EBD472B1EB620F00DA01274FF0CE
:10B4C0000008334890ED080AB4EEE80AF1EE10FAED
:10B4D00015DD014691ED080A30EE680ADFED2D0A10
:10B4E00020EE200ABCEEC00A10EE101A89B204EB5E
:10B4F000D472B1EB620F17DA4FF0010814E024495F
:10B5000091ED080A38EEC00ADFED220A20EE200A8B
:10B51000BCEEC00A10EE101A89B204EBD472B1EB83
:10B52000620F01DA4FF001080026012F04D1B8F1B3
:10B53000010F01D1012612E0154890ED090ADFED57
:10B54000150A20EE200ABCEEC00A10EE100A1049BF
:10B55000088300BF681CC5B2052DFFF651AF00BFC0
:10B56000012E03D100F064FA00203EE701203CE701
:10B5700000000000A83A01209A0500200000C842FF
:10B580009C050020BA050020BB0500209E05002078
:10B59000ECE7002000007A4484D9002010B52DED9E
:10B5A000048B02E00220FDF75DF840480078002897
:10B5B000F8D0FAF77BFDFAF75DFD3C4800780128EA
:10B5C00068D13B4890ED000A3A4880ED000A3848BF
:10B5D00090ED010A384880ED000A3648006804F012
:10B5E0008BFC41EC180B9FED350B53EC102B04F04A
:10B5F0008BFA11D22F48006804F07EFC41EC190B45
:10B600009FED300B53EC102B04F08CFB41EC180B2E
:10B6100003F0A8FE274908602748006804F06CFC86
:10B6200041EC180B9FED250B53EC102B04F06CFA3A
:10B6300012D22148006804F05FFC41EC190B9FED29
:10B64000210B53EC102B04F095FA41EC180B03F08E
:10B6500089FE1949086008E0174890ED000ADFEDFF
:10B660001B0A30EEC00A80ED000A1948008800EE7F
:10B67000100AF8EE400A9FED171A80EE810A0E4874
:10B68000D0ED000A30EEC00A80ED000A0020BDECCB
:10B69000048B10BD9FED0D0A064880ED000A9FED5A
:10B6A0000B0A054880ED000A0120F0E73C05002068
:10B6B000B80800207C050020800500200000000064
:10B6C000008066400000000000807640000000001E
:10B6D000D40500200000C84210B5002006490870BB
:10B6E000FAF728FBF9F7E8FF0348007808B90120CA
:10B6F00010BD0020FCE700005B050020F0B591B014
:10B70000202109A8F5F71EF8202101A8F5F71AF85D
:10B710000027002400250026354800788DF82400F5
:10B72000344800788DF8250003208DF82600062087
:10B730008DF8270001208DF828002F48008800EEA2
:10B74000100AB8EE400ADFED2D0A80EE201A2C48D0
:10B7500090ED070A31EE000ADFED280A20EE200AFC
:10B76000BCEEC00A10EE100A84B22648008800EE33
:10B77000100AB8EE400A9FED211AC0EE010A2048D7
:10B7800090ED080A30EE800ADFED1C0A20EE200A58
:10B79000BCEEC00A10EE100A85B2194890ED090AF5
:10B7A000DFED190A20EE200ABCEEC00A10EE100AE6
:10B7B00086B2200A8DF82900E0B28DF82A00280A06
:10B7C0008DF82B00E8B28DF82C00300A8DF82D0092
:10B7D000F0B28DF82E0001AA0B2109A8F6F71AFD88
:10B7E0000746394601A8F6F7CBF811B0F0BD0000C6
:10B7F0005B020020780600209A0500200000C84265
:10B80000ECE700209C05002000007A4470B590B061
:10B8100000240025202108A8F4F794FF2021684681
:10B82000F4F790FF0026002025490880254908806C
:10B830002549087005208DF82000244800788DF8EF
:10B84000210003208DF822000D208DF823001C48D4
:10B850000088000A8DF82400194800788DF825002A
:10B860006A46062108A8F6F7D5FC064600201849C6
:10B8700008701849087031466846F6F781F800BF2D
:10B8800000BF12E01E20FCF7EDFE601CC4B2142CB9
:10B890000BDD0024681CC5B2042D02DD012010B0B0
:10B8A00070BD31466846F6F76BF809480078002805
:10B8B000E8D0084800780028E4D00020EFE7000036
:10B8C0009205002078050020BC05002078060020A5
:10B8D00044020020450200202DE9F04F93B00546B8
:10B8E0000E4617461C46DDF870B0DDF87C8020213E
:10B8F0000BA8F4F727FF202103A8F4F723FF00206B
:10B900000290814682464149088041490870414879
:10B910000078401C3F49087003208DF82C0004205B
:10B920008DF82D008DF82E508DF82F608DF8307029
:10B93000200A8DF83100E0B28DF832008DF833B076
:10B940001D988DF834001E988DF835004FEA1820A8
:10B950008DF8360008F0FF008DF837002E4800788B
:10B960008DF838002D48008800128DF839002B48DA
:10B9700000788DF83A002A480078032303AA0F21A3
:10B9800000900BA8FCF79EF8029003A80299F5F727
:10B99000F7FF0020234908702349087000BF00BF4B
:10B9A00027E01E20FCF75EFE09F1010000F0FF0910
:10B9B000B9F1090F1DDD4FF000090AF1010000F097
:10B9C000FF0ABAF1050F10DD18480078401C17492E
:10B9D000087008460078032803DB00200870F5F79C
:10B9E0004BFF012013B0BDE8F08F03A80299F5F7D3
:10B9F000C7FF0C4800780028D3D00B4800780028F7
:10BA0000CFD000200949087000BFEBE7780500207F
:10BA1000BC05002002090020DA0500209205002064
:10BA2000780600204402002045020020F80500208E
:10BA3000F0B591B0202109A8F4F784FE202101A8D7
:10BA4000F4F780FE002700240025002602208DF850
:10BA50002400334800788DF8250003208DF8260057
:10BA600007208DF8270001208DF828002D48008838
:10BA700000EE100AB8EE400A9FED2B1AC0EE010A44
:10BA80002A4890ED070A30EE800ADFED270A20EE03
:10BA9000200ABCEEC00A10EE100A84B224480088C6
:10BAA00000EE100AB8EE400ADFED1F0A80EE201A01
:10BAB0001E4890ED080A31EE000ADFED1B0A20EE69
:10BAC000200ABCEEC00A10EE100A85B2174890EDAD
:10BAD000090ADFED180A20EE200ABCEEC00A10EEBB
:10BAE000100A86B2200A8DF82900E0B28DF82A00EB
:10BAF000280A8DF82B00E8B28DF82C00300A8DF85A
:10BB00002D00F0B28DF82E0001AA0B2109A8F6F73E
:10BB100081FB0746394601A8F5F732FF11B0F0BDA9
:10BB2000780600209A0500200000C842ECE70020BB
:10BB30009C05002000007A4430B593B024210AA867
:10BB4000F4F700FE242101A8F4F7FCFD00250024F1
:10BB5000504800788DF828004F4800788DF829006B
:10BB600003208DF82A000C208DF82B004B48007D17
:10BB70008DF82C004948407D8DF82D004748807D88
:10BB80008DF82E00454890F860008DF82F0043484E
:10BB900090F868008DF83000404890F869008DF802
:10BBA00031003E48B0F86200000A8DF832003B4890
:10BBB00090F862008DF833003848B0F86400000A4D
:10BBC0008DF83400354890F864008DF8350033481E
:10BBD000B0F86600000A8DF83600304890F866002C
:10BBE0008DF837002D48B0F85200000A8DF8380063
:10BBF0002A4890F852008DF839002848B0F85400CF
:10BC0000000A8DF83A00254890F854008DF83B0062
:10BC1000224890F850008DF83C00204890F85100E0
:10BC20008DF83D001E4800788DF83E001D480078D4
:10BC30008DF83F0002208DF8280001AA18210AA8DB
:10BC4000F6F7E8FA0546002017490870134890F8FF
:10BC5000600016490870114890F86800144908708F
:10BC60000E4890F869001349087003240BE0022C79
:10BC700004DD0024294601A8F5F782FE3220FCF7F6
:10BC8000F1FC601CC4B2084800780028EFD013B063
:10BC900030BD00005B02002078060020ECE70020A9
:10BCA0009005002091050020C4050020C505002056
:10BCB000C6050020C705002010B512E000200B4982
:10BCC00008700B480078012800D10BE00848007884
:10BCD000032803D1FBF706FC012010BD0A20FCF766
:10BCE000C1FCEBE700BF0020F7E70000BE05002025
:10BCF000BD050020F0B593B005460C4624210AA8E6
:10BD0000F4F720FD242101A8F4F71CFD00270026EC
:10BD1000FE48807AA8427DDDFC48C07AA0425FDD03
:10BD20000320FA49087581F860000846807A401EB1
:10BD3000401B81F868000846C07A401E001B81F84D
:10BD40006900488A00EBD071491000EE101AB8EE75
:10BD5000C00AEE4991F8681000EE901AB8EE601A29
:10BD6000EA49498A00EE901AF8EE600A01EE200ACC
:10BD7000F2EE040A80EE201ABCEEC10A10EE101A90
:10BD8000E24AA2F862101146488A00EBD0714910CD
:10BD900000EE101AB8EEC00A114691F8691000EED4
:10BDA000901AB8EE601A1146498A00EE901AF8EE21
:10BDB000600A01EE200AF2EE040A80EE201ABCEEC0
:10BDC000C10A10EE101AA2F86410C5EB0510D04994
:10BDD00001EB001030F824001146A1F8660020E1C4
:10BDE0000220CA49087581F860000846807A401E22
:10BDF000401B81F868000846C07A201A81F8690063
:10BE0000488A00EBD071491000EE101AB8EEC00A53
:10BE1000BE4900E045E091F8681000EE901AB8EED7
:10BE2000601ABA49498A00EE901AF8EE600A01EEEB
:10BE3000200AF2EE040A80EE201ABCEEC10A10EECF
:10BE4000101AB24AA2F862101146488A00EBD0716B
:10BE5000491000EE101AB8EEC00A114691F86910A8
:10BE600000EE901AB8EE601A1146498A00EE901A58
:10BE7000F8EE600A01EE200AF2EE040A80EE201AC3
:10BE8000BCEEC10A10EE101AA2F86410C5EB051042
:10BE90009F4901EB001030F824001146A1F866001C
:10BEA000BFE09A48C07AA0425EDD04209749087539
:10BEB00081F860000846807A281A81F868000846F0
:10BEC000C07A401E001B81F86900488A00EBD071DF
:10BED000491000EE101AB8EEC00A8C4991F86810AB
:10BEE00000EE901AB8EE601A8849498A00EE901A5E
:10BEF000F8EE600A01EE200AF2EE040A80EE201A43
:10BF0000BCEEC10A10EE101A804AA2F86210114667
:10BF1000488A00EBD071491000EE101AB8EEC00A42
:10BF2000114691F8691000EE901AB8EE601A1146A9
:10BF3000498A00EE901AF8EE600A01EE200AF2EE4D
:10BF4000040A80EE201ABCEEC10A10EE101AA2F804
:10BF50006410C5EB05106E4901EB001030F82400A9
:10BF60001146A1F866005CE001206849087581F877
:10BF700060000846807A281A81F868000846C07A6E
:10BF8000201A81F86900488A00EBD071491000EE50
:10BF9000101AB8EEC00A5D4991F8681000EE901AC8
:10BFA000B8EE601A5949498A00EE901AF8EE600A14
:10BFB00001EE200AF2EE040A80EE201ABCEEC10A5D
:10BFC00010EE101A514AA2F862101146488A00EB8E
:10BFD000D071491000EE101AB8EEC00A114691F85F
:10BFE000691000EE901AB8EE601A1146498A00EE08
:10BFF000901AF8EE600A01EE200AF2EE040A80EED2
:10C00000201ABCEEC10A10EE101AA2F86410C5EB9B
:10C0100005103F4901EB001030F824001146A1F84B
:10C0200066003C4800788DF828003B4800788DF881
:10C03000290003208DF82A000C208DF82B003348AE
:10C04000007D8DF82C00314890F868008DF82D00A7
:10C050002E4890F869008DF82E002C4890F860006A
:10C060008DF82F00294890F868008DF83000274897
:10C0700090F869008DF831002448B0F86200000A99
:10C080008DF83200214890F862008DF833001F4887
:10C09000B0F86400000A8DF834001C4890F8640081
:10C0A0008DF835001948B0F86600000A8DF83600A2
:10C0B000164890F866008DF837001448B0F8520022
:10C0C000000A8DF83800114890F852008DF83900B8
:10C0D0000E48B0F85400000A8DF83A000B4890F86A
:10C0E00054008DF83B00094890F850008DF83C0052
:10C0F000064890F851008DF83D00084800788DF80A
:10C100003E00074800788DF83F000BE0ECE7002088
:10C11000580101205B0200207806002090050020D5
:10C120009105002001AA18210AA8F6F773F807461E
:10C13000002012490870124890F8600011490870F8
:10C140000F4890F86800104908700D4890F8690091
:10C150000E49087003260BE0022E04DD0026394646
:10C1600001A8F5F70DFC3220FCF77CFA701CC6B272
:10C17000024800780028EFD013B0F0BDC4050020BD
:10C18000ECE70020C5050020C6050020C7050020FB
:10C190002DE9F04F2DED108B8FB000200C900D90FD
:10C1A0000E908246002600249FEDFE0AF0EE408AA3
:10C1B0009FEDFC0AB0EE40FA0B900A9000258046F5
:10C1C000834609909FEDF70AB0EE408A002781462A
:10C1D000F5484179C07B0844801CC7B2F248417CD5
:10C1E000C07E0844801C00F0FF0900BF1DE000264F
:10C1F00015E0CAEB0A10ED4901EB001000EB8600D8
:10C200008078012809D1CAEB0A1001EB001030F840
:10C210002600E7490989081A0444701C86B24E4575
:10C22000E7DB0AF101001FFA80FABA45DFDBDE48DE
:10C23000408800EE100AB8EE400A60EE000A00EEF8
:10C24000104AB8EE400A20EE800AF0EE408A18EE5E
:10C25000900A03F051FE41EC1A0B9FEDD60B53EC04
:10C26000102B03F065F941EC190B03F07BF808EE95
:10C27000900ACD484088CC494979491C48430A2155
:10C2800090FBF1F0CD490988CD4A1288891A081A25
:10C2900085B2C5484088C449C979491C48430A2128
:10C2A00090FBF1F0C7490988C74A1288891A081A11
:10C2B0001FFA80F8BC48C08ABB49497E491C4843E4
:10C2C0000A2190FBF1F0BE490988081A1FFA80FB89
:10C2D000B548C08AB449C979491C48430A2190FB32
:10C2E000F1F0B9490988081A80B2099000249FED3D
:10C2F000AD0AB0EE408A002D31DD002617E0781E31
:10C30000C0EB0010A94901EB001000EB860080781B
:10C3100001280AD1781EC0EB001001EB001030F8A4
:10C320002600A3490989081A0444701C86B24E45A8
:10C33000E5DB9D48408800EE100AF8EE400A00EE6A
:10C34000105AB8EE400A60EE800A00EE104AB8EECD
:10C35000401AB0EE480A00EE810AB0EE408A00248E
:10C36000B8F1000F31DD002617E0781EC0EB001099
:10C370008E4901EB001000EB8600807801280AD17D
:10C38000781EC0EB001001EB001030F82600884941
:10C390000989081A0444701C86B24E45E5DB8248C0
:10C3A000408800EE100AF8EE400A00EE105AB8EE8F
:10C3B000400A60EE800A00EE104AB8EE401AB0EE75
:10C3C000480A00EE810AB0EE408A0024BBF1000F5B
:10C3D00031DD002617E0781EC0EB0010734901EB39
:10C3E000001000EB8600807801280AD1781EC0EB8F
:10C3F000001001EB001030F826006D490989081A79
:10C400000444701C86B24E45E5DB6748408800EE68
:10C41000100AF8EE400A00EE105AB8EE400A60EE3C
:10C42000800A00EE104AB8EE401AB0EE480A00EE5C
:10C43000810AB0EE408A00240998002831DD0026E8
:10C4400017E0781EC0EB0010584901EB001000EB1C
:10C450008600807801280AD1781EC0EB001001EB1D
:10C46000001030F8260052490989081A0444701C4B
:10C4700086B24E45E5DB4C48408800EE100AF8EEE7
:10C48000400A00EE105AB8EE400A60EE800A00EE54
:10C49000104AB8EE401AB0EE480A00EE810AB0EE3B
:10C4A000408A002D18DDB8F1000F15DD3E484088A8
:10C4B00000EE100AF8EE400A00EE105AB8EE400AFC
:10C4C00060EE800A00EE104AB8EE401AB0EE480A5C
:10C4D00000EE810AB0EE408A002D18DDB8F1000FA1
:10C4E00015DD3148408800EE100AF8EE400A00EEF3
:10C4F000105AB8EE400A60EE800A00EE104AB8EE1C
:10C50000401AB0EE480A00EE810AB0EE408A002DD3
:10C5100018DDB8F1000F15DD2348408800EE100A41
:10C52000F8EE400A00EE105AB8EE400A60EE800ABB
:10C5300000EE104AB8EE401AB0EE480A00EE810A4A
:10C54000B0EE408A002D18DDB8F1000F15DD164859
:10C55000408800EE100AF8EE400A00EE105AB8EEDD
:10C56000400A60EE800A00EE104AB8EE401AB0EEC3
:10C57000480A00EE810AB0EE408A38EE880AF0EEF2
:10C58000408A1048008800EE100AF8EE400A0B4876
:10C59000008800EE100AB8EE400A60EE800A0448F7
:10C5A000008913E000000000A8D9002058010120F4
:10C5B000ECE7002000000000D01263419605002047
:10C5C0009A050020940500209C05002000EE100A2A
:10C5D000B8EE400A20EE800A10EE101A084603F06A
:10C5E0008BFC9FED430B53EC102BCDE900019DED2F
:10C5F000000B51EC100B02F09BFF41EC1E0B18EEF0
:10C60000900A03F079FC53EC1E2BCDE902019DED5D
:10C61000020B51EC100B02F08BFF41EC1C0B364867
:10C62000008800EE100AB8EE400A10EE100A03F07F
:10C6300063FC41EC1D0B53EC1C2B03F067F941EC40
:10C640001A0B18EE900A03F057FC41EC1B0B53EC4D
:10C650001A2B03F067FB41EC190B02F083FE08EE86
:10C66000900A2648008800EE100AB8EE400A38EE1C
:10C67000C00AF2EE040A80EE201AF0EE418ABCEE07
:10C68000E80A1F4880ED000A1E48008800EE100AE4
:10C69000B8EE400A28EE800AF2EE040A80EE201A74
:10C6A000B0EE41FA9FED180ACFEE000AB0EE60FA44
:10C6B000BCEECF0A154880ED000A15480088401CE2
:10C6C0001349088008460088ADF818000C48006837
:10C6D000CDF81A000D480068CDF81E000A22282166
:10C6E00006A8F5F791FC0FB0BDEC108BBDE8F08FFC
:10C6F00000000000006AF840AA050020AC050020F8
:10C70000B0050020A80500200000C842B4050020A4
:10C71000A405002010B50020304908804AE02F4AC7
:10C72000128802EB42022E4B03EB420291882B4A05
:10C73000128802EB420203EB4202508800F05EF8DE
:10C74000C0B9284800682549098801EB4101264AFB
:10C7500002EB4101C1F802002048008800EB4000D4
:10C760001F4931F810001D49098801EB410122F8E9
:10C77000110017E04FF0EE301849098801EB410134
:10C78000194A02EB4101C1F802001448008800EB8D
:10C790004000134931F810001049098801EB4101AC
:10C7A00022F811000A20FBF75DFF0C480088401CAE
:10C7B0000A490880094800880C4909888842AEDB8C
:10C7C0000A4800880A49088000200A490880074969
:10C7D0000880024908800849088010BD1E06002014
:10C7E000B23A0120E4050020C248012020060020C2
:10C7F0002606002024060020220600202DE9F04312
:10C800002DED068B85B005460E460024A046002778
:10C810000020EC490860EC490860EC490860EC49EC
:10C820000860EC4908608146B6F5FA7F08DB40F6FF
:10C83000C410864204DCB5F5FA7F01DB854205DDD4
:10C84000012005B0BDEC068BBDE8F083A5F5FA70BC
:10C8500002F0F5FF41EC1A0B9FEDDF0B53EC102BB0
:10C8600003F054F841EC190B9FEDDD0B53EC102B4A
:10C8700002F0AAFD41EC180B02F074FDDA4988635E
:10C88000A6F5FA7002F0DBFF41EC1A0B9FEDD20B1C
:10C8900053EC102B03F03AF841EC190B9FEDD30B3E
:10C8A00053EC102B02F090FD41EC180B02F05AFDF6
:10C8B000CD49C863084690ED0E0AB5EEC00AF1EE08
:10C8C00010FA0FDD90ED0E0ADFEDCA0A20EE200A05
:10C8D000BCEEC00A10EE100AA1F84200012081F857
:10C8E000400014E0C04890ED0E0ADFEDC30A30EEC0
:10C8F000C00ADFEDC00A20EE200ABCEEC00A10EE2E
:10C90000100AB949A1F84200022081F84000B64857
:10C9100090ED0F0AB5EEC00AF1EE10FA10DD90EDC1
:10C920000F0ADFEDB40A20EE200ABCEEC00A10EEBA
:10C93000100AAD49A1F84400012081F8410014E03B
:10C94000A94890ED0F0ADFEDAC0A30EEC00ADFED2A
:10C95000A90A20EE200ABCEEC00A10EE100AA24975
:10C96000A1F84400022081F841000120A349087089
:10C97000A3490870A3480088401CA24908800120F0
:10C98000A14908709848B0F84400974991F84110BF
:10C990009B4A12780123CDE90032CDE9021092487A
:10C9A000B0F8423090F84020944801780120FEF71A
:10C9B00093FF012800D144E790480078012806D170
:10C9C000924890ED000A884880ED120A01E00120AB
:10C9D00037E78B480078012806D18D4890ED000A92
:10C9E000814880ED130A01E001202AE70A20FBF7C5
:10C9F00039FE00275FE0FEF76FFE012800D120E737
:10CA00009CB9844890ED000A8348D0ED000A30EECE
:10CA1000200ADFED820A20EE200ABCEEC00A6A4836
:10CA200080ED000A601CC4B240E0012C13D17948AB
:10CA300090ED000A7848D0ED000A30EE200ADFEDD4
:10CA4000770A20EE200ABCEEC00A604880ED000A9A
:10CA5000601CC4B22AE0022C13D16E4890ED000A8B
:10CA60006D48D0ED000A30EE200ADFED6C0A20EEB2
:10CA7000200ABCEEC00A564880ED000A601CC4B211
:10CA800014E0032C12D1634890ED000A6248D0ED07
:10CA9000000A30EE200ADFED610A20EE200ABCEE2B
:10CAA000C00A4C4880ED000A601CC4B20320FBF7AA
:10CAB000D9FD781CC7B2022F9DDB042C4DD1434811
:10CAC000016841480068F4F707FAE0B94048016896
:10CAD0003D480068F4F700FA30B93B48006839492E
:10CAE00008604FF001085EE03A4801683648006887
:10CAF000F4F7F2F9002856D133480068314908604C
:10CB00004FF001084FE0324801682F480068F4F701
:10CB1000E3F968B92F4801682B480068F4F7DCF99D
:10CB200088BB29480068274908604FF001083AE0AF
:10CB30002748016825480068F4F7CEF918BB254856
:10CB4000016822480068F4F7C7F9E0B91F48006897
:10CB50001C4908604FF0010825E0032C14D11B4844
:10CB6000016819480068F4F7B7F960B91848016816
:10CB700015480068F4F7B0F928B91348006811495E
:10CB800008604FF001080EE0022C0CD10F4801683C
:10CB90000D480068F4F7A0F928B90B480068094966
:10CBA00008604FF00108B8F1000F01D1012048E6FC
:10CBB000044800681A49884201D9012041E6002052
:10CBC0003FE60000E4050020E8050020EC05002019
:10CBD000F0050020F405002048E17A14AE47C13F7B
:10CBE00000000000008046C0ECE7002000000000CC
:10CBF00000E060C00000C842000000009005002076
:10CC00009105002092050020DA050020880500200B
:10CC10008C05002054050020C805002000007A443F
:10CC20007011010030B52DED068B85B00025002474
:10CC30000020B1490860B1490860B1490860B149B4
:10CC40000860B1490860B1480088B0F5FA7F0EDB92
:10CC5000AE48008840F6C411884208DCAC48008821
:10CC6000B0F5FA7F03DBAA480088884204DD012082
:10CC700005B0BDEC068B30BDA5490988A1F5FA7059
:10CC800002F0DDFD41EC1A0B9FEDA20B53EC102BD3
:10CC900002F03CFE41EC190B9FEDA00B53EC102B66
:10CCA00002F092FB41EC180B02F05CFB9D4988639B
:10CCB00096490988A1F5FA7002F0C1FD41EC1A0B02
:10CCC0009FED940B53EC102B02F020FE41EC190B5E
:10CCD0009FED950B53EC102B02F076FB41EC180BFB
:10CCE00002F040FB8F49C863084690ED0E0AB5EE8E
:10CCF000C00AF1EE10FA0FDD90ED0E0ADFED8C0A9E
:10CD000020EE200ABCEEC00A10EE100AA1F8420084
:10CD1000012081F8400014E0824890ED0E0ADFED1A
:10CD2000850A30EEC00ADFED820A20EE200ABCEE52
:10CD3000C00A10EE100A7B49A1F84200022081F8D7
:10CD40004000784890ED0F0AB5EEC00AF1EE10FAF7
:10CD500010DD90ED0F0ADFED760A20EE200ABCEE22
:10CD6000C00A10EE100A6F49A1F84400012081F8B2
:10CD7000410014E06B4890ED0F0ADFED6E0A30EED3
:10CD8000C00ADFED6B0A20EE200ABCEEC00A10EEEE
:10CD9000100A6449A1F84400022081F841000120F2
:10CDA000654908706549087065480088401C6449F9
:10CDB00008800120634908705A48B0F84400594976
:10CDC00091F841105D4A12780123CDE90032CDE996
:10CDD00002105448B0F8423090F84020564801788C
:10CDE0000120FEF779FD012800D141E75248007883
:10CDF000012806D1544890ED000A4A4880ED120AF5
:10CE000001E0012034E74D480078012806D14F4861
:10CE100090ED000A434880ED130A01E0012027E766
:10CE20004B48007838B9FF2200214948007800F0CB
:10CE300069FE00201CE7FEF74FFC012801D1012507
:10CE400010E0444890ED000A4348D0ED000A30EE6F
:10CE5000200ADFED420A20EE200ABCEEC00A274875
:10CE600080ED000AFEF738FC012801D1012410E012
:10CE7000384890ED000A3848D0ED000A30EE200A1C
:10CE8000DFED360A20EE200ABCEEC00A1C4880ED19
:10CE9000000A05BBFCB9194800681949096808442B
:10CEA0004008154908601548006815490968884216
:10CEB00008D91248006812490968401A96280CD30C
:10CEC0000120D5E60E4800680C490968401A9628EA
:10CED00003D30120CCE60120CAE6074800682049B8
:10CEE000884201D90120C3E6FF22002118480078BA
:10CEF00000F008FE0020BBE6E4050020E805002065
:10CF0000EC050020F0050020F4050020DE050020DF
:10CF1000E005002048E17A14AE47C13F0000000060
:10CF2000008046C0ECE700200000000000E060C088
:10CF30000000C8420000000090050020910500207C
:10CF400092050020DA050020880500208C050020CD
:10CF5000DC05002054050020C805002000007A44AC
:10CF60007011010002460020704770B5064600258A
:10CF7000B46B20684069C0F3C01594F839002128CB
:10CF800005D125B10020E084204600F026F8206875
:10CF90004069C0F3801594F83A00222805D125B1E4
:10CFA0000020E085204600F008F8E06B40F010001B
:10CFB000E0632046F7F73CFE70BD0168C96821F4C4
:10CFC00090710268D1600168496921F0010102682D
:10CFD0005161202180F83A1070470168C96821F03A
:10CFE000C0010268D160202180F83910704700002C
:10CFF0002DE9F041044600252068056925F44055D7
:10D00000E0680543206805612068C56849F20C6046
:10D0100085432169A068084361690843E1690843C1
:10D0200005432068C5602068456925F44075A069FE
:10D03000054320684561E069B0F5004F7ED1C449E1
:10D040002068884203D0C349206888425DD1F6F742
:10D05000FBFB00EBC00101EB001061684900B0FB75
:10D06000F1F06421B0FBF1F00601F6F7EDFB00EB07
:10D07000C00101EB001061684900B0FBF1F7F6F761
:10D08000E3FB00EBC00101EB001061684900B0FB5D
:10D09000F1F06421B0FBF1F000EBC00101EB0010F6
:10D0A000A7EB8000322101EBC0006421B0FBF1F05E
:10D0B00000F0F80006EB4006F6F7C6FB00EBC001F7
:10D0C00001EB001061684900B0FBF1F7F6F7BCFB1B
:10D0D00000EBC00101EB001061684900B0FBF1F00A
:10D0E0006421B0FBF1F000EBC00101EB0010A7EBF5
:10D0F0008000322101EBC0006421B0FBF1F000F0B0
:10D10000070030442168886020E1F6F78DFB00EBD2
:10D11000C00101EB001061684900B0FBF1F064212F
:10D12000B0FBF1F00601F6F77FFB00EBC00101EB6D
:10D13000001061684900B0FBF1F700E045E0F6F748
:10D1400073FB00EBC00101EB001061684900B0FB0C
:10D15000F1F06421B0FBF1F000EBC00101EB001035
:10D16000A7EB8000322101EBC0006421B0FBF1F09D
:10D1700000F0F80006EB4006F6F756FB00EBC001A6
:10D1800001EB001061684900B0FBF1F7F6F74CFBCA
:10D1900000EBC00101EB001061684900B0FBF1F049
:10D1A0006421B0FBF1F000EBC00101EB0010A7EB34
:10D1B0008000322101EBC0006421B0FBF1F000F0EF
:10D1C0000700304421688860C0E0614920688842D7
:10D1D00003D06049206888425CD1F6F735FB00EB4C
:10D1E000C00101EB001061688900B0FBF1F6F6F7B1
:10D1F0002BFB00EBC00101EB001061688900B0FB64
:10D20000F1F06421B0FBF1F000EBC00101EB001084
:10D21000A6EB8000322101EB00106421B0FBF1F09D
:10D2200000F0F006F6F710FB00EBC00101EB001078
:10D2300061688900B0FBF1F06421B0FBF1F006EB0E
:10D240000016F6F701FB00EBC00101EB001061686E
:10D250008900B0FBF1F7F6F7F7FA00EBC00101EB3C
:10D26000001061688900B0FBF1F06421B0FBF1F0BF
:10D2700000EBC00101EB0010A7EB8000322101EBB5
:10D2800000106421B0FBF1F000F00F003044216881
:10D2900088605BE0F6F7C8FA00EBC00101EB001014
:10D2A00061688900B0FBF1F6F6F7BEFA00EBC00149
:10D2B00001EB001061688900B0FBF1F06421B0FB64
:10D2C000F1F000EBC00101EB0010A6EB8000322171
:10D2D00001EB00106421B0FBF1F000F0F006F6F76E
:10D2E000A3FA00EBC00101EB001061688900B0FBFC
:10D2F000F1F06421B0FBF1F006EB0016F6F794FABA
:10D3000000EBC00101EB001061688900B0FBF1F790
:10D31000F6F78AFA00EBC00101EB001061688900A2
:10D32000B0FBF1F06421B0FBF1F000EBC00101EBC8
:10D330000010A7EB8000322101EB00106421B0FB4C
:10D34000F1F000F00F00304421688860BDE8F08102
:10D35000001001400014014010B50448008840F05E
:10D36000100002490880F4F709FD10BD8E06002068
:10D3700010B5002240210548F5F7C2FFF8F768FE16
:10D38000F8F7C6FCFBF748FD10BD0000000802409E
:10D3900070B5C0B04FF480716846F3F7D3F900243C
:10D3A00000260025C248008800287DD1C148008899
:10D3B0000128FAD1C0480088C0490988884273DA38
:10D3C000B5222046611CCCB20DF800200122204677
:10D3D000611CCCB20DF8002003222046611CCCB2A7
:10D3E0000DF80020B6480068020E2046611CCCB241
:10D3F0000DF80020B2480068C0F307422046611CC7
:10D40000CCB20DF80020AE480088C0F307222046B9
:10D41000611CCCB20DF80020A94802782046611C9E
:10D42000CCB20DF80020A5480088A3490988401A0D
:10D4300086B2142E79DD00222046611CCCB20DF894
:10D44000002014222046611CCCB20DF8002000BF41
:10D4500067E0FF222046611CCCB20DF80020204678
:10D46000611CCCB20DF800209348008800EB40000E
:10D47000944901EB4000D0F80200020E2046611CE6
:10D48000CCB20DF800208C48008800EB40008D499C
:10D4900001EB4000D0F80200C0F307422046611CB7
:10D4A000CCB20DF8002000E0C9E08348008800EB12
:10D4B0004000844901EB40004088C0F30722204629
:10D4C000611CCCB20DF800207B48008800EB4000C6
:10D4D0007C4901EB400082782046611CCCB20DF8FB
:10D4E00000207548008800EB4000764931F81000B4
:10D4F00002122046611CCCB20DF800206E48008854
:10D5000000EB40006F4911F810202046611CCCB29E
:10D510000DF8002068480088401C67490880681C96
:10D52000C5B2142D95DB84E0FFE700222046611C84
:10D53000CCB20DF80020F2B22046611CCCB20DF83E
:10D540000020002565E0FF222046611CCCB20DF8CA
:10D5500000202046611CCCB20DF8002056480088FF
:10D5600000EB4000574901EB4000D0F80200020EEA
:10D570002046611CCCB20DF800204F48008800EB1B
:10D580004000504901EB4000D0F80200C0F30742D0
:10D590002046611CCCB20DF800204748008800EB03
:10D5A0004000484901EB40004088C0F30722204674
:10D5B000611CCCB20DF800203F48008800EB400011
:10D5C000404901EB400082782046611CCCB20DF846
:10D5D00000203948008800EB40003A4931F810003B
:10D5E00002122046611CCCB20DF80020324800889F
:10D5F00000EB4000334911F810202046611CCCB2EA
:10D600000DF800202C480088401C2B490880681C1D
:10D61000C5B2B54297DBFF222146601CC4B20DF8AB
:10D6200001202046611CCCB20DF8002000202249C8
:10D63000088021466846F4F7A3F940B070BD002485
:10D64000B5222146641C0DF8012001222146641CEC
:10D650000DF8012004222146641C0DF80120184811
:10D660000068020E2146641C0DF801201448006871
:10D67000C0F307422146641C0DF8012010480088C1
:10D68000C0F307222146641C0DF801200C480278E3
:10D690002146641C0DF80120FF222046611CCCB2FB
:10D6A0000DF8002021466846F4F76AF900BFC4E788
:10D6B000280600202A060020240600202606002036
:10D6C0007C060020C24801202DE9FE4305460E4697
:10D6D0000020009001900290002781460024687885
:10D6E000297800EB01201FFA80F8B8F1000F61DD06
:10D6F000687A297A00EB01201FFA80F94D480088EA
:10D70000814557DB022400BF3EE0E01C295CA01CE1
:10D71000285C01EB00204849098801EB4101474A98
:10D7200002EB41018880601D295C201D285C01EB13
:10D7300000204149098801EB410102EB4101488089
:10D74000E01D295CA01D285C01EB00203A490988F6
:10D7500001EB410122F811003748008800EB40003E
:10D76000114631F810003349088033480088401CC6
:10D770003149088032480088401C3149088004F152
:10D780000800C4B2781CC7B24745BEDBA01C864265
:10D7900010DB285DFF280DD1601C285CFF2809D113
:10D7A000012028490880002027490880274908804F
:10D7B000274908800024B5222146641C0DF8012069
:10D7C00001222146641C0DF8012003222146641C1D
:10D7D0000DF801201F480068020E2146641C0DF858
:10D7E00001201C480068C0F307422146641C0DF864
:10D7F000012018480088C0F307222146641C0DF858
:10D800000120144802782146641C0DF801202A7872
:10D810002146601CC4B20DF801206A782146601CC4
:10D82000C4B20DF8012021466846F4F7A9F8BDE816
:10D83000FE830000220600201E060020B23A0120CE
:10D8400020060020280600202A06002024060020AA
:10D85000260600207C0600202DE9FE430646884669
:10D8600000200090019002900025002700243068DD
:10D87000009070680190B5208DF8000000BF05E0B1
:10D880001DF80500384487B2681C85B2072DF7DB08
:10D89000F8B28DF80700082411480068020E2146EE
:10D8A000641C0DF801200E480068C0F307422146B1
:10D8B000641C0DF801200A480088C0F307222146A5
:10D8C000641C0DF80120064802782146641C0DF8FE
:10D8D000012021466846F4F753F8BDE8FE830000B6
:10D8E0007C0600202DE9FE43064688460020009075
:10D8F0000190029000250027002430680090706895
:10D900000190B5208DF8000000BF05E01DF805006E
:10D91000384487B2681C85B2072DF7DBF8B28DF862
:10D920000700082412480068020E2146641C0DF806
:10D9300001200F480068C0F307422146641C0DF81F
:10D9400001200B480088C0F307222146641C0DF813
:10D950000120074802782146641C0DF80120214669
:10D960006846F4F70DF8F8F74FFBBDE8FE830000BA
:10D970007C0600202DE9FE430746884600200090E3
:10D9800001900290002400250026B5222146641C47
:10D990000DF8012001222146641C0DF8012000220F
:10D9A0002146641C0DF801202146641C0DF801205D
:10D9B0002146641C0DF801202146641C0DF801204D
:10D9C00008222146641C0DF8012000BF05E01DF867
:10D9D0000500304486B2681C85B2072DF7DBF2B231
:10D9E0002046611CCCB20DF8002013480068020EDE
:10D9F0002046611CCCB20DF800200F480068C0F32F
:10DA000007422046611CCCB20DF800200A4800886D
:10DA1000C0F307222046611CCCB20DF80020064856
:10DA200002782046611CCCB20DF8002021466846E1
:10DA3000F3F7A6FFBDE8FE837C0600202DE9FE4338
:10DA4000074688460020009001900290002400259F
:10DA50000026B5222146641C0DF801200122214632
:10DA6000641C0DF8012000222146641C0DF80120E1
:10DA70002146641C0DF801202146641C0DF801208C
:10DA80002146641C0DF8012009222146641C0DF872
:10DA9000012000BF05E01DF80500304486B2681C77
:10DAA00085B2072DF7DBF2B22046611CCCB20DF82F
:10DAB000002013480068020E2046611CCCB20DF80D
:10DAC00000200F480068C0F307422046611CCCB21A
:10DAD0000DF800200A480088C0F307222046611C88
:10DAE000CCB20DF80020064802782046611CCCB26A
:10DAF0000DF8002021466846F3F742FFBDE8FE839B
:10DB00007C0600202DE9F04385B005460E46904680
:10DB100014216846F2F716FE00240027A146B5221C
:10DB20002146641C0DF8012001222146641C0DF8D9
:10DB300001202DB92046611CCCB20DF8002005E073
:10DB400002222046611CCCB20DF80020012D61D1CB
:10DB50006948008802122046611CCCB20DF80020F2
:10DB6000654802782046611CCCB20DF8002063485D
:10DB7000008802122046611CCCB20DF800205F48DC
:10DB800002782046611CCCB20DF800200EBB5C4828
:10DB90000068020E2046611CCCB20DF800205848E7
:10DBA0000068C0F307422046611CCCB20DF800208B
:10DBB00053480088C0F307222046611CCCB20DF800
:10DBC00000204F4802782046611CCCB20DF800209E
:10DBD00014E0EE222046611CCCB20DF80020204655
:10DBE000611CCCB20DF800202046611CCCB20DF8AF
:10DBF00000202046611CCCB20DF8002000222046F7
:10DC0000611CCCB20DF800202046611CCCB20DF88E
:10DC1000008034E0F6B93848008802122046611CC2
:10DC2000CCB20DF80020344802782046611CCCB2FA
:10DC30000DF800203148008802122046611CCCB249
:10DC40000DF800202D4802782046611CCCB20DF85A
:10DC5000002014E0EE222046611CCCB20DF800201A
:10DC60002046611CCCB20DF800202046611CCCB2CD
:10DC70000DF800202046611CCCB20DF800204FF0BA
:10DC80000009002706E01DF8070048441FFA80F944
:10DC9000781C87B2A742F6DB09F0FF022046611C20
:10DCA000CCB20DF8002017480068020E2046611C17
:10DCB000CCB20DF8002013480068C0F3074220469C
:10DCC000611CCCB20DF800200E480088C0F307227A
:10DCD0002046611CCCB20DF800200A48027820468C
:10DCE000611CCCB20DF8002021466846F3F748FECF
:10DCF00005B0BDE8F0830000DE050020E00500204F
:10DD0000E40500207C06002003B40198410000983F
:10DD100050EAC12018BF04204A0D18BF40F001008E
:10DD200040F2FF72B2EB515F08BF40F002000128E1
:10DD300008BF052002B0704710B5B94A2DED020B9F
:10DD40002DED0C8B82B00F9921F000409FEDB6CBEA
:10DD500090422CDBA0F140530E9AA3F17F631A434B
:10DD60000FD0B349884202DC16D10E98A0B19DEDC8
:10DD70000E0B02B0BDEC0C8B02B0BDE8104001F000
:10DD8000CBB90029C1BF9FEDAC0B02B0BDEC0C8B31
:10DD900002B0C8BF10BD16E00120F2F702FD02B0CC
:10DDA000BDEC0C8B02B0BDE8104001F0C1B9A44A33
:10DDB0009FEDA59B9FEDA6AB90425EDAA6499FED35
:10DDC000A8CB814208DBB0EE4C0AF0EE6C0A02B040
:10DDD000BDEC0C8B02B010BD9DED0E0B53EC102B67
:10DDE00051EC100B01F092FD41EC180B9E480621FE
:10DDF000B0EE480AF0EE680A784400F0D1FE53EC29
:10DE0000182B51EC100B01F081FD41EC1B0B9748D6
:10DE1000B0EE480AF0EE680A0421784400F0C0FE33
:10DE200053EC182B51EC100B01F070FD53EC192B37
:10DE300001F0CAFA41EC100B51EC1B0B53EC102B08
:10DE400001F076FB41EC100B53EC102B9DED0E0B0B
:10DE500051EC100B01F05AFD53EC1A2B01F08AFE25
:10DE60009DED0E1B53EC112B01F084FE53EC1C2B8B
:10DE700001F080FE41EC100BA9E79FED7D8B9FED3B
:10DE80007EBB9DED0E0B002953EC192B51EC100BB2
:10DE900052DA01F099FA53EC182B01F037FD41ECFE
:10DEA000180B77480621B0EE480AF0EE680A78446D
:10DEB00000F076FE53EC182B51EC100B01F026FD10
:10DEC00041EC1D0B6F48B0EE480AF0EE680A0421E1
:10DED000784400F065FE53EC182B51EC100B01F068
:10DEE00015FD53EC192B01F06FFA41EC190B51ECB5
:10DEF000180B01F0D7F941EC180B53EC192B51EC2E
:10DF00001D0B01F015FB53EC182B01F0FFFC53EC3B
:10DF10001A2B01F007FF41EC100B51EC180B53ECDE
:10DF2000102B01F051FA53EC1B2B01F0EFFC53ECDA
:10DF30001C2B01F01FFE6DE001F01CFE53EC182BB2
:10DF400001F0E4FC41EC180B01F0ACF941EC1A0BC8
:10DF500000208DED00AB00909DED000B51EC1A0BF5
:10DF600053EC102B01F030FA9DED000B41EC1C0B33
:10DF700053EC102B51EC100B01F0C8FC53EC182B98
:10DF800001F0F8FD53EC1C2B01F0D2FA41EC1C0B14
:10DF90003D48B0EE480AF0EE680A0621784400F0E9
:10DFA000FFFD53EC182B51EC100B01F0AFFC41ECD2
:10DFB0001D0B3648B0EE480AF0EE680A042178449A
:10DFC00000F0EEFD53EC182B51EC100B01F09EFC11
:10DFD00053EC192B01F0F8F941EC100B51EC1D0B2F
:10DFE00053EC102B01F0A4FA53EC1A2B01F08EFC29
:10DFF00053EC1C2B01F0E8F941EC100B53EC102B07
:10E000009DED000B51EC100B01F0DEF953EC1B2BD6
:10E0100001F07CFC41EC100BD9E600000000000090
:10E020000000F03F00000000182D4454FB2109407F
:10E030000000F07F00000000000000000000000071
:10E040000000E03F00000000000000000000F03F82
:10E05000075C143326A6913C0000603C00000000E1
:10E06000182D4454FB21F93F142300002223000003
:10E07000000000000000E03F000000000000004041
:10E080005E2200006C220000702100007E21000052
:10E0900070B59B482DED020B2DED068B079D25F0ED
:10E0A0000044A04218DC9748844202DC0AD106985A
:10E0B00040B19DED060BBDEC068B02B0BDE8704093
:10E0C00001F02AB8002DCCBF9FED8F0B9FED900B78
:10E0D000BDEC068B02B070BD8F48A04215DD8F48A5
:10E0E000A042D8BF4FF0FF3458DD9DED060B51EC38
:10E0F000100BFFF709FE042808BF01F029F89DED79
:10E10000060BBDEC068B02B070BD9DED060B51EC0D
:10E11000100B01F06FF8CDE9060181489FED828B6D
:10E12000A0423CDD8248A0421FDD00249FED82AB6F
:10E130009DED060B53EC1A2B51EC100B01F044F93A
:10E140009DED060B41EC190B53EC1A2B51EC100B07
:10E1500001F0DCFB53EC182B01F0E4FD53EC192B20
:10E1600001F0E6F9CDE9060149E09DED060B012439
:10E1700053EC182B51EC100B01F026F99DED060B1A
:10E1800041EC190B53EC182B51EC100B01F0CAFDAC
:10E1900053EC192B01F0CCF9CDE906012FE06848CA
:10E1A000A0421FDD02249FED689B9DED060B53EC02
:10E1B000192B51EC100B01F0A9FB53EC182B01F0BB
:10E1C00003F99DED060B41EC180B53EC192B51ECA8
:10E1D000100B01F0A7FD53EC182B01F0A9F9CDE9C4
:10E1E00006010CE09DED060B032453EC102B9FED74
:10E1F000580B51EC100B01F09BF9CDE906019DED98
:10E20000060B53EC102B51EC100B01F07FFB41EC93
:10E21000180B53EC182B01F079FB41EC190B4E480D
:10E220000621B0EE490AF0EE690A784400F0B8FC25
:10E2300053EC182B51EC100B01F068FB41EC180B60
:10E240004648B0EE490AF0EE690A0521784400F02C
:10E25000A7FC53EC192B51EC100B01F057FB41ECD0
:10E26000100B51EC180B53EC102B002C0EDA01F0B4
:10E27000ABF89DED061B53EC112B01F047FB9DED18
:10E28000061B53EC112B01F075FC35E001F09CF8F6
:10E290009DED061B53EC112B01F038FB41EC100BEC
:10E2A0002F48784400EBC40090ED001B51EC100B9C
:10E2B00053EC112B01F036FD9DED061B53EC112B99
:10E2C00001F030FD41EC100B2648784400EBC4000F
:10E2D00090ED001B51EC100B53EC112B01F04AFC9C
:10E2E00041EC100B002DA2BFBDEC068B02B070BD3F
:10E2F00051EC100B01F02AF841EC100B01E7000083
:10E30000000010440000F07F182D4454FB21F93F19
:10E31000182D4454FB21F9BF0000DC3F0000203ED3
:10E320000000F33F00000000000000000000F03F8C
:10E330000000E63F00000000000000000000004078
:10E340000080034000000000000000000000F83FD3
:10E35000000000000000F0BF9A1F0000501F0000E6
:10E36000DA1E0000921E000010B52F499FED2C1BF5
:10E370002DED020B84B0059820F000408842D8BFF4
:10E380009DED040B2DDD2949884209D1049840B93F
:10E390004FF00100F2F705FA00F0CAFE06B010BD1A
:10E3A00005DB9DED040B00F0B7FE06B010BD68461E
:10E3B0009DED040B00F020F910F0030004BF9DED6B
:10E3C000021B9DED000B0CD001280ED09DED021B11
:10E3D0009DED000B022817D0012000F05DFC06B077
:10E3E00010BD00F025FB06B010BD9DED021B9DED9C
:10E3F000000B012000F050FC51EC100B00F0A6FFC8
:10E4000006B041EC100B10BD00F012FB51EC100BEC
:10E4100000F09CFF06B041EC100B10BD00000000A6
:10E420000000000000000000FB21E93F0000F07F39
:10E4300010B52F499FED2C1B2DED020B84B00598D4
:10E4400020F000408842DCBF00209DED040B32DD4F
:10E450002849884209D1049840B94FF00100F2F7E9
:10E46000A0F900F065FE06B010BD05DB9DED040BC4
:10E4700000F052FE06B010BD68469DED040B00F0A2
:10E48000BBF810F0030011D0012818D09DED021B3D
:10E490009DED000B02281AD000F0CAFA51EC100BC7
:10E4A00000F054FF06B041EC100B10BD9DED021BB7
:10E4B0009DED000B012000F0EFFB06B010BD9DEDBF
:10E4C000021B9DED000B00F0B3FA06B010BD012059
:10E4D00000F0E2FB51EC100B00F038FF06B041EC0D
:10E4E000100B10BD00000000000000000000000044
:10E4F000FB21E93F0000F07F00B52DED048BB0EE6D
:10E50000409AF0EE609A83B051EC190B01F03EFB9B
:10E5100041EC180B18EE100A18EE901A8DED008BD6
:10E52000002818BF0120084320F00040C0F17F60A0
:10E5300000F1E040C00F14D019EE101A19EE900A45
:10E540008DED009B002918BF0121084320F00040F9
:10E55000C0F17F6000F1E040C00F04BF0120F2F77E
:10E5600020F9B0EE480A03B0F0EE680ABDEC048B67
:10E5700000BD00000000000010B51D499FED1A1BF2
:10E580002DED020B84B0059820F000408842DCBFDE
:10E5900001209DED040B21DD1649884209D1049824
:10E5A00040B94FF00100F2F7FCF800F0C1FD06B0F1
:10E5B00010BD05DB9DED040B00F0AEFD06B010BDF7
:10E5C00068469DED040B00F017F800F001000121F2
:10E5D000A1EB40009DED021B9DED000B00F0F4FB54
:10E5E00006B010BD000000000000000000000000A8
:10E5F000FB21E93F0000F07F2DE9F14F04462DEDAE
:10E60000020B2DED088B8AB09FEDE70B80ED020B1E
:10E61000139EE74826F0004585420ADC9DED120B6B
:10E62000002084ED000B0AB0BDEC088B03B0BDE800
:10E63000F08FE0489FEDE0AB9FEDE1BBA84247DDE6
:10E64000E14F9FEDE39B9FEDE48B9DED120B53ECAF
:10E650001A2B51EC100B002E1CDD01F063FB41EC7A
:10E66000100BBD4208D053EC1B2B51EC100B01F0EA
:10E6700059FBC4E900010BE053EC192B51EC100BD2
:10E6800001F050FB53EC182B01F04CFBC4E90001E6
:10E690000120C8E700F098FE41EC100BBD4208D005
:10E6A00053EC1B2B51EC100B00F08EFEC4E9000163
:10E6B0000BE053EC192B51EC100B00F085FE53ECE2
:10E6C000182B00F081FEC4E900014FF0FF30AAE7EB
:10E6D000C348A84279DB9DED120B51EC100B00F002
:10E6E00089FD41EC180B9FEDC00B53EC102B01F092
:10E6F0000DF99FEDBF1B53EC112B00F065FE01F0EF
:10E700006FF8074601F09BF841EC190B53EC1A2BFC
:10E7100001F0FCF853EC182B01F02CFA41EC180B2B
:10E7200053EC1B2B51EC190B01F0F0F8DFF8C8A2E9
:10E7300041EC100B4FEA15580125FA4453EC102B0D
:10E7400051EC180B01F0EEFA032DC4E900013DD0A5
:10E75000C1F30A5005EB4511A8EB000011398142C5
:10E7600034DA0AEB051BB0EE48AA9BED000BF0EE85
:10E7700068AA53EC102B51EC190B01F0C7F841ECCF
:10E780001B0B51EC1A0B53EC1B2B01F0CBFA41EC99
:10E79000180B51EC1A0B53EC182B01F0C3FA53EC85
:10E7A0001B2B01F0BFFA9BED020B41EC1A0B53EC53
:10E7B000102B51EC190B01F0A9F853EC1A2B01F0B6
:10E7C000B1FA41EC100B6D1CB8E70EE0002EA8BFAB
:10E7D0003846BFF628AF94ED000B51EC100B00F05B
:10E7E000B5FDC4E9000178421DE7C6F3130040F40B
:10E7F000801EC6F30A50A0F2F530471100F01F0545
:10E80000C5F12000DDF848B0089000200690079080
:10E810000520EC467949002D07EB0002794408BF3A
:10E8200051F8221009D051F8223001EB8201AB409F
:10E830004A68089922FA01F11943A1FB0E26A1FBAF
:10E840000B131A449A4234BF0123002303EB06083A
:10E850000CEB8003D3E901A60E448E4234BF0121A4
:10E86000002192448A4411B1924502D903E09245B5
:10E8700001D2012100E00021C3E901A641444CF886
:10E880002010011EA0F10100C4DC029800F100502C
:10E89000850F0298DDE903678000DDF8148000F041
:10E8A000CEFF41EC1A0B304600F0E0FF9FED541B09
:10E8B00053EC112B01F02AF841EC1B0B384600F009
:10E8C000D5FF9FED511B53EC112B01F01FF841ECCC
:10E8D000180B404600F0CAFF9FED4D1B53EC112B67
:10E8E00001F014F841EC190B51EC180B53EC192BF7
:10E8F00000F06AFD53EC1B2B00F066FD53EC1A2B65
:10E9000000F062FDCDE90801002008909DED080BA4
:10E9100053EC1A2B51EC100B01F004FA53EC1B2BA7
:10E9200001F000FA53EC182B01F0FCF953EC192B11
:10E9300001F020F99FED381B53EC112B00F0E6FF9E
:10E940009FED370B41EC180B53EC102B9DED080B92
:10E9500051EC100B00F0DAFF53EC182B00F034FDF3
:10E960009FED310B41EC180B53EC102B9DED080B78
:10E9700051EC100B00F0CAFF53EC182B00F024FDF3
:10E9800041EC100B139810F0004F06D06D4251EC83
:10E99000100B00F0DBFC41EC100B284684ED000B63
:10E9A00041E6000000000000000000000000000040
:10E9B000FB21E93F7CD9024000004054FB21F93F94
:10E9C0003163621A61B4D03DFB21F93F00000000C1
:10E9D0000000601A61B4D03D7370032E8A19A33B06
:10E9E000FB2139410000000083C8C96D305FE43F5E
:10E9F000000000000000E03FEA1A0000381A0000A2
:10EA0000000000000000103E000000000000103C6C
:10EA1000000000000000103A182D4454FB21F93D7D
:10EA20003326A611460B113C00000054FB21F93D92
:10EA300010B52DED040B2DED088B82B0B0EE419A90
:10EA4000F0EE619A0B9820F000449FED4BABB4F1CF
:10EA5000795F11DA9DED0A0B51EC100B00F0C0FE4E
:10EA6000002801BFB0EE4A0AF0EE6A0A02B0BDEC1F
:10EA7000088B04BF04B010BD9DED0A0B53EC102BA6
:10EA800051EC100B00F042FF41EC180B3C48062102
:10EA9000B0EE480AF0EE680A784400F081F853ECD2
:10EAA000182B51EC100B00F031FF9DED0A0B41ECDF
:10EAB0001B0B53EC192B51EC100B00F027FF41EC12
:10EAC000190B53EC1B2B51EC180B00F01FFF53ECF0
:10EAD000192B01F027F99FED2C0B41EC190B53EC8E
:10EAE000102B51EC180B00F011FF41EC100B2848D3
:10EAF000844210DA53EC192B51EC100B01F012F98F
:10EB000053EC1A2B01F036F841EC100B02B0BDECBF
:10EB1000088B04B010BD1F48A042BCBF9FED1E1B58
:10EB20008DED001B06DBA4F5001001900020009085
:10EB30009DED001B51EC100B53EC112B01F0F2F882
:10EB40009DED000B41EC180B53EC102B51EC1A0B04
:10EB500001F0E8F841EC1A0B53EC192B51EC180BAF
:10EB600001F0E0F853EC1A2B01F004F841EC100B23
:10EB7000CCE7000000000000000000000000F03FB3
:10EB80005C17000000000000000000000000E03FF3
:10EB90003333D33F0000E93F000000000000D23FC4
:10EBA00070B504462DED028B4D1E00EBC500B0EE96
:10EBB000408AF0EE608A90ED000B35F0060017D029
:10EBC00053EC182B51EC100B00F0A0FE41EC100B95
:10EBD0006D1E04EBC50090ED001B51EC100B53ECC7
:10EBE000112B00F0F1FB41EC100B35F00600E7D1E2
:10EBF000022D36D0042D1CD0062D1CBFBDEC028B7F
:10EC000070BD53EC182B51EC100B00F07FFE94ED0F
:10EC10000A1B53EC112B00F0D7FB53EC182B00F020
:10EC200075FE94ED081B53EC112B00F0CDFB41EC6D
:10EC3000100B53EC182B51EC100B00F067FE94ED09
:10EC4000061B53EC112B00F0BFFB53EC182B00F00C
:10EC50005DFE94ED040B53EC102B00F0B5FB41EC82
:10EC6000100B53EC182B51EC100B00F04FFE94EDF1
:10EC7000021B53EC112B00F0A7FB53EC182B00F0F8
:10EC800045FE94ED001B53EC112B00F09DFBBDECF9
:10EC9000028B41EC100B70BD31B504462DED040B19
:10ECA0002DED0A8BB0EE41BAF0EE61BA0B989DEDF6
:10ECB0000A0B20F00040B0F1795F0DDA51EC100B37
:10ECC000FFF722F8042808BF00F042FA9DED0A0B76
:10ECD000BDEC0A8B05B030BD53EC102B51EC100B82
:10ECE00000F014FE41EC180B9DED0A0B53EC182BB1
:10ECF00051EC100B00F00AFE41EC190B2C48B0EE61
:10ED0000480AF0EE680A05217844FFF749FF9FEDB5
:10ED10002ACBB0EE40AAF0EE60AA9CB353EC1C2BB9
:10ED200051EC190B00F0F2FD41EC1C0B53EC1A2BCB
:10ED300051EC190B00F0EAFD9FED210B41EC190B92
:10ED400053EC102B51EC1B0B00F0E0FD53EC192B96
:10ED500000F0E8FF53EC182B00F0D8FD53EC1B2B10
:10ED600000F0E0FF53EC1C2B00F0DCFF9DED0A1BD4
:10ED700053EC112B00F0FEFEBDEC0A8B05B041EC0C
:10ED8000100B30BDFFE753EC1A2B51EC180B00F0C1
:10ED9000BDFD53EC1C2B00F017FB53EC192B00F0BE
:10EDA000B5FD9DED0A1B53EC112B00F00DFBE3E7C5
:10EDB000E415000000000000495555555555C5BFE4
:10EDC000000000000000E03FF1B506462DED040B09
:10EDD000BD482DED0C8B8AB0B0EE418AF0EE618A11
:10EDE000179D25F000449FEDBABB9FEDBBCB84423D
:10EDF00008DA9DED160B51EC100B00F0F1FC002829
:10EE000000F0E980B64FA74231DC002D0DDA9DED10
:10EE1000160B51EC100B00F099FACDE9160151ECEC
:10EE2000180B00F093FA41EC180B9FEDAF0B53EC6D
:10EE3000102B9DED160B51EC100B00F09BFE53ECCC
:10EE4000182B9FEDAB0BCDE9040151EC100B00F03A
:10EE500069FF41EC100B53EC102B9DED040B51ECB2
:10EE6000100B00F0B1FA9FEDA48BCDE916019DEDDA
:10EE7000160B53EC102B51EC100B00F047FDCDE9B5
:10EE800004019DED040B53EC102B51EC100B00F022
:10EE90003DFD41EC190B9A480621B0EE490AF0EE0F
:10EEA000690A7844FFF77CFE9648B0EE40DAF0EE4F
:10EEB00060DAB0EE490AF0EE690A06217844FFF7FD
:10EEC0006FFE9DED041B51EC100B53EC112B00F069
:10EED0001DFD9DED040B41EC1A0B53EC102B9DED29
:10EEE000160B51EC100B00F011FD41EC190B53EC1B
:10EEF0001A2B51EC1D0B00F067FA53EC192B00F0A4
:10EF000005FD53EC182B00F05FFA9DED041B53EC4C
:10EF1000112B00F0FBFC53EC182B00F055FA41ECE0
:10EF2000180B9FED790B51EC190B53EC102B00F0E3
:10EF3000EDFC53EC182B00F047FA41EC190B9DED5A
:10EF4000160B53EC192B51EC100B00F03DFA41EC71
:10EF5000180BA74269DC304600F071FC41EC1A0B3B
:10EF600051EC180B53EC1A2B00F02EFA41EC1B0B52
:10EF700053EC182B51EC180B00F0C8FC53EC1B2B76
:10EF800000F0D6FA53EC192B00F0CCFE9DED161BC9
:10EF900053EC112B00F0EEFD9FED5D1B53EC112B9C
:10EFA00000F0B4FC53EC1A2B00F0E4FD41EC180B1C
:10EFB000022000EAA570C0F1010000F040FC53EC13
:10EFC000182B00F0A3FC00BF41EC100B0AB0BDEC05
:10EFD0000C8B05B0F0BD711C1698214308430CD072
:10EFE0009DED160B012E1CBF53EC102B51EC1C0B8E
:10EFF00010D000BF00F09CFAE6E79DED160B51EC37
:10F00000100B00F0F7F841EC100B51EC1B0B53EC1C
:10F01000102BEFE751EC100BFEF776FE042808BF2B
:10F0200000F096F89DED160BD0E7012E04BFB0EE70
:10F03000480AF0EE680AC9D08DED048B00240494D0
:10F040009DED040B53EC102B9DED160B51EC100BAA
:10F0500000F090FD53EC192B00F08CFD41EC190BE6
:10F0600053EC182B51EC1C0B00F062FA41EC180B1E
:10F070008DED008B00949DED040B53EC102B9DED5A
:10F08000000B51EC100B00F041FC53EC1B2B00F07B
:10F090009BF99DED000B41EC1A0B53EC192B51EC35
:10F0A000100B00F033FC53EC1A2B00F08DF953ECED
:10F0B000182B00F02BFC9DED001B53EC112B00F0E6
:10F0C00083F981E7000000000000303E00000000EE
:10F0D000000000000000F03F000000000000F0BF52
:10F0E0002894E53F00000000182D4454FB21E93F1F
:10F0F000075C143326A6813C0000000000000000DD
:10F100007214000088140000635555555555D53FBD
:10F11000000000000000004010B553EC102B51EC33
:10F12000100B00F051F941EC100B10BD0000000075
:10F130009FED050B10B553EC102B51EC100B00F0AC
:10F14000F7F941EC100B10BD0000000000000000BA
:10F150009FED050B10B553EC102B51EC100B00F08C
:10F16000D5FB41EC100B10BD0000000000000010AA
:10F1700000BF8100491E1E4A1268D1628100491EEB
:10F180001B4AD16000BF002112685162891E184AD3
:10F190001268116116490968096841F00101144AB1
:10F1A0001268116000BF12490968096901F0010184
:10F1B0000029F8D000BF0E490968096A41F211120E
:10F1C000114069B90A490968096A9210114039B9B0
:10F1D00007490968096821F00101054A12681160B0
:10F1E00000BF6FF00101024A126811617047000010
:10F1F0004863012082B0CDE9000121F00040019078
:10F200009DED000B02B051EC100B704710B50024BF
:10F21000F4F7B2F80520F4F75DF9FBF7E3FB022001
:10F22000F4F7C2F8F6F756F9F8F77CFEF1F740F973
:10F2300004460523114A00211148F8F70BFF062365
:10F24000104A00211048F8F705FF07230F4A002154
:10F250000F48F8F7FFFE08230E4A00210E48F8F782
:10F26000F9FE09230D4A00210D48F8F7F3FE204668
:10F27000F1F722F9F8F7C8FE002010BD146900204C
:10F28000B159010814A90020A95A010814B9002095
:10F29000E95A010814C90020295B010814D900208B
:10F2A000615C010800B52DED048B83B041EC190BB6
:10F2B00000F06CFC41EC180B18EE100A18EE901AD6
:10F2C0008DED008B002818BF0120084320F000407E
:10F2D000C0F17F6000F1E040C00F14D019EE101AA9
:10F2E00019EE900A8DED009B002918BF01210843FB
:10F2F00020F00040C0F17F6000F1E040C00F04BF8B
:10F300000120F1F74EFA51EC180B03B0BDEC048B61
:10F3100000BD000010B500BF4FF47A600A490968CB
:10F32000C86201460848C16000BF0020064909685C
:10F330004862801E0449096808610348F5F7DEF851
:10F3400008B1F2F767F910BD0C63012081F00041AC
:10F35000704780F00040704721F00041704720F076
:10F360000040704721F00042A2F16052B2F5801FC8
:10F3700001F0004328BFD2F17F6C0BD95FEA001C7B
:10F3800043EAC20242EB507018BF704728BF20F01A
:10F3900001007047B2F5801FBCBF184670474FEAA6
:10F3A000410C1CF5001F02D2084600F01BBE70B5D0
:10F3B00000F056FB00000089FFF7F6BF4FF0004059
:10F3C000A0F580007047000010B591EA030F48BF18
:10F3D00083F0004300F1AE84841A71EB030C05D274
:10F3E000121943EB0C03001B61EB0C01DFF824E165
:10F3F0004FEA1154A4EB135C1EEA430F18BF9EEAB8
:10F40000445F73D023EA0E03DCF1200E21EA04519D
:10F4100043F4801332D322FA0CFE10EB0E0023FAD1
:10F420000CFE41EB0E01CCF1200E03FA0EFE10EBA8
:10F430000E0051F10001B1F5801FCCF1200E32D247
:10F4400001EB045112FA0EF2BDE8104058BF7047AC
:10F45000401C38BF5FEA420218BF7047002814BF43
:10F4600020F0010041F100014FEA410313F5001FB4
:10F4700038BF7047A1F1C04100F040BB012A43EB07
:10F480000302ACF1200CDCF11F0E32BF4FF0000E76
:10F4900023FA0CF310EB030041EB0451B4EB115FC2
:10F4A000D0D0A1EB045101F5801149085FEA30008A
:10F4B00001EB04510ED350F1000038BF12FA0EFEDA
:10F4C00008D1BDE81040C9E7401C38BF5FEA4202DE
:10F4D000CAD1C3E7BDE810404FEA410313F5001F4E
:10F4E00038BF7047A1F1C04100F008BB9EEA445FFD
:10F4F00008D011EA5E0FBDE8104004BF01F00041E2
:10F5000000207047BDE8104070B500F0A9FA00BFB8
:10F5100064FBBE3E0000E0FF491058BFC1F140410E
:10F520005B1058BFC3F140438B42EFF3008070473C
:10F530002DE9C04130B4DFF8A0C23CEA111418BF75
:10F540003CEA131400F0EC8081EA03051CEA111474
:10F5500044EAD57418BF1CEA131500F0C780A4EB69
:10F5600005044FF0004545EAC12145EAC32341EABD
:10F57000505143EA525304F17F74994204F5003428
:10F580004FEAC0204FEAC22208BF904200F09C80A0
:10F590004FEA13650FF24016765D4FEA134506FBFE
:10F5A00005F7C7F1807706FB07F74FEAD737A7FBC8
:10F5B00003687642C8F58038A7FB06CE38BFA8F1AD
:10F5C000010807FB08E64FF0000EA6FB028CE6FBE5
:10F5D00003CEDCF1000CCEF1004E38BFAEF1010ECF
:10F5E000A6FB0C584FF000074FF00005E6FB0E8716
:10F5F000A1FB08C6A0FB07CE16EB0E0645F10005E1
:10F60000E1FB076515F1E04E7EBFA4F580345FEAAB
:10F6100046066D4116F1800745F100054FEA1727B0
:10F620004FEA066647EA0567A6F1DE46B6F1805F57
:10F630004FEA15251FD9384624F0010C05EBC4719B
:10F64000BCF1FE6F01EB0C1102D8F0BCBDE80081EB
:10F6500024425CBF01F5801E9EEAC47F02D4F0BC48
:10F66000BDE80081244238D4F0BCA1F1C041BDE81E
:10F67000004100F043BA4FEAD22242EA43524FEA35
:10F68000D323A7FB02864FEAD02040EA415007FB74
:10F6900003661EEA0E0F4FEAD12105FB026658BF32
:10F6A000A6EB0056B6EB00564FEA520E4EEAC37E6A
:10F6B00018EB0E0E56EB530EBDD518EB02085E414B
:10F6C0007F1C55F10005B6E74FF480154FF0000799
:10F6D0004FF000064FF00008ADE7F0BC4FF000001F
:10F6E00001F1C04101F00041BDE8008111EA0C1FA9
:10F6F0000CEA131500D00CE013EA0C1F00F0258073
:10F700004FF00000F0BC81EA030101F00041BDE8C8
:10F710000081F0BCBDE8004181EA030100F0EEB9D0
:10F72000F0BCBDE8004170B500F09AF9097EFC3EDE
:10F7300000F007B881EA03014FF0000001F000413A
:10F74000704781EA030100F0D9B9F0BCBDE800417F
:10F750004FF0000021497047FFFDFBF9F7F5F4F287
:10F76000F0EEEDEBE9E8E6E4E3E1E0DEDDDBDAD85C
:10F77000D7D5D4D3D1D0CFCDCCCBCAC8C7C6C5C4BA
:10F78000C2C1C0BFBEBDBCBBBAB9B8B7B6B5B4B3D1
:10F79000B2B1B0AFAEADACABAAA9A8A8A7A6A5A4BC
:10F7A000A3A3A2A1A09F9F9E9D9C9C9B9A99999880
:10F7B0009797969595949393929191908F8F8E8E23
:10F7C0008D8C8C8B8B8A89898888878786858584B0
:10F7D00084838382828181800000FF070000F87F9C
:10F7E0004FEA41034FEA5353A3F58063D3F11E035D
:10F7F000C8BFD3F1210C0CDD4FF0004242EAC12218
:10F8000042EA505232FA03FC8CEAE17CACEBE17044
:10F810007047102BC4BF0020704703F5787CBCF103
:10F82000FF3F04D06FF0004282EA2100704770B5BC
:10F8300000F016F94992248000207047F2E710F09A
:10F84000004248BF4042B0FA80F310FA03F10AD0F8
:10F85000C3F11D0303F580634FEA415002EB0352ED
:10F8600002EBD12170474FF000007047B0FA80F3EF
:10F8700010FA03F10AD0C3F11D0303F580634FEAC8
:10F8800041504FEA035202EBD12170474FF0000084
:10F890007047000051EA030C17D41CF5801F58BFB5
:10F8A000BCF5801F00F10680994218BF704708BF61
:10F8B0009042704707D711F5801F58BF13F5801F7E
:10F8C00019D499427047894270471CF5801F08D5AA
:10F8D000BCF5801FF7D58B4218BF704708BF824226
:10F8E00070474FF4001C1CEB410F38BF1CEB430F5B
:10F8F00001D28B42704770B500F0B2F892244900F3
:10F900004FF000514FF08053FFF706BEDFF848C1BB
:10F9100070B51CEA111E1EBF1CEA13159EEA0C0FDF
:10F9200095EA0C0F00F06F8081EA030423EA4C1380
:10F930004EEAD47E21EA4C1141F4801143F4801345
:10F94000AE44A1FB024CA0FB0365AEF17F7E3619ED
:10F9500055EB0C05A1FB034C4CF10003A0FB021C72
:10F9600016EB0C06654153F10003094218BF46F03F
:10F97000010613F4007F0BD14FEA03314FEA053043
:10F98000340341EA155140EA16506FF003020AE0D1
:10F990004FEAC3214FEAC520F40241EA555140EA3B
:10F9A00056506FF0020202EB2E4201EB025585EA3F
:10F9B000CE710AD05FEA440C18BF24F0004450F125
:10F9C000000041F1000120EAD47040F2FE7C624563
:10F9D00000D270BDA84214BF4FF080444FF04044A5
:10F9E000002E08BF0024BEF1806FA8BFA1F1C04166
:10F9F000BDE8704080F282804FF0000001F1C0410C
:10FA000001F0004170479EEA0C0F0CEA131518BF75
:10FA100095EA0C0F06D04FF0000081EA030E0EF0BD
:10FA2000004170BD00F01CF88900013E00F007B8ED
:10FA300000F009B84FEA430C5FEA5C5C08D081EA49
:10FA4000030100F05BB84FEA410C5FEA5C5CF6D161
:10FA50004FF00000014970470000FF070000F87FE9
:10FA60000EF1020E2EF0030E5EF8046B364205D442
:10FA7000012A43EB030515F5001F12D8012841EBBD
:10FA8000010C1CF5001F0CD80ED14FEAD17C15F5E6
:10FA9000001F0CEB4C0C0CF1020C08BF4CEBD37CA0
:10FAA00004E04FF0080C01E04FEAD37C0CEB4C056E
:10FAB00026FA05F606F00706B6F1040C06D20EEBA0
:10FAC000860CBDE870404CF0010C6047DFE80CF09C
:10FAD000090B02024FF000414FF00000A1F5002198
:10FAE00070BD19461046012851EB010418BFD4F52A
:10FAF000001484BF002001F0004170BD0808A0F58B
:10FB000000114FEA3101704753EA010C17D41CF57C
:10FB1000801F58BFBCF5801F00F106808B4218BFC4
:10FB2000704708BF8242704707D713F5801F58BF40
:10FB300011F5801F19D48B4270479B4270471CF50A
:10FB4000801F08D5BCF5801FF7D5994218BF7047B4
:10FB500008BF904270474FF4001C1CEB430F38BFA6
:10FB60001CEB410F01D2994270470FB40CBC03BC8F
:10FB7000FFF7C1BE91EA030F10B581F000413FF5D8
:10FB80002BAC83F0004300F0D5B800002DE9F04124
:10FB900001F5801CBCF5001FC0F2A9804FEA115C82
:10FBA00021EA0C510CF1FD0C41F480115FEA5C0C70
:10FBB0000CF5C07C01D34000494130A4890241EAE0
:10FBC000905187028E0E0A0CA45D04FB04F602FB22
:10FBD00006F6C6F14046A4FB0662F60D46EA42264A
:10FBE00006FB06F4A4FB01235242C3F1404338BF95
:10FBF0005B1EA6FB02420024E6FB0324D20B42EA72
:10FC00004446A6FB0623A1FB02E2A3FB07E4E3FBB9
:10FC100061426442C2F1404E38BFAEF1010EA6FB14
:10FC200004234FF00002E6FB0E32A2FB0346340031
:10FC3000E2FB6264A1FB06E6A4FB07E8E4FB616863
:10FC40007642C8F1405838BFA8F10108A2FB06E48B
:10FC5000A3FB08E5E2FB6854A1FB05E6A7FB04E86B
:10FC6000E1FB648618F1200556F10006A809A8F109
:10FC70001B08B10908F03F08B8F10A0F40EA866096
:10FC80001CD901EB0C51BDE8F08100BFFCF5EEE89A
:10FC9000E2DDD8D3CFCBC7C3C0BDB9B6B4B1AEAC2B
:10FCA000A9A7A5A3A19F9D9B9A9896959392908FA3
:10FCB0008D8C8B898887868584838281A0FB0068F0
:10FCC00000FB01F208EB4208B8EB872807D534188F
:10FCD00058EB0104D5D5401C51F10001D1E7341A8D
:10FCE00078EB0104CDD4401E71F10001C9E75FEA51
:10FCF0004C0C5FEA9C5C0DD105D34FF0000001F085
:10FD00000041BDE8F081BDE8F04170B5FFF7A8FE05
:10FD10006DDBFFBEBDE8F0414FF0000000497047C9
:10FD20000000F87F10B591EA030F48BF83F000434D
:10FD30003FF552AB841A71EB030C07D212198CF009
:10FD4000004C43EB0C03001B61EB0C01DFF8A4E15A
:10FD50004FEA1154A4EB135C1EEA430F18BF9EEA4E
:10FD6000445F00F0B08023EA6E03524221EA04515E
:10FD7000C3EB6E0338BF5B1EDCF1200E25D322FAE5
:10FD80000CFE10EB0E0043FA0CFE41EB0E01CCF121
:10FD9000200E03FA0EFE10EB0E0051F10001CCF123
:10FDA000200E29D412FA0EF201EB0451BDE81040E6
:10FDB00058BF7047401C1CBFB2F1004F704700286D
:10FDC0000CBF491C20F00100704712EB020E43EB00
:10FDD000030218BF4FF0010E4EEA4202ACF1200CB4
:10FDE000DCF11E0E54D943FA0CFE10EB0E0051F15B
:10FDF000FF31CCF11E0ED5D50EF1010E12FA0EFE1A
:10FE0000404141EB010101EB445C5FEA5C5C10D9CD
:10FE100010EBDE7001EB045138BFBEF1004FBDE8BE
:10FE2000104018BF704700280CBF491C20F001008B
:10FE3000704730D24FEAD42C11F5001124F400643D
:10FE40001BD0B1FA81F20B3AA41AA41ED2F12003FE
:10FE5000914030FA03F31943904001EBCC71002C30
:10FE600001EB0451BDE81040A8BF704701F1C0414B
:10FE70004FF0000001F000417047B0FA80F310FA33
:10FE800003F100D110BDE41A173C4805C90AE4E7A4
:10FE900001EB045110BD491001EB0451BDE81040C5
:10FEA0004FEA300002E04FF0000170474A0008BFFF
:10FEB0000042F8D0B2F5001F28BF704701F00041A2
:10FEC0004FF0000070479EEA445F07D011EA5E0FD2
:10FED000BDE8104004BF002100207047BDE810407D
:10FEE00070B5FFF7BDFD00BF40DFF63E83F0004177
:10FEF000104670470000E0FF43004FEAD30C4FEA82
:10FF00003C0C43401FBF40070CF1605113F0FE4F03
:10FF100070471CF0006F03D100200CF000417047C7
:10FF20000CF0004343EA507010B540EACC0000F0FA
:10FF30000EF800BF000000924FEA0001FFF7DEBD9F
:10FF40004FF000414FF00000A1F5002170470EF185
:10FF5000020E2EF0030E5EF8044B244204D44FEA46
:10FF60004102B2F17F4F11D84FEA4003B3F17F4F06
:10FF70000CD80ED14FEAD07CB2F17F4F0CEB4C0C79
:10FF80000CF1020C08BF4CEBD17C04E04FF0080CE4
:10FF900001E04FEAD17C0CEB4C0324FA03F404F0AB
:10FFA0000704B4F1040C06D20EEB840CBDE810403B
:10FFB0004CF0010C6047DFE80CF0070802024FF03C
:10FFC0000040A0F5800010BD0846420018BFD2F1E5
:10FFD000807288BF00F0004010BD4FF04070E1EE2D
:10FFE000100A7047FF2141EAD050C0057047000059
:10FFF00001000200010003000100020001000400F2
:020000040802F0
:1000000001000200010003000100020001000500E0
:1000100001000200010003000100020001000400D1
:1000200001000200010003000100020001000600BF
:1000300001000200010003000100020001000400B1
:1000400001000200010003000100020001000500A0
:100050000100020001000300010002000100040091
:10006000010002000100030001000200010007007E
:100070000100020001000300010002000100040071
:100080000100020001000300010002000100050060
:100090000100020001000300010002000100040051
:1000A000010002000100030001000200010006003F
:1000B0000100020001000300010002000100040031
:1000C0000100020001000300010002000100050020
:1000D0000100020001000300010002000100040011
:1000E00001000200010003000100020001000006FF
:1000F00010160006101600000000000000000102AB
:1001000003040607080900000000010203040000C0
:10011000555555555555C53F7D6FEB0312D6D4BF88
:100120005544880E55C1C93F3B8F68B52882A4BF8E
:1001300088B20175E0EF493F09F7FD0DE13D023F4F
:100140004B2D8A1C273A03C0C88A599CE52A0040D7
:1001500059018D1B6C06E6BF82922EB1C5B8B33F24
:100160004FBB610567ACDD3F182D4454FB21E93FCF
:100170009BF681D20B73EF3F182D4454FB21F93FBE
:10018000E2652F227F2B7A3C075C143326A6813C44
:10019000BDCBF07A8807703C075C143326A6913CEF
:1001A000C4EB98999999C9BF711623FEC671BCBF5B
:1001B0006D9A74AFF2B0B3BF9AFDDE522DDEADBFC3
:1001C0002F6C6A2C44B4A2BF0D5555555555D53FDB
:1001D000FF8300922449C23F6E204CC5CD45B73FF6
:1001E000513DD0A0660DB13FEB0D76244B7BA93F6E
:1001F00011DA22E33AAD903F4C5555555555A53F80
:100200007751C1166CC156BF9015CB19A001FA3EAB
:10021000AD529C804F7E92BEC4B1B4BD9EEE213ED5
:10022000D43888BEE9FAA8BD00004054FB21F93F4C
:100230003163621A61B4D03D0000601A61B4D03DF0
:100240007370032E8A19A33B0000002E8A19A33B6A
:10025000C14920259A837B3900000000000000007E
:100260006E83F9A22915444ED15727FCC0DD34F521
:10027000999562DB4190433CAB6351FE61C5BBDEA7
:100280003A6E24B7E0D24D42EA2E49061C92D109BB
:100290001CEB1DFE3EA729B1F53582E88444BB2E38
:1002A00026709CE9417E5FB439D69139F439538385
:1002B0008B5F849C3B28F9BDFF97F81F0F9805DEE4
:1002C0008B112FEF1F6D0A5ACF7E366DB709CB27E2
:1002D000663F464F2DEA5F9EC7BA27757BF1E5EB77
:1002E000F739073DEA92528AB15FFB6B085D8D1FBB
:1002F000A6F810111111813FD561C119A0012ABFC3
:100300007DFEB157E31DC73EEB9C2B8AE6E55ABE46
:100310007CD5CF5A3AD9E53D7AFE10111111C13F73
:1003200037D60684F464963F280356C9226D6D3F84
:100330000165F2F2D844433FA69237A0887E143F6D
:10034000735360DBCB75F3BEFE41B31BBAA1AB3F69
:1003500093846EE9E326823F1583E0FEC8DB573FB6
:1003600068108D1AF726303FE9A7F0320FB8123F18
:10037000D47ABF74702AFB3E980302080000002064
:10038000A0060000C403010838050208A0060020EA
:1003900008CB010028040108320001031B080001FA
:1003A000000CF30102030405060708090A00010511
:1003B000FE00B90D0A260227A1292008C1814001AB
:1003C000C0804104610C2108E118A11C011A300110
:1003D0001638013660012E70012F6000FF00C0C189
:1003E00001C30302C2C60607C705C5C404CC0C0D71
:1003F000CD0FCFCE0E0ACACB0BC90908C8D8181921
:10040000D91BDBDA1A1EDEDF1FDD1D1CDC14D4D580
:1004100015D71716D6D21213D311D1D010F0303110
:10042000F133F3F23236F6F737F53534F43CFCFDB0
:100430003DFF3F3EFEFA3A3BFB39F9F83828E8E940
:1004400029EB2B2AEAEE2E2FEF2DEDEC2CE42425C0
:10045000E527E7E62622E2E323E12120E0A0606130
:10046000A163A3A26266A6A767A56564A46CACADF0
:100470006DAF6F6EAEAA6A6BAB69A9A86878B8B9A0
:1004800079BB7B7ABABE7E7FBF7DBDBC7CB4747500
:10049000B577B7B67672B2B373B17170B050909150
:1004A000519353529296565797559594549C5C5D30
:1004B0009D5F9F9E5E5A9A9B5B99595898884849C0
:1004C000894B8B8A4A4E8E8F4F8D4D4C8C44848540
:1004D0004587474686824243834181800E6440437C
:1004E000040D6EA7040E1C0110030E1A0146030230
:1004F000151C3712015512C8026C09F4016400641E
:1005000000E8034103031CF401870C0D9DEC51B876
:100510003D0AD7233ECDCCCC3D410411E42F01014F
:100520001D04040512785634121C1210043D4304B5
:08053000000400127A00000033
:040000050801038962
:00000001FF
